:100000000C9455470C9476470C9482D10C94764707
:100010000C9476470C9476470C9476470C9476476C
:100020000C9476470C9476470C9476470C94ADD399
:100030000C9476470C9476470C9419B40C9476473C
:100040000C9476470C9476470C9476470C9476473C
:100050000C9476470C9476470C9476470C9476472C
:100060000C9476470C949CD10C942BD10C9476472D
:100070000C9402CB0C94A4CA0C94E0CA0C9476475E
:100080000C944DD20C9476470C9476470C9476479A
:100090000C9476470C9476470C9476470C947647EC
:1000A0000C9476470C9476470C9476470C94F4BAEB
:1000B0000C9498BB0C9476470C9476470C940AB633
:1000C0000C9476470C9476470C9476470C947647BC
:1000D0000C9476470C9476470C9476470C947647AC
:1000E0000C948FA50C9476470C9476470C94764725
:1000F0000C9476470C9476470C9476470C9476478C
:100100000C94CBBA0C946FBB0C94A2BA0C9446BB63
:100110000C9476470C9476470C9476470C9476476B
:100120000C9476470C9476470C9476470C9476475B
:100130000C9476470C946EB50C9476470C947647E5
:100140000C9476470C9476470C9476470C9476473B
:100150000C9476470C9476470C9485A50C947647BE
:100160000C9476470C9476470C9476470C9476471B
:100170000C9476470C9476470C9476470C9476470B
:100180000C9476470C9476470C9476470C947647FB
:100190000C9476470C9476470C9476470C947647EB
:1001A0000C941DBB0C94C1BB0C9476470C94764701
:1001B0000C94BCB50C9476470C9476470C94764717
:1001C0000C9476470C9476470C9476470C947647BB
:1001D0000C9476470C9476470C9476470C947647AB
:1001E0000C9476470C9476471A7124712E713871ED
:1001F0004371497749774977497749774971497711
:10020000497749774977497749774B7155715F71DC
:1002100069717371497749774977497749774977A0
:100220007D714977D371497749774977497749771C
:1002300049774977127249772E7549774977497717
:10024000497749774977497749772E7549774977CB
:1002500049773F7244724E7258725A7264726F726A
:1002600049777A7249774977B772497749774977F9
:10027000497749774977497749774977497749777E
:100280004977497749774977C172497749774977FB
:10029000497749774977497749774977CB72087326
:1002A00045738E739873B173B173BB73C573CF739A
:1002B000D973E373E873F273FC7347774777477733
:1002C000477747774777477747774777477747773E
:1002D000477747774777477747774777477747772E
:1002E0004777BB73477747774777477747774777AE
:1002F000477747774777477747774777477747770E
:10030000477747774777067410741A7424744777D1
:100310004777477747774777477747774777B17387
:10032000D476937697769F767B767F7687768B7674
:10033000AB76C076C876CC76D0762C77A3769F74D1
:10034000B074C1744977497739740B714977D274A5
:10035000E374F4742E75A273167549774A7449775D
:1003600005755B742E744977497749776C747D7491
:100370008E743BBA43BA4BBA53BA5BBA63BA6BBA20
:1003800073BA5EBDC3BCCBBCD3BCDBBCE3BCEBBCB3
:10039000F3BCFBBC03BD0BBD13BD1BBD23BD2BBDFF
:1003A00043BD43BD43BD43BD43BD43BD43BD43BD4D
:1003B00043BD43BD43BD43BD43BD43BD43BD43BD3D
:1003C00043BD43BD43BD43BD43BD43BD43BD43BD2D
:1003D00043BD43BD43BD43BD43BD43BD43BD43BD1D
:1003E00043BD43BD43BD33BD3BBD084AD73B3BCEB8
:1003F000016E84BCBFFDC12F3D6C74319ABD568324
:100400003DDA3D00C77F11BED9E4BB4C3E916BAADB
:10041000AABE000000803F05A84CCDB2D44EB9382A
:1004200036A9020C50B9918688083CA6AAAA2ABE11
:10043000000000803F07634236B79BD8A71A39688F
:100440005618AEBAAB558C1D3CB7CC5763BD6DED9D
:10045000FD753EF6177231BF000000803F080000B6
:1004600000BE922449123EABAAAA2ABECDCCCC4CE7
:100470003E00000080BEABAAAAAA3E00000000BF5A
:10048000000000803F0000000000084178D3BB431B
:1004900087D1133D190E3CC3BD4282AD2B3E68ECA3
:1004A0008276BED98FE1A93E4C80EFFFBE01C4FF2A
:1004B0007F3F0000000000000C9445AD0C94D55621
:1004C0000C943BBD0C94E7560C94A1630C941DC195
:1004D0000C94E4A60C9497760C9424740C9451CA52
:1004E0000C9473BA0C94955A0C943F720C94EEB918
:1004F0000C9443BD0C94C8760C948F5B0C94D2740E
:100500000C946D5A0C94ED560C9480CF0C94715A47
:100510000C9455710C9412BA0C942BBD0C94167556
:100520000C945B5B0C942C680C94EA5D0C9453BAAD
:100530000C948C470C941A710C9449770C940BBD55
:100540000C9482470C94FE560C9412C20C94915950
:100550000C94095F0C94A15A0C9485570C9493BC8D
:100560000C9478470C943E5D0C94F0A60C945F714B
:100570000C9469710C945EBD0C9441AD0C94625D59
:100580000C946D630C94B9590C94855A0C94CC63FB
:100590000C94915A0C947B5B0C94DB560C9433BDF9
:1005A0000C94FC730C941D570C9405AD0C94C07600
:1005B0000C9417CD0C94D9790C9406BA0C94726EE5
:1005C0000C94EB910C9469CE0C948E740C944E7236
:1005D0000C94775B0C94D05A0C946BBA0C943E57E5
:1005E0000C94E94A0C9438710C948D5A0C941E5852
:1005F0000C945A720C94AB590C94C8560C949D5A96
:100600000C94735B0C949A580C94FBBC0C9421AD25
:100610000C9409570C942E710C94A95E0C942154DF
:100620000C94E1560C94086D0C94F4740C94A55A37
:100630000C944A740C949F740C941A630C94675B2A
:100640000C940EBA0C943C640C94F2B90C942C6B80
:100650000C94F9780C9457570C94EF5A0C94B68379
:100660000C9428570C94B15A0C94D4760C94127FA5
:100670000C94CB470C943DAD0C94655A0C94817846
:100680000C944BBA0C94E3740C94F4570C94DCA6C1
:100690000C94F0AC0C94A0CE0C9408730C944B7199
:1006A0000C945BBA0C94B1730C949DAE0C941074C2
:1006B0000C94DF670C9413BD0C94ACAB0C94437199
:1006C0000C9449AD0C94A8AB0C94B46E0C941263CA
:1006D0000C947D710C9487580C94B0740C94F7B9F9
:1006E0000C94F4A60C9459680C948DBC0C9458721C
:1006F0000C94A6AB0C94E6590C94346B0C941E63CA
:100700000C9464720C94C1720C94795A0C94DBBCF6
:100710000C946E680C94ADB80C94D8A60C94C05987
:100720000C9493760C94E3730C94EB6D0C941BBDBA
:100730000C94BB730C9493B90C94ECA60C947F5B53
:100740000C9445CC0C9483790C9416630C94FBC6E2
:100750000C94575B0C94C7590C9403BD0C948E7386
:100760000C94DC470C943FB90C941A5D0C94D9732B
:100770000C945B740C94D0760C94C05C0C9401794E
:100780000C9498730C947B760C94D3BC0C94C25D3F
:100790000C94817F0C94975B0C94805E0C94605950
:1007A0000C949B770C9444790C94D05E0C947371E8
:1007B0000C94ABCD0C94935B0C94C45D0C94815A57
:1007C0000C94C1740C947A720C9499670C94966092
:1007D0000C9440C70C9412720C9435C10C9474AEF6
:1007E0000C947F760C940B710C948B760C945C813A
:1007F0000C9424710C9447770C9439740C94D97828
:100800000C941CC10C94E0C90C9452C90C94DF6880
:100810000C94055A0C9444720C94895D0C944573A5
:100820000C94CF730C94595E0C94C5730C9405759D
:100830000C94A1B80C946C740C942BB90C940F5EAE
:100840000C94BD570C94615A0C94165D0C946F7205
:100850000C9473620C94BBB90C941A740C94695A7E
:100860000C946CAB0C94A35B0C94755A0C946EAB0B
:100870000C94AE5B0C94E3BC0C9453630C94CC7658
:100880000C94895A0C946EC10C9457620C9459B90B
:100890000C943BBA0C94EAB90C94C1620C94345E8B
:1008A0000C94CBBC0C94A95A0C942E740C94125733
:1008B0000C9433570C9443BA0C94ADBC0C94835BEA
:1008C0000C9408590C9422630C943FCA0C94D4786D
:1008D0000C9405790C94F3560C9416670C94AE792D
:1008E0000C941CCF0C94995A0C9463BA0C94D4A613
:1008F0000C94C3BC0C94A3760C940ABA0C94857F18
:100900000C94F3BC0C94E8730C94066E0C94E8A65B
:100910000C94A2730C94CBD00C9423BD0C94097945
:100920000C942E750C9404640C9417CE0C9451C145
:100930000C94624E0C948B5B0C94635B0C94125B76
:100940000C947D5A0C948C590C94AD5A0C94EBBCBD
:100950000C946B5B0C94875B0C94B7720C94F35AF9
:100960000C947D740C9487760C9487630C946E576A
:100970000C94AB760C94E0A60C94B1BC0C94CB72A6
:100980000C940E680C949F760C9449710C946F5BD8
:100990000C945F5B0C94897F0C94FD780C94F2733B
:1009A0000C9470AB0C9457580C9406740C948B7781
:1009B0000C94B2590C94D3710C94BFC90C9495B893
:1009C0000C94F8A60C942C770C94DDA75B2573256A
:1009D000735D20257320257320706F736974696FB0
:1009E0006E2531382E336625730A005B2573257317
:1009F0005D202573202573206F666673657425322C
:100A0000302E336625730A005B257325735D202520
:100A100073207A65726F206261636B6F6666253141
:100A2000392E336625730A005B257325735D2025F7
:100A300073206C61746368206261636B6F66662506
:100A400031382E336625730A005B257325735D20CC
:100A50002573206C617463682076656C6F636974BC
:100A6000792531332E306625732F6D696E0A005B50
:100A7000257325735D20257320736561726368207B
:100A800076656C6F636974792531322E3066257313
:100A90002F6D696E0A005B257325735D2025732019
:100AA000737769746368206D617825313764205BE2
:100AB000303D6F66662C313D686F6D696E672C3214
:100AC0003D6C696D69742C333D6C696D69742B687C
:100AD0006F6D696E675D0A005B257325735D202568
:100AE0007320737769746368206D696E253137648C
:100AF000205B303D6F66662C313D686F6D696E67B7
:100B00002C323D6C696D69742C333D6C696D697470
:100B10002B686F6D696E675D0A005B257325735DD9
:100B2000202573207261646975732076616C756528
:100B30002532302E346625730A005B257325735DDC
:100B4000202573206A756E6374696F6E2064657604
:100B5000696174696F6E2531342E346625732028DF
:100B60006C61726765722069732066617374657267
:100B7000290A005B257325735D202573206A657241
:100B80006B20686F6D696E672531362E3066257370
:100B90002F6D696E5E33202A2031206D696C6C697F
:100BA0006F6E0A005B257325735D202573206A65CF
:100BB000726B206D6178696D756D2531352E3066EB
:100BC00025732F6D696E5E33202A2031206D696C8C
:100BD0006C696F6E0A005B257325735D2025732099
:100BE00074726176656C206D696E696D756D253105
:100BF000372E336625730A005B257325735D202528
:100C0000732074726176656C206D6178696D756DA5
:100C10002531372E336625730A005B257325735DF6
:100C20002025732076656C6F63697479206D617817
:100C3000696D756D2531312E306625732F6D696EA6
:100C40000A005B257325735D202573206665656446
:100C500072617465206D6178696D756D2531312E15
:100C6000306625732F6D696E0A005B257325735DF1
:100C70002025732061786973206D6F646525313894
:100C8000642025730A005B6D615D20206D696E2014
:100C9000617263207365676D656E742531382E331C
:100CA0006625730A005B736C5D2020736F66742089
:100CB0006C696D697420656E61626C6525313264A2
:100CC0000A005B63745D202063686F7264616C204E
:100CD000746F6C6572616E63652531372E346625DD
:100CE000730A005B6A615D20206A756E6374696FC8
:100CF0006E20616363656C65726174696F6E25381F
:100D00002E306625730A005B6764695D2064656642
:100D100061756C742067636F6465206469737461C6
:100D20006E6365206D6F6465253264205B303D47DE
:100D300039302C313D4739315D0A005B6770615DA8
:100D40002064656661756C742067636F64652070EC
:100D500061746820636F6E74726F6C253364205BFE
:100D6000303D4736312C313D4736312E312C323D26
:100D70004736345D0A005B67636F5D2064656661BA
:100D8000756C742067636F646520636F6F72642095
:100D900073797374656D253364205B312D3620289B
:100DA0004735342D473539295D0A005B67756E5D1F
:100DB0002064656661756C742067636F6465207577
:100DC0006E697473206D6F6465253564205B303DFA
:100DD0004732302C313D4732315D0A005B67706C21
:100DE0005D2064656661756C742067636F6465205F
:100DF000706C616E6525313064205B303D47313762
:100E00002C313D4731382C323D4731395D0A0025C0
:100E10006320776F726B206F66667365743A253155
:100E2000322E336625730A002563206D616368697D
:100E30006E6520706F736E3A2531312E33662573DF
:100E40000A00256320706F736974696F6E3A2531EB
:100E5000352E336625730A00546F6F6C206E756DE6
:100E60006265722020202020202020202025640A76
:100E700000466565642072617465206D6F64653A33
:100E800020202020202025730A0044697374616E9D
:100E90006365206D6F64653A202020202020202586
:100EA000730A0050617468204D6F64653A202020F9
:100EB000202020202020202025730A00506C616E05
:100EC000653A2020202020202020202020202020C3
:100ED0002025730A004D6F74696F6E206D6F646515
:100EE0003A20202020202020202025730A00436F54
:100EF0006F7264696E6174652073797374656D3A9D
:100F000020202025730A00556E6974733A20202032
:100F100020202020202020202020202025730A00AF
:100F2000486F6D696E672073746174653A20202084
:100F3000202020202025730A0046656564686F6CB8
:100F4000642073746174653A20202020202025736A
:100F50000A004D6F74696F6E2073746174653A2076
:100F60002020202020202025730A004379636C650F
:100F70002073746174653A202020202020202020D6
:100F800025730A00526177206D616368696E652080
:100F900073746174653A20202025730A004D6163E3
:100FA00068696E652073746174653A202020202082
:100FB000202025730A004C696E65206E756D626590
:100FC000723A2531302E30660A004665656420721B
:100FD0006174653A2531362E336625732F6D696E3F
:100FE0000A0056656C6F636974793A2531372E3380
:100FF0006625732F6D696E0A0050101F10FF0F4792
:101000003935202D20756E6974732D7065722D72BF
:1010100065766F6C7574696F6E206D6F64650047DF
:101020003934202D20756E6974732D7065722D6DA5
:10103000696E757465206D6F64652028692E652E54
:10104000206665656472617465206D6F6465290052
:10105000473933202D20696E766572736520746977
:101060006D65206D6F6465008C106C104739312000
:101070002D20696E6372656D656E74616C206469A4
:101080007374616E6365206D6F646500473930204D
:101090002D206162736F6C7574652064697374616F
:1010A0006E6365206D6F646500DD10C510AF10477D
:1010B0003634202D20636F6E74696E756F757320E2
:1010C0006D6F6465004736312E31202D20657861C3
:1010D00063742073746F70206D6F646500473631E0
:1010E000202D2065786163742070617468206D6FB5
:1010F00064650017110811F910473139202D205966
:101100005A20706C616E6500473138202D20585A86
:1011100020706C616E6500473137202D20585920B2
:10112000706C616E6500A311911178115711301127
:10113000473830202D2063616E63656C206D6F74BD
:10114000696F6E206D6F646520286E6F6E6520611B
:1011500063746976652900473320202D20636F75FD
:101160006E74657220636C6F636B77697365206161
:101170007263206665656400473220202D20636C11
:101180006F636B7769736520617263206665656460
:1011900000473120202D206C696E656172206665E4
:1011A000656400473020202D206C696E65617220D7
:1011B000747261766572736520287365656B2900AA
:1011C0006A12501236121C120212E811CE11473563
:1011D00039202D20636F6F7264696E6174652073AE
:1011E000797374656D203600473538202D20636F84
:1011F0006F7264696E6174652073797374656D20B4
:101200003500473537202D20636F6F7264696E613A
:1012100074652073797374656D203400473536200A
:101220002D20636F6F7264696E61746520737973CA
:1012300074656D203300473535202D20636F6F7244
:1012400064696E6174652073797374656D20320012
:10125000473534202D20636F6F7264696E61746549
:101260002073797374656D203100473533202D204C
:101270006D616368696E6520636F6F7264696E612A
:1012800074652073797374656D009D1297129012C6
:10129000486F6D696E6700486F6D6564004E6F74CE
:1012A00020486F6D656400D112CC12C712C112BC08
:1012B00012B312456E6420486F6C6400486F6C6412
:1012C00000446563656C00506C616E0053796E6319
:1012D000004F666600E412E012DB12486F6C640097
:1012E00052756E0053746F70000E130413FE12F7E4
:1012F00012F3124A6F6700486F6D696E6700507293
:101300006F6265004D616368696E696E67004F6664
:10131000660044133E13381333132F13291320137D
:1013200053687574646F776E004379636C6500452C
:101330006E640053746F7000416C61726D00526591
:1013400061647900496E697469616C697A696E6774
:1013500000A713A1139B13961392138E1389138363
:10136000137D1376137213691353687574646F7762
:101370006E004A6F6700486F6D696E67004379635E
:101380006C650050726F626500486F6C6400527546
:101390006E00456E640053746F7000416C61726D35
:1013A00000526561647900496E697469616C697A9B
:1013B000696E6700CE13B813473231202D206D6956
:1013C0006C6C696D65746572206D6F646500473281
:1013D00030202D20696E63686573206D6F64650031
:1013E0000814FD13F113E8135B7261646975735D92
:1013F000005B696E686962697465645D005B737443
:10140000616E646172645D005B64697361626C65E6
:10141000645D0022141E1419142064656700206D99
:101420006D0020696E002A2A2A204E4F54494345F8
:10143000202A2A2A20526573657474696E672062B7
:10144000617564207261746520746F202573005B80
:10145000626175645D20555342206261756420723B
:1014600061746525313564205B313D393630302C6F
:10147000323D31393230302C333D33383430302C3A
:10148000343D35373630302C353D31313532303022
:101490002C363D3233303430305D0A005B72786D6B
:1014A0005D2073657269616C205258206D6F6465B0
:1014B00025313564205B303D636861725F6D6F6418
:1014C000652C313D6C696E655F6D6F64655D0A000A
:1014D0005B65785D2020656E61626C6520666C6F6F
:1014E0007720636F6E74726F6C25313064205B30CF
:1014F0003D6F66662C313D584F4E2F584F46462C57
:10150000323D5254532F4354535D0A005B65655D71
:101510002020656E61626C65206563686F253138D7
:1015200064205B303D6F66662C313D6F6E5D0A0056
:101530005B65635D2020657870616E64204C462099
:10154000746F2043524C46206F6E205458253664E9
:10155000205B303D6F66662C313D6F6E5D0A0092F8
:10156000158D15871581157B1574156D1532333062
:1015700034303000313135323030003537363030AC
:1015800000333834303000313932303000393630C1
:1015900030003000737973006662000000000702BB
:1015A000F978895DC25DE0398F22DC43737973007D
:1015B0006676000000000703FD78895DC25DE439AE
:1015C000EC51783F737973006870000000000700E9
:1015D0000179895DD05EEC390000803F737973003A
:1015E00068760000000007000579895DD978F03938
:1015F000000000417379730069640000000004007A
:1016000009798178C25DDC3900000000000000002B
:101610006E00000000000100615A5757805E5B3287
:1016200000000000000000006C696E650000010011
:10163000615A6E57805E5B320000000000000000BF
:1016400076656C0000000002C7598557C25DDC3921
:1016500000000000000000006665656400000002F4
:10166000E659BD57C25DDC390000000000000000F3
:101670007374617400000000655AC856C25DDC399D
:1016800000000000000000006D61637300000000B6
:10169000695AD556C25DDC39000000000000000028
:1016A00063796373000000006D5ADB56C25DDC395C
:1016B00000000000000000006D6F74730000000067
:1016C000715AE156C25DDC390000000000000000E4
:1016D000686F6C6400000000755AE756C25DDC3923
:1016E0000000000000000000756E6974000000003A
:1016F0007D5AF356C25DDC39000000000000000096
:10170000636F6F7200000000815AFE56C25DDC39C3
:1017100000000000000000006D6F6D6F0000000011
:10172000855A0957C25DDC39000000000000000046
:10173000706C616E00000000895A1257C25DDC397E
:1017400000000000000000007061746800000000EC
:101750008D5A1D57C25DDC390000000000000000FA
:101760006469737400000000915A2857C25DDC3927
:10177000000000000000000066726D6F00000000B5
:10178000955A3357C25DDC390000000000000000AC
:10179000746F6F6C00000000995A3E57C25DDC39CF
:1017A000000000006D706F006D706F780000000326
:1017B000A35B1E58C25DDC39000000006D706F0035
:1017C0006D706F7900000003A35B1E58C25DDC39A9
:1017D000000000006D706F006D706F7A00000003F4
:1017E000A35B1E58C25DDC39000000006D706F0005
:1017F0006D706F6100000003A35B1E58C25DDC3991
:10180000000000006D706F006D706F6200000003DB
:10181000A35B1E58C25DDC39000000006D706F00D4
:101820006D706F6300000003A35B1E58C25DDC395E
:1018300000000000706F7300706F73780000000389
:10184000975BF457C25DDC3900000000706F7300D5
:10185000706F737900000003975BF457C25DDC3949
:1018600000000000706F7300706F737A0000000357
:10187000975BF457C25DDC3900000000706F7300A5
:10188000706F736100000003975BF457C25DDC3931
:1018900000000000706F7300706F7362000000033F
:1018A000975BF457C25DDC3900000000706F730075
:1018B000706F736300000003975BF457C25DDC39FF
:1018C000000000006F6673006F667378000000030D
:1018D000AE5B5758C25DDC39000000006F667300D4
:1018E0006F66737900000003AE5B5758C25DDC3948
:1018F000000000006F6673006F66737A00000003DB
:10190000AE5B5758C25DDC39000000006F667300A3
:101910006F66736100000003AE5B5758C25DDC392F
:10192000000000006F6673006F66736200000003C2
:10193000AE5B5758C25DDC39000000006F66730073
:101940006F66736300000003AE5B5758C25DDC39FD
:1019500000000000686F6D00686F6D65000000009A
:10196000795AED569159DC3900000000686F6D001E
:10197000686F6D7800000000975B1A5DC25D3032C1
:1019800000000000686F6D00686F6D790000000056
:10199000975B1A5DC25D313200000000686F6D0018
:1019A000686F6D7A00000000975B1A5DC25D32328D
:1019B00000000000686F6D00686F6D61000000003E
:1019C000975B1A5DC25D333200000000686F6D00E6
:1019D000686F6D6200000000975B1A5DC25D343273
:1019E00000000000686F6D00686F6D63000000000C
:1019F000975B1A5DC25D35320000000070726200B4
:101A000070726265000000001CC11A5DC25D363252
:101A100000000000707262007072627800000003C3
:101A20001CC1895DC25D3732000000007072620027
:101A300070726279000000031CC1895DC25D3B3297
:101A400000000000707262007072627A0000000391
:101A50001CC1895DC25D3F320000000070726200EF
:101A600070726261000000031CC1895DC25D433277
:101A70000000000070726200707262620000000379
:101A80001CC1895DC25D47320000000070726200B7
:101A900070726263000000031CC1895DC25D4B323D
:101AA000000000006A6F67006A6F6778000000003E
:101AB0001CC1165DAB595532000000006A6F67000B
:101AC0006A6F6779000000001CC1165DB25955327B
:101AD000000000006A6F67006A6F677A000000000C
:101AE0001CC1165DB9595532000000006A6F6700CD
:101AF0006A6F6761000000001CC1165DC059553255
:101B000000000000707772007077723100000000F2
:101B100012BA3FB9C25DDC39000000007077720074
:101B2000707772320000000012BA3FB9C25DDC3932
:101B300000000000707772007077723300000000C0
:101B400012BA3FB9C25DDC39000000007077720044
:101B5000707772340000000012BA3FB9C25DDC3900
:101B60000000000031000000316D61000000030042
:101B7000EEB91A5DC45D5E580000404031000000BF
:101B80003173610000000303F2B9895D95B86958AB
:101B90006666E63F310000003174720000000B04FD
:101BA000F7B9895DA1B86D580000B4433100000059
:101BB000316D69000000030006BA1A5DADB85F58C8
:101BC000000000413100000031706F000000030090
:101BD0000ABA1A5DEA5D63580000803F31000000D8
:101BE00031706D00000003000EBA1A5D2BB9645805
:101BF0000000004032000000326D61000000030070
:101C0000EEB91A5DC45D7D5800000040320000004E
:101C10003273610000000303F2B9895D95B88858FA
:101C20006666E63F320000003274720000000B046A
:101C3000F7B9895DA1B88C585C8F22413200000051
:101C4000326D69000000030006BA1A5DADB87E5817
:101C5000000000413200000032706F0000000300FD
:101C60000ABA1A5DEA5D82580000803F3200000027
:101C700032706D00000003000EBA1A5D2BB9835854
:101C80000000004033000000336D610000000300DD
:101C9000EEB91A5DC45D9C580000803F330000001F
:101CA0003373610000000303F2B9895D95B8A7584A
:101CB0006666E63F330000003374720000000B04D8
:101CC000F7B9895DA1B8AB585C8F224133000000A1
:101CD000336D69000000030006BA1A5DADB89D5867
:101CE000000000413300000033706F00000003006B
:101CF0000ABA1A5DEA5DA1580000803F3300000077
:101D000033706D00000003000EBA1A5D2BB9A258A3
:101D10000000004034000000346D6100000003004A
:101D2000EEB91A5DC45DBB5800000000340000002D
:101D30003473610000000303F2B9895D95B8C65899
:101D40006666E63F340000003474720000000B0445
:101D5000F7B9895DA1B8CA585C8F224134000000F0
:101D6000346D69000000030006BA1A5DADB8BC58B6
:101D7000000000413400000034706F0000000300D8
:101D80000ABA1A5DEA5DC058000000003400000085
:101D900034706D00000003000EBA1A5D2BB9C158F3
:101DA000000000407800000078616D000000030032
:101DB000125B87589A58EC300000803F7800000092
:101DC00078766D0000000B005B5B895DC162F130CD
:101DD0000080BB44780000007866720000000B00B1
:101DE000575B895DC162ED300080BB447800000024
:101DF00078746E0000000B03635B895DC162F9308B
:101E0000000000007800000078746D0000000B03F3
:101E10005F5B895DC162F53000000A437800000015
:101E2000786A6D0000000B00675B895D0859FD3022
:101E30000000FA4378000000786A680000000B0098
:101E40006B5B895D6059013100007A4478000000C5
:101E5000786A640000000B046F5B895DC162093120
:101E60000AD7233C7800000078736E00000003005E
:101E7000775B1A5D93BC10300000803F7800000053
:101E800078737800000003007B5B1A5D93BC11300F
:101E900000000000780000007873760000000B005E
:101EA0007F5B895DC16211310000FA437800000058
:101EB000786C760000000B00835B895DC162153190
:101EC0000000C84178000000786C620000000B033D
:101ED000875B895DC16219310000A0407800000075
:101EE000787A620000000B038B5B895DC1621D3153
:101EF000000000007900000079616D00000003001F
:101F0000125B87589A5821310000803F7900000009
:101F100079766D0000000B005B5B895DC162263144
:101F20000080BB44790000007966720000000B005D
:101F3000575B895DC16222310080BB44790000009B
:101F400079746E0000000B03635B895DC1622E3102
:101F5000000000007900000079746D0000000B03A0
:101F60005F5B895DC1622A310000E64279000000B2
:101F7000796A6D0000000B00675B895D085932319A
:101F80000000FA4379000000796A680000000B0045
:101F90006B5B895D6059363100007A44790000003E
:101FA000796A640000000B046F5B895DC1623E3199
:101FB0000AD7233C7900000079736E00000003000B
:101FC000775B1A5D93BC12300000803F79000000FF
:101FD00079737800000003007B5B1A5D93BC1330BB
:101FE00000000000790000007973760000000B000B
:101FF0007F5B895DC16246310000FA4379000000D1
:10200000796C760000000B00835B895DC1624A3108
:102010000000C84179000000796C620000000B03E9
:10202000875B895DC1624E310000A04079000000ED
:10203000797A620000000B038B5B895DC1625231CB
:10204000000040407A0000007A616D00000003004B
:10205000125B87589A5856310000803F7A00000082
:102060007A766D0000000B005B5B895DC1625B31BD
:102070000080BB447A0000007A66720000000B000A
:10208000575B895DC16257310080BB447A00000014
:102090007A746E0000000B03635B895DC16263317B
:1020A00000008CC27A0000007A746D0000000B03FF
:1020B0005F5B895DC1625F31000000007A00000053
:1020C0007A6A6D0000000B00675B895D0859673113
:1020D0000000FA437A0000007A6A680000000B00F2
:1020E0006B5B895D60596B3100007A447A000000B7
:1020F0007A6A640000000B046F5B895DC162733112
:102100000AD7233C7A0000007A736E0000000300B7
:10211000775B1A5D93BC1430000000007A00000069
:102120007A737800000003007B5B1A5D93BC153066
:102130000000803F7A0000007A73760000000B00F8
:102140007F5B895DC1627B310000FA437A00000049
:102150007A6C760000000B00835B895DC1627F3181
:102160000000C8417A0000007A6C620000000B0396
:10217000875B895DC16283310000A0407A00000066
:102180007A7A620000000B038B5B895DC162873144
:10219000000000006100000061616D0000000300AC
:1021A000125B87589A588B31000040406100000054
:1021B00061766D00000003005B5B895DD05E90314D
:1021C0000000B4446100000061667200000003007A
:1021D000575B895DD05E8C310000B4446100000023
:1021E00061746E0000000303635B895DC162983116
:1021F000000080BF6100000061746D0000000303F7
:102200005F5B895DD05E9431000080BF610000009B
:10221000616A6D0000000300675B895D08599C31AD
:102220000000FA4361000000616A680000000300DA
:102230006B5B895D6059A0310000FA4361000000CA
:10224000616A6400000003046F5B895DD05EA831A1
:102250000AD7233C610000006172610000000B039B
:10226000735B895DD05EAC31CF2E654261000000AA
:1022700061736E0000000300775B1A5D93BC16303B
:102280000000803F610000006173780000000300DF
:102290007B5B1A5D93BC17300000000061000000FA
:1022A00061737600000003007F5B895DD05EB03112
:1022B0000000164461000000616C7600000003001D
:1022C000835B895DD05EB4310000C84261000000CC
:1022D000616C620000000303875B895DD05EB831EA
:1022E0000000A04061000000617A6200000003036A
:1022F0008B5B895DD05EBC31000000406200000055
:1023000062616D0000000300125B87589A58C0316B
:10231000000000006200000062766D000000030013
:102320005B5B895DD05EC5310000B4446200000093
:102330006266720000000300575B895DD05EC131A8
:102340000000B4446200000062746E0000000303E9
:10235000635B895DC162CD31000080BF6200000017
:1023600062746D00000003035F5B895DD05EC9315C
:10237000000080BF62000000626A6D000000030080
:10238000675B895D0859D1310000FA4362000000A3
:10239000626A6400000003006F5B895DD05EDD311E
:1023A0000AD7233C620000006272610000000B0348
:1023B000735B895DD05EE131CF2E65426300000022
:1023C00063616D0000000300125B87589A58F53175
:1023D000000000006300000063766D000000030051
:1023E0005B5B895DD05EFA310000B444630000009D
:1023F0006366720000000300575B895DD05EF631B2
:102400000000B4446300000063746E000000030326
:10241000635B895DC1620232000080BF630000001F
:1024200063746D00000003035F5B895DD05EFE3165
:10243000000080BF63000000636A6D0000000300BD
:10244000675B895D085906320000FA4363000000AB
:10245000636A6400000003006F5B895DD05E123226
:102460000AD7233C630000006372610000000B0385
:10247000735B895DD05E1632CF2E654270310000ED
:102480007031667271000300D4A6895DD05E3A5740
:102490000000C84270310000703163736C000300AB
:1024A000D8A6895DD05E3E5700E0F6457031000049
:1024B0007031637368000300DCA6895DD05E42570B
:1024C0000000484670310000703163706C000303F7
:1024D000E0A6895DD05E4657B81E053E703100000B
:1024E0007031637068000303E4A6895DD05E4A57CB
:1024F0007B142E3E70310000703177736C00030046
:10250000E8A6895DD05E4E570000000070310000E3
:102510007031777368000300ECA6895DD05E525776
:102520000000000070310000703177706C00030310
:10253000F0A6895DD05E5657CDCCCC3D7031000001
:102540007031777068000303F4A6895DD05E5A5736
:10255000CDCCCC3D703100007031706F660003034C
:10256000F8A6895DD05E5E57CDCCCC3D6735340092
:102570006735347800000B038F5B895DC1625C3086
:1025800000000000673534006735347900000B0324
:102590008F5B895DC16260300000000067353400E8
:1025A0006735347A00000B038F5B895DC16264304C
:1025B00000000000673534006735346100000B030C
:1025C0008F5B895DC16268300000000067353400B0
:1025D0006735346200000B038F5B895DC1626C302C
:1025E00000000000673534006735346300000B03DA
:1025F0008F5B895DC1627030000000006735350077
:102600006735357800000B038F5B895DC1627430DC
:1026100000000000673535006735357900000B0391
:102620008F5B895DC162783000000000673535003E
:102630006735357A00000B038F5B895DC1627C30A2
:1026400000000000673535006735356100000B0379
:102650008F5B895DC1628030000000006735350006
:102660006735356200000B038F5B895DC162843082
:1026700000000000673535006735356300000B0347
:102680008F5B895DC16288300000A0C1673536006C
:102690006735367800000B038F5B895DC1628C3033
:1026A00000000000673536006735367900000B03FF
:1026B0008F5B895DC1629030000000006735360095
:1026C0006735367A00000B038F5B895DC1629430F9
:1026D00000000000673536006735366100000B03E7
:1026E0008F5B895DC162983000000000673536005D
:1026F0006735366200000B038F5B895DC1629C30D9
:1027000000000000673536006735366300000B03B4
:102710008F5B895DC162A030000000006735370023
:102720006735377800000B038F5B895DC162A43089
:1027300000000000673537006735377900000B036C
:102740008F5B895DC162A8300000000067353700EB
:102750006735377A00000B038F5B895DC162AC304F
:1027600000000000673537006735376100000B0354
:102770008F5B895DC162B0300000000067353700B3
:102780006735376200000B038F5B895DC162B4302F
:1027900000000000673537006735376300000B0322
:1027A0008F5B895DC162B83000000000673538007A
:1027B0006735387800000B038F5B895DC162BC30E0
:1027C00000000000673538006735387900000B03DA
:1027D0008F5B895DC162C030000000006735380042
:1027E0006735387A00000B038F5B895DC162C430A6
:1027F00000000000673538006735386100000B03C2
:102800008F5B895DC162C830000000006735380009
:102810006735386200000B038F5B895DC162CC3085
:1028200000000000673538006735386300000B038F
:102830008F5B895DC162D0300000000067353900D0
:102840006735397800000B038F5B895DC162D43036
:1028500000000000673539006735397900000B0347
:102860008F5B895DC162D830000000006735390098
:102870006735397A00000B038F5B895DC162DC30FC
:1028800000000000673539006735396100000B032F
:102890008F5B895DC162E030000000006735390060
:1028A0006735396200000B038F5B895DC162E430DC
:1028B00000000000673539006735396300000B03FD
:1028C0008F5B895DC162E83000000000673932002B
:1028D00067393278000001038F5B895DC25DCD32BC
:1028E00000000000673932006739327900000103C7
:1028F0008F5B895DC25DD132000000006739320014
:102900006739327A000001038F5B895DC25DD53281
:1029100000000000673932006739326100000103AE
:102920008F5B895DC25DD9320000000067393200DB
:1029300067393262000001038F5B895DC25DDD3261
:10294000000000006739320067393263000001037C
:102950008F5B895DC25DE1320000000067323800A4
:102960006732387800000103935B895DC25DE53210
:102970000000000067323800673238790000010338
:10298000935B895DC25DE932000000006732380068
:102990006732387A00000103935B895DC25DED32D6
:1029A0000000000067323800673238610000010320
:1029B000935B895DC25DF132000000006732380030
:1029C0006732386200000103935B895DC25DF532B6
:1029D00000000000673238006732386300000103EE
:1029E000935B895DC25DF9320000000067333000FF
:1029F0006733307800000103935B895DC25DFD326F
:102A000000000000673330006733307900000103B5
:102A1000935B895DC25D01330000000067333000C5
:102A20006733307A00000103935B895DC25D053333
:102A3000000000006733300067333061000001039D
:102A4000935B895DC25D093300000000673330008D
:102A50006733306200000103935B895DC25D0D3313
:102A6000000000006733300067333063000001036B
:102A7000935B895DC25D1133000000006A696400E8
:102A80006A696461000000001CC1625DA95E063ACB
:102A9000000000006A6964006A6964620000000066
:102AA0001CC1625DA95E0A3A000000006A69640008
:102AB0006A696463000000001CC1625DA95E0E3A91
:102AC000000000006A6964006A6964640000000034
:102AD0001CC1625DA95E123A0000000073797300A8
:102AE0006A61000000000F00B15A895DC1622A309E
:102AF0000050C347737973006374000000000F0433
:102B0000D05A895DC1622E300AD7233C7379730095
:102B1000736C000000000700EF5A1A5DC45D32308C
:102B20000000000073797300737400000000070058
:102B3000ADBC1A5D8DBC05300000803F7379730019
:102B40006D74000000000702EAB9895D59B95A584E
:102B500000000040000000006D6500000000000063
:102B60001DC1BBB9BBB9DC3900000000000000008A
:102B70006D640000000000001DC193B993B9DC39F9
:102B80000000000073797300656A00000000070010
:102B9000817F1A5DEA5DF8390000803F7379730028
:102BA0006A76000000000700857F1A5D127FCC3C2A
:102BB00000004040737973006A7300000000070052
:102BC000897F1A5DEA5DCE3C0000803F7379730017
:102BD000747600000000070012C21A5DEA5DCD594C
:102BE0000000803F737973007176000000000700D9
:102BF00049AD1A5D345E935700000000737973008D
:102C00007376000000000700ACAB1A5D0F5EA057A2
:102C10000000803F737973007369000000000700B3
:102C2000A8AB3E5D70ABA15700007A437379730087
:102C3000656300000000070012631A5DCC63E22F99
:102C40000000000073797300656500000000070054
:102C500016631A5D3C64E32F000000007379730073
:102C600065780000000007001A631A5D0464E42F11
:102C70000000803F7379730072786D0000000700D8
:102C80001E631A5DEA5DE52F0000803F73797300D3
:102C9000626175640000040022631A5D7362E02FB4
:102CA0000000A0400000000073720000000000005F
:102CB000A6AB6CAB6EABDC3900000000000000007E
:102CC00071720000000000003DADF0ACC25DDC3967
:102CD000000000000000000071690000000000001A
:102CE00041AD05ADC25DDC39000000000000000010
:102CF000716F00000000000045AD21ADC25DDC3900
:102D000000000000000000006572000000000000EC
:102D10001CC1DDA7C25DDC3900000000000000001E
:102D200071660000000000001CC1165D8C59DC3982
:102D300000000000000000007278000000000000A9
:102D400051C15762C25DDC39000000000000000084
:102D50006D736700000000001DC1165DC25DDC39A7
:102D60000000000000000000636C6561720000005C
:102D70001CC1624E624EDC39000000000000000001
:102D800074657374000000001CC18379B1BCDC3928
:102D900000000000000000006465666100000000A3
:102DA0001CC1AE79C05CDC390000000000000000EE
:102DB000626F6F74000000001CC1D979D478DC39CF
:102DC000000000000000000068656C70000000005A
:102DD0001CC14479C25DDC39000000000000000025
:102DE00068000000000000001CC14479C25DDC39AD
:102DF000000000007379730067706C00000007002A
:102E00009D5A1A5D0F5E4030000000007379730018
:102E100067756E0000000700A15A1A5DEA5D413037
:102E20000000803F7379730067636F000000070044
:102E3000A55A1A5DC45D3F300000004073797300ED
:102E40006770610000000700A95A1A5D0F5E4230EA
:102E50000000004073797300676469000000070098
:102E6000AD5A1A5DEA5D433000000000000000002A
:102E700067630000000000001CC18B779B77DC3982
:102E800000000000000000006D61000000000B0465
:102E9000F35A895DC1623730CDCCCC3D00000000D3
:102EA000666400000000030035C11A5DEA5DCD3C98
:102EB000000000007564610075646130000003006B
:102EC00051C1625DA95E983900000000756461001F
:102ED000756461310000030051C1625DA95E9C39D7
:102EE0000000000075646100756461320000030039
:102EF00051C1625DA95EA0390000000075646100E7
:102F0000756461330000030051C1625DA95EA4399C
:102F10000000000075646200756462300000030008
:102F200051C1625DA95EA8390000000075646200AD
:102F3000756462310000030051C1625DA95EAC3965
:102F400000000000756462007564623200000300D6
:102F500051C1625DA95EB039000000007564620075
:102F6000756462330000030051C1625DA95EB4392B
:102F700000000000756463007564633000000300A6
:102F800051C1625DA95EB83900000000756463003C
:102F9000756463310000030051C1625DA95EBC39F4
:102FA0000000000075646300756463320000030074
:102FB00051C1625DA95EC039000000007564630004
:102FC000756463330000030051C1625DA95EC439BA
:102FD0000000000075646400756464300000030044
:102FE00051C1625DA95EC8390000000075646400CB
:102FF000756464310000030051C1625DA95ECC3983
:103000000000000075646400756464320000030011
:1030100051C1625DA95ED039000000007564640092
:10302000756464330000030051C1625DA95ED43948
:10303000000000005F7465005F74657800000002A6
:103040006EC1895DC25D0355000000005F746500BC
:103050005F746579000000026EC1895DC25D07552D
:10306000000000005F7465005F74657A0000000274
:103070006EC1895DC25D0B55000000005F74650084
:103080005F746561000000026EC1895DC25D0F550D
:10309000000000005F7465005F746562000000025C
:1030A0006EC1895DC25D1355000000005F7465004C
:1030B0005F746563000000026EC1895DC25D1755D3
:1030C000000000005F7472005F74727800000002FC
:1030D0006EC1895DC25D2856000000005F747200F9
:1030E0005F747279000000026EC1895DC25D2C566A
:1030F000000000005F7472005F74727A00000002CA
:103100006EC1895DC25D3056000000005F747200C0
:103110005F747261000000026EC1895DC25D345649
:10312000000000005F7472005F74726200000002B1
:103130006EC1895DC25D3856000000005F74720088
:103140005F747263000000026EC1895DC25D3C560F
:10315000000000005F7473005F74733100000002B0
:103160006EC1895DC25D9355000000005F70730001
:103170005F707331000000026EC1895DC25DA355AE
:10318000000000005F6373005F63733100000002A2
:103190006EC1895DC25DB355000000005F657300BC
:1031A0005F657331000000026EC1895DC25DC35569
:1031B000000000005F7873005F7873310000000248
:1031C0006EC1895DC25DF558000000005F66650054
:1031D0005F666531000000026EC1895DC25DD35536
:1031E000000000005F7473005F747332000000021F
:1031F0006EC1895DC25D9755000000005F7073006D
:103200005F707332000000026EC1895DC25DA75518
:10321000000000005F6373005F6373320000000210
:103220006EC1895DC25DB755000000005F65730027
:103230005F657332000000026EC1895DC25DC755D3
:10324000000000005F7873005F78733200000002B6
:103250006EC1895DC25D0D59000000005F666500AA
:103260005F666532000000026EC1895DC25DD755A0
:10327000000000005F7473005F747333000000028D
:103280006EC1895DC25D9B55000000005F707300D8
:103290005F707333000000026EC1895DC25DAB5583
:1032A000000000005F6373005F637333000000027F
:1032B0006EC1895DC25DBB55000000005F65730093
:1032C0005F657333000000026EC1895DC25DCB553E
:1032D000000000005F7873005F7873330000000225
:1032E0006EC1895DC25D2559000000005F66650002
:1032F0005F666533000000026EC1895DC25DDB550B
:10330000000000005F7473005F74733400000002FB
:103310006EC1895DC25D9F55000000005F70730043
:103320005F707334000000026EC1895DC25DAF55ED
:10333000000000005F6373005F63733400000002ED
:103340006EC1895DC25DBF55000000005F657300FE
:103350005F657334000000026EC1895DC25DCF55A8
:10336000000000005F7873005F7873340000000293
:103370006EC1895DC25D3D59000000005F66650059
:103380005F666534000000026EC1895DC25DDF5575
:1033900000000000000000005F64616D000000009C
:1033A0001CC1055A055ADC3900000000000000006D
:1033B00073653030000002001CC13E5D595EAC57A1
:1033C00000000000000000007365303100000200C2
:1033D0001CC13E5D595EAE570000000000000000B9
:1033E00073653032000002001CC13E5D595EB0576B
:1033F0000000000000000000736530330000020090
:103400001CC13E5D595EB257000000000000000084
:1034100073653034000002001CC13E5D595EB45734
:10342000000000000000000073653035000002005D
:103430001CC13E5D595EB657000000000000000050
:1034400073653036000002001CC13E5D595EB857FE
:10345000000000000000000073653037000002002B
:103460001CC13E5D595EBA5700000000000000001C
:1034700073653038000002001CC13E5D595EBC57C8
:1034800000000000000000007365303900000200F9
:103490001CC13E5D595EBE570000000000000000E8
:1034A00073653130000002001CC13E5D595EC0579B
:1034B00000000000000000007365313100000200D0
:1034C0001CC13E5D595EC2570000000000000000B4
:1034D00073653132000002001CC13E5D595EC45765
:1034E000000000000000000073653133000002009E
:1034F0001CC13E5D595EC657000000000000000080
:1035000073653134000002001CC13E5D595EC8572E
:10351000000000000000000073653135000002006B
:103520001CC13E5D595ECA5700000000000000004B
:1035300073653136000002001CC13E5D595ECC57F8
:103540000000000000000000736531370000020039
:103550001CC13E5D595ECE57000000000000000017
:1035600073653138000002001CC13E5D595ED057C2
:103570000000000000000000736531390000020007
:103580001CC13E5D595ED2570000000000000000E3
:1035900073653230000002001CC13E5D595ED45795
:1035A00000000000000000007365323100000200DE
:1035B0001CC13E5D595ED6570000000000000000AF
:1035C00073653232000002001CC13E5D595ED8575F
:1035D00000000000000000007365323300000200AC
:1035E0001CC13E5D595EDA5700000000000000007B
:1035F00073653234000002001CC13E5D595EDC5729
:103600000000000000000000736532350000020079
:103610001CC13E5D595EDE57000000000000000046
:1036200073653236000002001CC13E5D595EE057F2
:103630000000000000000000736532370000020047
:103640001CC13E5D595EE257000000000000000012
:1036500073653238000002001CC13E5D595EE457BC
:103660000000000000000000736532390000020015
:103670001CC13E5D595EE6570000000000000000DE
:1036800073797300000000001CC19660095FDC398B
:103690000000000000000000703100000000000089
:1036A0001CC19660095FDC390000000000000000CA
:1036B00031000000000000001CC19660095FDC3989
:1036C00000000000000000003200000000000000C8
:1036D0001CC19660095FDC3900000000000000009A
:1036E00033000000000000001CC19660095FDC3957
:1036F0000000000000000000340000000000000096
:103700001CC19660095FDC39000000000000000069
:1037100078000000000000001CC19660095FDC39E1
:103720000000000000000000790000000000000020
:103730001CC19660095FDC39000000000000000039
:103740007A000000000000001CC19660095FDC39AF
:103750000000000000000000610000000000000008
:103760001CC19660095FDC39000000000000000009
:1037700062000000000000001CC19660095FDC3997
:1037800000000000000000006300000000000000D6
:103790001CC19660095FDC390000000000000000D9
:1037A00067353400000000001CC19660095FDC39F9
:1037B0000000000000000000673535000000000038
:1037C0001CC19660095FDC390000000000000000A9
:1037D00067353600000000001CC19660095FDC39C7
:1037E0000000000000000000673537000000000006
:1037F0001CC19660095FDC39000000000000000079
:1038000067353800000000001CC19660095FDC3994
:1038100000000000000000006735390000000000D3
:103820001CC19660095FDC39000000000000000048
:1038300067393200000000001CC19660095FDC3966
:1038400000000000000000006732380000000000A7
:103850001CC19660095FDC39000000000000000018
:1038600067333000000000001CC19660095FDC393E
:1038700000000000000000006D706F0000000000FC
:103880001CC19660095FDC390000000000000000E8
:10389000706F7300000000001CC19660095FDC3986
:1038A00000000000000000006F66730000000000D0
:1038B0001CC19660095FDC390000000000000000B8
:1038C000686F6D00000000001CC19660095FDC3964
:1038D00000000000000000007072620000000000A4
:1038E0001CC19660095FDC39000000000000000088
:1038F00070777200000000001CC19660095FDC391F
:1039000000000000000000006A6F67000000000077
:103910001CC19660095FDC39000000000000000057
:103920006A696400000000001CC19660095FDC3910
:10393000000000000000000075646100000000004D
:103940001CC19660095FDC39000000000000000027
:1039500075646200000000001CC19660095FDC39DC
:10396000000000000000000075646300000000001B
:103970001CC19660095FDC390000000000000000F7
:1039800075646400000000001CC19660095FDC39AA
:1039900000000000000000005F74650000000000EF
:1039A0001CC19660095FDC390000000000000000C7
:1039B0005F747200000000001CC19660095FDC3972
:1039C00000000000000000005F74730000000000B1
:1039D0001CC19660095FDC39000000000000000097
:1039E0005F707300000000001CC19660095FDC3945
:1039F00000000000000000005F6373000000000092
:103A00001CC19660095FDC39000000000000000066
:103A10005F657300000000001CC19660095FDC391F
:103A200000000000000000005F787300000000004C
:103A30001CC19660095FDC39000000000000000036
:103A40005F666500000000001CC19660095FDC39FC
:103A500000000000000000006D00000000000000F9
:103A60001CC18763C25DDC3900000000000000005B
:103A700071000000000000001CC16D63C25DDC39F4
:103A800000000000000000006F00000000000000C7
:103A90001CC15363C25DDC3900000000000000005F
:103AA00024000000000000001CC1A163C25DDC39DD
:103AB00000000000486F6D696E67206572726F725A
:103AC000202D2025632061786973207365747469E3
:103AD0006E6773206D6973636F6E66696775726573
:103AE000640050726F62696E67206572726F722037
:103AF0002D20256320617869732063616E6E6F7479
:103B0000206D6F766520647572696E672070726FC4
:103B100062696E67005B69645D202054696E794755
:103B2000204944253330730A005B68765D202068A5
:103B3000617264776172652076657273696F6E2554
:103B400031362E32660A005B68705D202068617233
:103B5000647761726520706C6174666F726D253177
:103B6000352E32660A005B66765D20206669726DCE
:103B7000776172652076657273696F6E2531362EB6
:103B800032660A005B66625D20206669726D77614D
:103B90007265206275696C642531382E32660A00C0
:103BA000456E7465722024626F6F743D3120746FAE
:103BB00020656E7465722074686520626F6F742072
:103BC0006C6F616465722E0A000A0A0A232323209F
:103BD00054696E794720424F4F54204C4F41444521
:103BE000522048656C70202323230A00456E7465BB
:103BF000722024646566613D3120746F20726573A4
:103C00006574207468652073797374656D20746FB2
:103C10002074686520666163746F727920646566DC
:103C200061756C742076616C7565732E0A546869D1
:103C3000732077696C6C206F766572777269746532
:103C400020616E79206368616E67657320796F7596
:103C50002068617665206D6164652E0A000A0A0A93
:103C60002323232054696E794720524553544F52E1
:103C7000452044454641554C54532048656C7020BE
:103C80002323230A00496E766F6B652073656C668B
:103C9000207465737420627920656E746572696E34
:103CA000672024746573743D4E20776865726520C3
:103CB0004E206973206F6E65206F663A0A202024BB
:103CC000746573743D312020736D6F6B652074656E
:103CD00073740A202024746573743D322020686F49
:103CE0006D696E67207465737420202028796F7564
:103CF000206D757374207472697020686F6D696EC1
:103D000067207377697463686573290A20202474B7
:103D10006573743D3320207371756172652074651D
:103D20007374202020286120736572696573206F89
:103D3000662073717561726573290A202024746589
:103D400073743D3420206172632074657374202085
:103D50002020202028736F6D65206C6172676520BC
:103D6000636972636C6573290A2020247465737417
:103D70003D3520206477656C6C2074657374202059
:103D80002020286D6F7665732073706163656420F1
:103D900062792031207365636F6E64206477656C8F
:103DA0006C73290A202024746573743D36202066C4
:103DB000656564686F6C6420746573742028656E33
:103DC000746572202120616E64207E20746F2068EB
:103DD0006F6C6420616E6420726573746172742C00
:103DE00020726573706563746976656C79290A2041
:103DF0002024746573743D3720204D20636F646503
:103E00007320746573742020284D20636F6465737C
:103E100020696E7465726D696E676C656420776980
:103E20007468206D6F766573290A20202474657389
:103E3000743D3820204A534F4E20746573742020FF
:103E4000202020286D6F74696F6E20746573742054
:103E500072756E207573696E67204A534F4E2063EA
:103E60006F6D6D616E6473290A202024746573740C
:103E70003D392020696E76657273652074696D65C1
:103E800020746573740A202024746573743D313086
:103E900020726F74617279206D6F74696F6E207417
:103EA0006573740A202024746573743D3131207366
:103EB0006D616C6C206D6F76657320746573740A28
:103EC000202024746573743D313220736C6F772029
:103ED0006D6F76657320746573740A202024746591
:103EE00073743D313320636F6F7264696E61746502
:103EF0002073797374656D206F66667365742074C2
:103F000065737420284739322C204735342D4735C6
:103F100039290A0A546573747320617373756D656A
:103F200020612063656E7465726564205859206F46
:103F3000726967696E20616E64206174206C6561CE
:103F400073742038306D6D20636C656172616E63CF
:103F50006520696E20616C6C2064697265637469A8
:103F60006F6E730A546573747320617373756D6536
:103F7000205A20686173206174206C65617374201D
:103F800034306D6D20706F73696974697665206374
:103F90006C656172616E63650A5465737473207336
:103FA00074617274207769746820612047302058EA
:103FB00030205930205A30206D6F76650A486F6D79
:103FC000696E672069732074686520657863657021
:103FD00074696F6E2E204E6F20696E697469616C12
:103FE00020706F736974696F6E206F7220636C65E7
:103FF0006172616E636520697320617373756D65AD
:10400000640A000A0A0A2323232054696E79472090
:1040100053454C4620544553542048656C7020232A
:1040200023230A0045616368202420636F6D6D615E
:104030006E642061626F766520616C736F206469C5
:1040400073706C6179732074686520746F6B656E32
:1040500020666F7220656163682073657474696E91
:104060006720696E205B205D20627261636B6574FE
:10407000730A546F20766965772073657474696E6E
:10408000677320656E746572206120746F6B656E56
:104090003A0A0A2020243C746F6B656E3E0A0A4679
:1040A0006F72206578616D706C652024796672206E
:1040B000746F20646973706C61792074686520592D
:1040C000206D6178206665656420726174650A0AF6
:1040D000546F207570646174652073657474696EC3
:1040E000677320656E74657220746F6B656E2065F2
:1040F0007175616C732076616C75653A0A0A2020CF
:10410000243C746F6B656E3E3D3C76616C75653E1C
:104110000A0A466F72206578616D706C652024799B
:1041200066723D38303020746F2073657420746877
:10413000652059206D617820666565642072617420
:104140006520746F20383030206D6D2F6D696E756D
:1041500074650A466F7220636F6E66696775726177
:1041600074696F6E2064657461696C732073656532
:104170003A2068747470733A2F2F67697468756297
:104180002E636F6D2F73796E746865746F732F541F
:10419000696E79472F77696B692F54696E79472D5E
:1041A000436F6E66696775726174696F6E0A005459
:1041B0006865736520636F6D6D616E6473206172F5
:1041C000652061637469766520666F7220636F6E27
:1041D00066696775726174696F6E3A0A202024738C
:1041E00079732053686F772073797374656D202815
:1041F00067656E6572616C292073657474696E679A
:10420000730A2020243120202053686F77206D6F9F
:10421000746F7220312073657474696E677320281F
:104220006F72207768617465766572206D6F746F48
:104230007220796F752077616E7420312C322C33A7
:104240002C34290A2020247820202053686F7720DE
:104250005820617869732073657474696E67732080
:10426000286F72207768617465766572206178695D
:104270007320796F752077616E7420782C792C7A91
:104280002C612C622C63290A2020246D20202053CD
:10429000686F7720616C6C206D6F746F722073652E
:1042A0007474696E67730A2020247120202053687B
:1042B0006F7720616C6C206178697320736574740A
:1042C000696E67730A2020246F20202053686F775F
:1042D00020616C6C206F66667365742073657474FE
:1042E000696E67730A2020242420202053686F778A
:1042F00020616C6C2073657474696E67730A20208A
:10430000246820202053686F7720746869732068C0
:10431000656C702073637265656E0A0A000A0A0A8A
:104320002323232054696E794720434F4E46494743
:1043300055524154494F4E2048656C702023232329
:104340000A000A466F722064657461696C656420B6
:1043500054696E794720696E666F207365653A20EF
:1043600068747470733A2F2F6769746875622E636E
:104370006F6D2F73796E746865746F732F54696EE7
:1043800079472F77696B692F0A466F7220746865C9
:10439000206C6174657374206669726D77617265F3
:1043A000207365653A2068747470733A2F2F6769BB
:1043B000746875622E636F6D2F73796E746865749F
:1043C0006F732F54696E79470A506C65617365206D
:1043D0006C6F6720616E79206973737565732061F6
:1043E0007420687474703A2F2F7777772E73796EF4
:1043F000746865746F732E636F6D2F666F72756D61
:10440000730A486176652066756E0A000A4E6F74FD
:10441000653A2054696E79472067656E65726174EC
:104420006573206175746F6D617469632073746165
:10443000747573207265706F727473206279206472
:10444000656661756C740A546869732063616E20D7
:1044500062652064697361626C65642062792065BD
:104460006E746572696E67202473763D300A5365F9
:1044700065207468652077696B692062656C6F7769
:1044800020666F72206D6F72652064657461696C5F
:10449000732E0A00546865736520636F6D6D616EDD
:1044A0006473206172652061637469766520667249
:1044B0006F6D2074686520636F6D6D616E64206C34
:1044C000696E653A0A205E78202020202020202076
:1044D000202020202052657365742028636F6E743D
:1044E000726F6C207829202D20736F66747761724B
:1044F000652072657365740A20203F2020202020EB
:1045000020202020202020204D616368696E6520D6
:10451000706F736974696F6E20616E642067636F7A
:104520006465206D6F64656C2073746174650A2026
:104530002024202020202020202020202020205344
:10454000686F7720616E642073657420636F6E6698
:10455000696775726174696F6E2073657474696ED2
:1045600067730A20202120202020202020202020C6
:1045700020202046656564686F6C64202D2073746C
:104580006F70206D6F74696F6E20776974686F75D6
:1045900074206C6F73696E6720706F736974696FD4
:1045A0006E0A20207E202020202020202020202075
:1045B00020204379636C65205374617274202D2030
:1045C000726573746172742066726F6D20666565C2
:1045D00064686F6C640A202068202020202020203E
:1045E00020202020202053686F7720746869732072
:1045F00068656C702073637265656E0A202024689C
:1046000020202020202020202020202053686F7789
:1046100020636F6E66696775726174696F6E20687A
:10462000656C702073637265656E0A202024746562
:1046300073742020202020202020204C69737420B7
:1046400073656C662D74657374730A202024746519
:1046500073743D4E2020202020202052756E207340
:10466000656C662D74657374204E0A202024686F73
:104670006D653D312020202020202052756E206164
:1046800020686F6D696E67206379636C650A20200E
:1046900024646566613D3120202020202020526561
:1046A00073746F726520616C6C2073657474696ECD
:1046B000677320746F2022666163746F72792220A1
:1046C00064656661756C74730A000A0A0A23232301
:1046D0002054696E79472048656C70202323230A93
:1046E000005B6A735D20206A736F6E207365726968
:1046F000616C697A65207374796C65253964205B17
:10470000303D72656C617865642C313D73747269FB
:1047100063745D0A005B6A765D20206A736F6E20A9
:10472000766572626F7369747925313564205B3008
:104730003D73696C656E742C313D666F6F74657284
:104740002C323D6D657373616765732C333D636F08
:104750006E666967732C343D6C696E656E756D2C81
:10476000353D766572626F73655D0A005B656A5DF3
:104770002020656E61626C65206A736F6E206D6FBC
:10478000646525313364205B303D746578742C3169
:104790003D4A534F4E5D0A00C958C358BC58B758DC
:1047A000AE58A35898588C58805872585B584C583B
:1047B0003F5833581F581258FD57E957E657E357EB
:1047C000D457BF57AA579B578B57795762574557AE
:1047D00028570F57F956E856D656C956B7569D561C
:1047E0009A569756945691568E568B56885685569D
:1047F00082567F567C5679567656735670566D564D
:104800006A566756645661565E565B5658565556FC
:1048100052564F564C5649564656435640563D56AC
:104820003A563756345631562E562B56285625565C
:1048300022561F561C5619561656135610560D560C
:104840000A56075604560156FE55D755B35593558B
:1048500079555F55455521550455EC54D654BC54F3
:1048600098547B546954495432541954F753DE53C5
:10487000C053A4538C537A535C53475343533F5311
:104880003B53375333532F532B53275323531F5328
:104890001B53175313530F530B530753ED52D3525C
:1048A000C052A45292527B525A5249522952095232
:1048B000EF51D551BE518B515E513E511C51F650B6
:1048C000CF50B35094507A5060503B501250FA4F32
:1048D000CF4FA34F6D4F384F264F144F054FF24E19
:1048E000D94EB74EA54E934E814E6F4E5D4E4B4EF8
:1048F000394E274E154E034EF14DDF4DCD4DBB4D7C
:10490000B74DB34DAF4DAB4DA74DA34D9F4D9B4DF7
:10491000974D934D8F4D8B4D874D834D7F4D7B4DE7
:10492000774D734D6F4D6B4D574D394D1D4DF24CBD
:10493000CD4CA84CA44CA04C9C4C984C944C904C06
:104940008C4C884C844C804C7C4C784C744C704C17
:104950005C4C404C244C084CEC4BD04BB44B984B2B
:104960007C4B604B444B284B0C4B084B044B004B8F
:10497000FC4AF84AF44AF04ADC4AB44A8D4A674A8B
:104980003A4A144AE749E349DF49DB49C849A7499C
:1049900092494A6F6767696E67206379636C652027
:1049A0006661696C65640050726F626520656E6453
:1049B000706F696E74206973207374617274696EAC
:1049C0006720706F696E740050726F626520637942
:1049D000636C65206661696C65640032343900324D
:1049E00034380032343700486F6D696E6720457285
:1049F000726F72202D20486F6D696E672073776922
:104A00007463686573206D6973636F6E666967753B
:104A100072656400486F6D696E67204572726F72CF
:104A2000202D204E65676174697665206C61746322
:104A300068206261636B6F666600486F6D696E67C0
:104A4000204572726F72202D2054726176656C2041
:104A50006D696E2026206D61782061726520746812
:104A6000652073616D6500486F6D696E67204572E2
:104A7000726F72202D204C617463682076656C6FB4
:104A800063697479206973207A65726F00486F6D6D
:104A9000696E67204572726F72202D2053656172B6
:104AA00063682076656C6F63697479206973207A16
:104AB00065726F00486F6D696E67204572726F7224
:104AC000202D20426164206F72206E6F2061786912
:104AD000732073706563696669656400486F6D690A
:104AE0006E67206379636C65206661696C6564003C
:104AF0003233390032333800323337003233360044
:104B0000323335003233340032333300536F66743E
:104B1000206C696D697420657863656564656420DF
:104B20002D2043206D617800536F6674206C696D91
:104B30006974206578636565646564202D20432071
:104B40006D696E00536F6674206C696D69742065C1
:104B500078636565646564202D2042206D6178006E
:104B6000536F6674206C696D697420657863656540
:104B7000646564202D2042206D696E00536F667459
:104B8000206C696D6974206578636565646564206F
:104B90002D2041206D617800536F6674206C696D23
:104BA0006974206578636565646564202D20412003
:104BB0006D696E00536F6674206C696D6974206551
:104BC00078636565646564202D205A206D617800E6
:104BD000536F6674206C696D6974206578636565D0
:104BE000646564202D205A206D696E00536F6674D1
:104BF000206C696D697420657863656564656420FF
:104C00002D2059206D617800536F6674206C696D9A
:104C10006974206578636565646564202D2059207A
:104C20006D696E00536F6674206C696D69742065E0
:104C300078636565646564202D2058206D61780077
:104C4000536F6674206C696D69742065786365655F
:104C5000646564202D2058206D696E00536F667462
:104C6000206C696D697420657863656564656400AE
:104C700032313900323138003231370032313600CA
:104C800032313500323134003231330032313200CA
:104C900032313100323130003230390032303800B8
:104CA000323037003230360054726170657A6F6985
:104CB0006420706C616E6E6572206661696C6564FB
:104CC00020746F20636F6E7665726765004C696D46
:104CD00069742073776974636820686974202D2073
:104CE00053687574646F776E206F63637572726555
:104CF00064004D616368696E6520697320616C6151
:104D0000726D6564202D20436F6D6D616E64206E41
:104D10006F742070726F636573736564004D6F7696
:104D200065206C657373207468616E206D696E69AF
:104D30006D756D2074696D65004D6F7665206C65CD
:104D40007373207468616E206D696E696D756D2076
:104D50006C656E6774680047656E657269632054A0
:104D6000696E7947206572726F720031393900318E
:104D700039380031393700313936003139350031B1
:104D800039340031393300313932003139310031B1
:104D90003930003138390031383800313837003196
:104DA000383600313835003138340031383300318D
:104DB00038320031383100313830005420776F728A
:104DC0006420697320696E76616C69640054207791
:104DD0006F7264206973206D697373696E67005226
:104DE00020776F726420697320696E76616C6964E4
:104DF000005220776F7264206973206D6973736944
:104E00006E67005120776F726420697320696E7637
:104E1000616C6964005120776F7264206973206D42
:104E2000697373696E67004C20776F7264206973D1
:104E300020696E76616C6964004C20776F72642023
:104E40006973206D697373696E67004820776F72AC
:104E50006420697320696E76616C6964004820770C
:104E60006F7264206973206D697373696E670045A2
:104E700020776F726420697320696E76616C696453
:104E8000004520776F7264206973206D69737369C0
:104E90006E67004420776F726420697320696E76B4
:104EA000616C6964004420776F7264206973206DBF
:104EB000697373696E67005020776F72642069733D
:104EC000206E6F7420612076616C696420746F6F4E
:104ED0006C206E756D626572005020776F72642071
:104EE0006973206E6F7420616E20696E74656765EA
:104EF00072005020776F7264206973206E6567615D
:104F000074697665005020776F7264206973207A27
:104F100065726F005020776F726420697320696E2C
:104F200076616C6964005020776F72642069732029
:104F30006D697373696E6700417263207370656396
:104F4000696669636174696F6E206572726F722041
:104F50002D20656E64706F696E74206973207374A0
:104F6000617274696E6720706F696E74004172635C
:104F70002073706563696669636174696F6E20652B
:104F800072726F72202D2072616469757320617274
:104F900063206F7574206F6620746F6C6572616E2C
:104FA000636500417263207370656369666963615C
:104FB00074696F6E206572726F72202D206D697337
:104FC00073696E67206F6666736574287329004184
:104FD00072632073706563696669636174696F6E7B
:104FE000206572726F72202D206D697373696E6710
:104FF000206178697328657329004172632073709A
:105000006563696669636174696F6E206572726F4A
:1050100072005370696E646C65206D7573742062E4
:1050200065207475726E696E6720666F7220746891
:10503000697320636F6D6D616E64005370696E6497
:105040006C65206D757374206265206F66662066DE
:105050006F72207468697320636F6D6D616E640098
:105060005370696E646C65205320776F7264206999
:105070007320696E76616C6964005370696E646C4C
:1050800065205320776F7264206973206D69737394
:10509000696E67005370696E646C65207370656536
:1050A00064206578636565646564206D6178696D09
:1050B000756D005370696E646C652073706565640E
:1050C0002062656C6F77206D696E696D756D00503B
:1050D000726F6772616D6D656420706F696E7420A8
:1050E00073616D652061732063757272656E7420E3
:1050F000706F696E740043757474657220636F6DB0
:1051000070656E736174696F6E2063616E6E6F742B
:1051100020626520656E61626C6564005265717520
:1051200065737465642076656C6F63697479206556
:10513000786365656473206C696D697473004730CA
:10514000206F72204731206D757374206265206175
:10515000637469766520666F722047353300526F3D
:105160007461727920617865732063616E6E6F740B
:10517000206265207573656420776974682074689F
:10518000697320636F6D6D616E6400496E76657240
:1051900073652074696D65206D6F64652063616E51
:1051A0006E6F74206265207573656420776974681A
:1051B000207468697320636F6D6D616E640046656D
:1051C000656472617465206E6F74207370656369C5
:1051D000666965640053656C656374656420706C12
:1051E000616E6520697320696E76616C6964005335
:1051F000656C656374656420706C616E65206973AD
:10520000206D697373696E670041786973207461FA
:105210007267657420706F736974696F6E2069734B
:1052200020696E76616C69640041786973207461ED
:105230007267657420706F736974696F6E2069732B
:10524000206D697373696E670041786973206973B3
:105250002064697361626C656400417869732069D8
:105260007320696E76616C696420666F7220746861
:10527000697320636F6D6D616E640041786973209E
:1052800063616E6E6F742062652070726573656E07
:1052900074004178697320776F7264206D6973734D
:1052A000696E670047636F6465206D6F64616C2091
:1052B00067726F75702076696F6C6174696F6E00CC
:1052C0004D20636F646520756E737570706F7274B6
:1052D00065640047636F646520636F6D6D616E6424
:1052E00020756E737570706F727465640047656EBB
:1052F000657269632047636F646520696E707574B9
:10530000206572726F7200313239003132380031EB
:10531000323700313236003132350031323400312B
:10532000323300313232003132310031323000312B
:105330003139003131380031313700313136003107
:10534000313500313134004A534F4E207374726945
:105350006E6720746F6F206C6F6E67004A534F4EFC
:1053600020696E7075742068617320746F6F206D92
:10537000616E79207061697273004A534F4E2073D9
:10538000796E746178206572726F7200496E707503
:10539000742076616C75652072616E676520657238
:1053A000726F7200496E707574206578636565640C
:1053B00073206D6178696D756D2076616C7565001F
:1053C000496E707574206C657373207468616E200B
:1053D0006D696E696D756D2076616C756500496EDD
:1053E0007075742065786365656473206D617820DD
:1053F0006C656E67746800436F6D6D616E64206EDE
:105400006F742061636365707465642061742074D7
:105410006869732074696D6500506172616D6574AF
:1054200065722063616E6E6F7420626520726561C3
:105430006400506172616D657465722069732072D9
:105440006561642D6F6E6C7900556E737570706F49
:1054500072746564206E756D626572206F72204A89
:10546000534F4E207479706500426164206E756DF3
:1054700062657220666F726D617400496E76616C50
:105480006964206F72206D616C666F726D65642057
:10549000636F6D6D616E6400556E7265636F676EEC
:1054A000697A656420636F6D6D616E64206F722030
:1054B000636F6E666967206E616D650047656E6536
:1054C00072696320617373657274696F6E206661BF
:1054D000696C757265004D656D6F727920666175D6
:1054E0006C742064657465637465640053746163EF
:1054F0006B206F766572666C6F7720646574656388
:1055000074656400436F6E74726F6C6C65722061B9
:105510007373657274696F6E206661696C7572650C
:105520000043616E6F6E6963616C206D61636869D1
:105530006E6520617373657274696F6E2066616950
:105540006C75726500506C616E6E6572206173736C
:10555000657274696F6E206661696C75726500535F
:1055600074657070657220617373657274696F6EB3
:10557000206661696C75726500456E636F64657263
:1055800020617373657274696F6E206661696C75F2
:10559000726500494F207375622D73797374656D60
:1055A00020617373657274696F6E206661696C75D2
:1055B000726500436F6E666967207375622D73793B
:1055C0007374656D20617373657274696F6E2066A4
:1055D00061696C75726500494F206D656D6F7279F8
:1055E00020616C6C6F636174696F6E2061737365A9
:1055F0007274696F6E206661696C75726500383807
:105600000038370038360038350038340038330079
:105610003832003831003830003739003738003739
:10562000370037360037350037340037330037322C
:105630000037310037300036390036380036370051
:105640003636003635003634003633003632003612
:105650003100363000353900353800353700353601
:105660000035350035340035330035320035310032
:1056700035300034390034380034370034360034E3
:1056800035003434003433003432003431003430E7
:105690000033390033380033370033360042616459
:1056A00020737461747573207265706F72742073E7
:1056B000657474696E670050657273697374656EA2
:1056C0006365206572726F7200466C6F6174206949
:1056D00073204E414E00466C6F61742069732069DF
:1056E0006E66696E697465004D6F76652074696DCC
:1056F00065206973204E414E004D6F7665207469B8
:105700006D6520697320696E66696E69746500470E
:10571000656E6572696320657863657074696F6E24
:10572000207265706F7274004661696C65642074E4
:105730006F2067657420706C616E6E657220627593
:10574000666665720053797374656D20616C617271
:105750006D202D207368757474696E6720646F778F
:105760006E00496E697469616C697A6174696F6E03
:10577000206661696C75726500526561642D6F6E9B
:105780006C79206164647265737300496E76616C34
:105790006964204164647265737300446976696466
:1057A00065206279207A65726F00466C6F6174695A
:1057B0006E6720706F696E74206572726F72004937
:1057C0006E7465726E616C2072616E6765206572C1
:1057D000726F7200496E7465726E616C20657272D0
:1057E0006F720031390031380046756E6374696F2D
:1057F0006E206973207374756262656400456E740F
:105800006572696E6720626F6F74206C6F6164658A
:105810007200496E697469616C697A696E670042E9
:1058200075666665722066756C6C202D20666174E5
:10583000616C004275666665722066756C6C00422C
:10584000756666657220656D707479004E6F2073A1
:1058500075636820646576696365004D61782066CC
:10586000696C652073697A65206578636565646530
:10587000640046696C65206E6F74206F70656E0001
:10588000456E64206F662066696C6500456E642015
:105890006F66206C696E6500486172642072657382
:1058A0006574005465726D696E6174656400436F60
:1058B0006D706C657465004E6F6F70004561676157
:1058C000696E004572726F72004F4B005B703170F1
:1058D0006F665D2070776D207068617365206F66FC
:1058E000662020202531352E3366205B302E2E3168
:1058F0005D0A005B70317770685D2070776D2063A2
:1059000063772070686173652068692531352E33AF
:1059100066205B302E2E315D0A005B703177706C33
:105920005D2070776D2063637720706861736520F8
:105930006C6F2531352E3366205B302E2E315D0A9B
:10594000005B70317773685D2070776D20636377DB
:105950002073706565642068692531352E306620B6
:1059600052504D0A005B703177736C5D2070776D1B
:1059700020636377207370656564206C6F25313513
:105980002E30662052504D0A005B70316370685DA6
:105990002070776D20637720706861736520686977
:1059A000202531352E3366205B302E2E315D0A00E6
:1059B0005B703163706C5D2070776D206377207051
:1059C00068617365206C6F202531352E3366205B4E
:1059D000302E2E315D0A005B70316373685D20707C
:1059E000776D206377207370656564206869202572
:1059F00031352E30662052504D0A005B7031637392
:105A00006C5D2070776D206377207370656564200E
:105A10006C6F202531352E30662052504D0A005BC8
:105A200070316672715D2070776D20667265717578
:105A3000656E63792020202531352E306620487A26
:105A40000A0053595354454D205245414459004C86
:105A50006F6164696E6720636F6E66696773206645
:105A6000726F6D20454550524F4D00496E69746903
:105A7000616C697A696E6720636F6E66696773200F
:105A8000746F204F4D43204F746865724D696C6C84
:105A90002073657474696E6773007B226572223AA5
:105AA0007B226662223A25302E32662C22737422C3
:105AB0003A25642C226D7367223A222573227D7D5C
:105AC0000A007B65723A7B66623A25302E32662C7C
:105AD00073743A25642C6D73673A222573227D7D99
:105AE0000A005B71765D20207175657565207265B1
:105AF000706F727420766572626F7369747925377E
:105B000064205B303D6F66662C313D73696E676C57
:105B1000652C323D747269706C655D0A00716F3A74
:105B200025640A0071693A25640A0071723A256495
:105B30000A005B73765D2020737461747573207244
:105B400065706F727420766572626F7369747925FF
:105B50003664205B303D6F66662C313D66696C743F
:105B6000657265642C323D766572626F73655D0A9D
:105B7000005B73695D202073746174757320696EB6
:105B800074657276616C2531342E3066206D730A2F
:105B9000004D6F746F7220256320706F77657220DF
:105BA000656E61626C65642073746174653A253258
:105BB0002E30660A005B257325735D206D257320EA
:105BC000706F776572206D616E6167656D656E746B
:105BD00025313064205B303D64697361626C6564BB
:105BE0002C313D616C77617973206F6E2C323D6989
:105BF0006E206379636C652C333D7768656E206D2C
:105C00006F76696E675D0A005B257325735D206D95
:105C1000257320706F6C6172697479253138642046
:105C20005B303D6E6F726D616C2C313D72657665D7
:105C30007273655D0A005B257325735D206D2573A6
:105C4000206D6963726F73746570732531366420DB
:105C50005B312C322C342C385D0A005B25732573A4
:105C60005D206D25732074726176656C207065729D
:105C7000207265766F6C7574696F6E2531302E34C5
:105C80006625730A005B257325735D206D257320DF
:105C90007374657020616E676C652532302E3366D3
:105CA00025730A005B257325735D206D2573206DB8
:105CB000617020746F206178697325313564205BD1
:105CC000303D582C313D592C323D5A2E2E2E5D0A36
:105CD000005B6D745D20206D6F746F722069646C61
:105CE000652074696D656F75742531342E326620B8
:105CF0005365630A00045D005DFB5C20646567001A
:105D0000206D6D0020696E005B73745D20207377D9
:105D100069746368207479706525313864205B305C
:105D20003D4E4F2C313D4E435D0A00546573742047
:105D3000232564206E6F7420666F756E640A004EB2
:105D4000312054314D360A4E32204731370A4E3316
:105D5000204732310A4E382046313830300A4E3929
:105D60002047310A4E3130302047393220582D3209
:105D7000352E313737592D33342E303732205A2DC6
:105D8000312E303030202854454D502C2052454D76
:105D90004F5645204C41544552290A4E3334332046
:105DA000582D32352E353935592D33342E3334397B
:105DB0000A4E33343420582D32352E373031592D98
:105DC00033342E3433360A4E33343520582D3235A1
:105DD0002E373931592D33342E3532300A4E333483
:105DE0003620582D32352E383634592D33342E3650
:105DF00030310A4E33343720582D32352E39323077
:105E0000592D33342E3637390A4E33343820582D35
:105E100032352E393630592D33342E3735340A4E3B
:105E200033343920582D32352E393832592D333408
:105E30002E3832360A4E33353020582D32352E3931
:105E40003837592D33342E3839350A4E3335312011
:105E5000582D32352E393736592D33342E393631C7
:105E60000A4E33353220582D32352E393438592DDB
:105E700033352E3032330A4E33353320582D3235F8
:105E80002E393033592D33352E3038320A4E3335D2
:105E90003420582D32352E383431592D33352E31AA
:105EA00033380A4E33353520582D32352E373633B8
:105EB000592D33352E3139300A4E33353620582D91
:105EC00032352E363639592D33352E3233390A4E86
:105ED00033353720582D32352E353539592D333558
:105EE0002E3238340A4E33353820582D32352E3480
:105EF0003333592D33352E3332350A4E333539206D
:105F0000582D32352E323931592D33352E33363323
:105F10000A4E33363020582D32352E313334592D38
:105F200033352E3339370A4E33363120582D32343B
:105F30002E393633592D33352E3432380A4E333616
:105F40003220582D32342E373737592D33352E34F1
:105F500035350A4E33363320582D32342E35373707
:105F6000592D33352E3437370A4E33363420582DD9
:105F700032342E333637592D33352E3439360A4ED6
:105F800033363520582D32342E313434592D3335B3
:105F90002E3531310A4E33363620582D32332E39D4
:105FA0003039592D33352E3532320A4E33363720BB
:105FB000582D32332E363631592D33352E35323970
:105FC0000A4E33363820582D32332E343033592D83
:105FD00033352E3533320A4E33363920582D32338D
:105FE0002E313333592D33352E3533320A4E333774
:105FF0003020582D32322E383533592D33352E3549
:1060000032370A2F4E3235313820473058302E3350
:106010003237592D33332E3532315A2D312E30301F
:10602000300A4E32353139204D3330004E31204761
:1060300032300A4E3520473430204731370A4E314E
:1060400030205431204D30360A284E313520473922
:1060500030204730205830205930205A30290A4EFD
:106060003230205335303030204D3033200A4E321C
:10607000352058302E3036342059302E33323620E9
:106080005A300A4E343020473031204631362E30D7
:106090000A4E35302058302E3036342059302E33C9
:1060A00032360A4E35352058302E303630205930B1
:1060B0002E3239330A4E36302058302E30373720C2
:1060C00059302E3236370A4E36352058302E31317F
:1060D000312059302E3235370A4E37302058302E85
:1060E0003134392059302E3235320A4E3735205866
:1060F000302E3138382059302E3235350A4E38306E
:106100002058302E3232372059302E3236380A4E4F
:1061100038352058302E3235372059302E3237312D
:106120000A4E39302058302E3333352059302E3234
:1061300036350A4E39352058302E34313220593018
:106140002E3237310A4E3130302058302E34373429
:106150002059302E3238370A4E3130352058302E03
:106160003439312059302E3238390A4E313130200D
:1061700058302E3531372059302E3237330A4E31D0
:1061800031352058302E3534342059302E323633C4
:106190000A4E3132302058302E3538302059302ECA
:1061A0003236310A4E3132352058302E35393520CD
:1061B00059302E3236330A4E3133302058302E3695
:1061C00032312059302E3237340A4E31333520588F
:1061D000302E3635392059302E3330360A4E313490
:1061E000302058302E3637332059302E3333350A8D
:1061F0004E3134352058302E3637392059302E3331
:1062000036310A4E3135302058302E363738205945
:10621000302E3338390A4E3135352058302E363746
:10622000302059302E3432300A4E3136302058303A
:106230002E3637302059302E3434360A4E3136352A
:106240002058302E3638302059302E3437340A4E0C
:106250003137302058302E3730342059302E3439F1
:10626000370A4E3137352058302E373332205930E7
:106270002E3531350A4E3138302058302E373934EA
:106280002059302E3533350A4E3138352058302ECE
:106290003837322059302E3536370A4E31393020D2
:1062A00058302E3935302059302E3630340A4E31A0
:1062B00039352058312E3033312059302E3634378D
:1062C0000A4E3230302058312E3134392059302E98
:1062D0003732320A4E3230352058312E33303820A2
:1062E00059302E3835340A4E3231302058312E3460
:1062F00033302059302E3938340A4E323135205857
:10630000312E3434372059302E3938360A4E323255
:10631000302058312E3632382059302E3832320A59
:106320004E3232352058312E3733322059302E3705
:1063300031340A4E3233302058322E303039205921
:10634000302E3338310A4E3233352058322E313127
:10635000362059302E3236360A4E323430205832FA
:106360002E3232382059302E3135370A4E323435FC
:106370002058322E3238302059302E3132330A4EE6
:106380003235302058322E3333322059302E3039C6
:10639000340A4E3235352058322E343233205930BB
:1063A0002E3037300A4E3236302058322E343839BB
:1063B0002059302E3036350A4E3236352058322E9E
:1063C0003535372059302E3036360A4E32373020A8
:1063D00058322E3632372059302E3038340A4E3269
:1063E00037352058322E3639332059302E31303956
:1063F0000A4E3238302058322E3733302059302E62
:106400003133330A4E3238352058322E3830352069
:1064100059302E3139300A4E3239302058322E3828
:1064200032392059302E3231360A4E323935205821
:10643000322E3838302059302E3239310A4E33302E
:10644000302058322E3838342059302E3330300A2C
:106450004E3330352058322E3839382059302E33CB
:1064600033320A4E3331302058322E3930352059EC
:10647000302E3336370A4E3331352058322E3931EB
:10648000302059302E3430370A4E333230205832D3
:106490002E3930382059302E3434360A4E333235C6
:1064A0002058322E3930312059302E3439350A4EA9
:1064B0003333302058322E3839372059302E343982
:1064C000350A4E3333352058322E38393020593082
:1064D0002E3532340A4E3334302058322E3834328E
:1064E0002059302E3630340A4E3334352058322E6F
:1064F0003831342059302E3636350A4E3335302077
:1065000058322E3739342059302E3735300A4E3331
:1065100035352058322E3739312059302E3833381E
:106520000A4E3336302058322E3831392059302E29
:106530003937360A4E3336352058322E3833372025
:1065400059312E3034340A4E3337302058322E38F9
:1065500036322059312E3131320A4E3337352058F8
:10656000322E3837372059312E3134350A4E3338F0
:10657000302058322E3931322059312E3231370AFB
:106580004E3338352058322E3931372059312E329A
:1065900032360A4E3339302058322E3935312059AF
:1065A000312E3238310A4E3339352058322E3937B0
:1065B000302059312E3239350A4E3430302058329D
:1065C0002E3939362059312E3239350A4E3430358C
:1065D0002058332E3031332059312E3237350A4E80
:1065E0003431302058332E3032342059312E323568
:1065F000340A4E3431352058332E3037302059315B
:106600002E3135310A4E3432302058332E30373760
:106610002059312E3133340A4E3432352058332E3E
:106620003132352059312E3033390A4E343330204F
:1066300058332E3133382059312E3031390A4E3407
:1066400033352058332E3230352059302E393038FA
:106650000A4E3434302058332E3238322059302EFE
:106660003739370A4E3434352058332E33363120FB
:1066700059302E3639310A4E3435302058332E34C5
:1066800032362059302E3539320A4E3435352058BD
:10669000332E3435362059302E3534330A4E3436C5
:1066A000302058332E3437392059302E3439330ABC
:1066B0004E3436352058332E3439342059302E3468
:1066C00037320A4E3437302058332E353035205982
:1066D000302E3434360A4E3437352058332E353187
:1066E000382059302E3431370A4E34383020583360
:1066F0002E3533302059302E3339310A4E34383567
:106700002058332E3536342059302E3330300A4E4F
:106710003439302058332E3537372059302E323522
:10672000330A4E3439352058332E35363820593017
:106730002E3231320A4E3530302058332E35343433
:106740002059302E3137360A4E3530352058332E09
:106750003534312059302E3134360A4E353130201F
:1067600058332E3535332059302E3131390A4E35D4
:1067700031352058332E3537362059302E313036CA
:106780000A4E3532302058332E3539372059302EC5
:106790003130320A4E3532352058332E36313820DA
:1067A00059302E3130390A4E3533302058332E3699
:1067B00033392059302E3132390A4E35333520588D
:1067C000332E3635302059302E3135390A4E353496
:1067D000302058332E3636332059302E3137380A90
:1067E0004E3534352058332E3637382059302E3137
:1067F00039320A4E3535302058332E363939205942
:10680000302E3139370A4E3535352058332E373250
:10681000332059302E3139360A4E35363020583330
:106820002E3736342059302E3137390A4E35363529
:106830002058332E3830352059302E3136350A4E17
:106840003537302058332E3838342059302E3135F2
:10685000390A4E3537352058332E393439205930DE
:106860002E3136350A4E3538302058332E393636EB
:106870002059302E3137350A4E3538352058332ED1
:106880003937382059302E3139340A4E35393020D5
:1068900058332E3937382059302E3232330A4E359C
:1068A00039352058332E3936302059302E32343590
:1068B0000A4E3630302058332E3833342059302E9B
:1068C0003331310A4E3630352058332E37363220A8
:1068D00059302E3334350A4E3631302058332E3766
:1068E00032362059302E3338390A4E363135205859
:1068F000332E3730332059302E3435380A4E363265
:10690000302058332E3638322059302E3533300A65
:106910004E3632352058332E3637392059302E3501
:1069200033340A4E3633302058332E36323620591F
:10693000302E3638310A4E3633352058332E353620
:10694000382059302E3832380A4E363430205833F9
:106950002E3434342059312E3038300A4E36343506
:106960002058332E3430352059312E3136370A4EE7
:106970003635302058332E3430342059312E3136CC
:10698000370A4E3635352058332E333837205931B3
:106990002E3230380A4E3636302058332E333834C3
:1069A0002059312E3230380A4E3636352058332EA3
:1069B0003336352059312E3236350A4E36373020AF
:1069C00058332E3335352059312E3238350A4E366C
:1069D00037352058332E3334382059312E33303860
:1069E0000A4E3638302058332E3333332059312E67
:1069F0003335300A4E3638352058332E3332312075
:106A000059312E3339310A4E3639302058332E332E
:106A100031312059312E3432380A4E36393520582A
:106A2000332E3333392059312E3432330A4E373036
:106A3000302058332E3434302059312E3430360A39
:106A40004E3730352058332E3531302059312E34E1
:106A500030380A4E3731302058332E3538352059EA
:106A6000312E3432310A4E3731352058332E3631FB
:106A7000312059312E3433390A4E373230205833D1
:106A80002E3631312059312E3434310A4E373235D9
:106A90002058332E3631352059312E3434310A4EB8
:106AA0003733302058332E3633362059312E343890
:106AB000380A4E3733352058332E36333420593187
:106AC0002E3531370A4E3734302058332E36323295
:106AD0002059312E3534330A4E3734352058332E71
:106AE0003630352059312E3536330A4E3735302081
:106AF00058332E3537362059312E3537350A4E3733
:106B000035352058332E3534342059312E3538312F
:106B10000A4E3736302058332E3437392059312E2B
:106B20003539320A4E3736352058332E3435312038
:106B300059312E3539380A4E3737302058332E33F5
:106B400038372059312E3632360A4E3737352058ED
:106B5000332E3339302059312E3633360A4E3738FA
:106B6000302058332E3533322059312E3630320A08
:106B70004E3738352058332E3630312059312E35A6
:106B800039370A4E3739302058332E3636382059A7
:106B9000312E3539380A4E3739352058332E3738AB
:106BA000322059312E3631320A4E383030205833A7
:106BB0002E3739342059312E3631380A4E38303597
:106BC0002058332E3836382059312E3633360A4E77
:106BD0003831302058332E3931382059312E36355E
:106BE000350A4E3831352058332E39343520593155
:106BF0002E3636370A4E3832302058332E39363456
:106C00002059312E3638350A4E3832352058332E39
:106C10003936372059312E3638350A4E3833302040
:106C200058332E3937342059312E3639390A4E38F7
:106C300033352058332E3938342059312E373235F8
:106C40000A4E3834302058332E3938342059312EFA
:106C50003735380A4E3834352058332E39373020FE
:106C600059312E3739300A4E3835302058332E39C5
:106C700034352059312E3831370A4E3835352058C1
:106C8000332E3931382059312E3832360A4E3836C3
:106C9000302058332E3839312059312E3832370AC6
:106CA0004E3836352058332E3834322059312E386C
:106CB00030390A4E3837302058332E37393820597A
:106CC000312E3738340A4E3837352058332E373482
:106CD000362059312E3737320A4E38383020583363
:106CE0002E3639382059312E3736340A4E38383559
:106CF0002058332E3633352059312E3736360A4E4A
:106D00003839302058332E3535332059312E373825
:106D1000350A4E3839352058332E3437382059311A
:106D20002E3832300A4E3930302058332E34303934
:106D30002059312E3836340A4E3930352058332E0A
:106D40003334352059312E3931380A4E393130201B
:106D500058332E3236342059322E3032330A4E39DF
:106D600031352058332E3234382059322E303531D7
:106D70000A4E3932302058332E3234302059322ED8
:106D80003038310A4E3932352058332E33313620DF
:106D900059322E3038360A4E3933302058332E339C
:106DA00039302059322E3130340A4E39333520589B
:106DB000332E3431342059322E3132310A4E3934A7
:106DC000302058332E3433312059322E3135330AA6
:106DD0004E3934352058332E3433332059322E3146
:106DE00038300A4E3935302058332E343237205956
:106DF000322E3230350A4E3935352058332E343163
:106E0000332059322E3232340A4E3936302058333C
:106E10002E3339322059322E3234320A4E39363539
:106E20002058332E3333352059322E3234340A4E23
:106E30003937302058332E3237382059322E3233FA
:106E4000360A4E3937352058332E323536205932EE
:106E50002E3234320A4E3938302058332E323339FC
:106E60002059322E3235310A4E3938352058332EDA
:106E70003231312059322E3238300A4E39393020F1
:106E800058332E3137342059322E3335360A4E39A5
:106E900039352058332E3135392059322E33393790
:106EA0000A4E313030302058332E313530205932AF
:106EB0002E3433380A4E313030352058332E3134A9
:106EC000302059322E3438310A4E3130313020588A
:106ED000332E3133322059322E3531300A4E313093
:106EE00031352058332E3131382059322E35343354
:106EF0000A4E313032302058332E30393920593251
:106F00002E3537360A4E313032352058332E303553
:106F1000312059322E3633310A4E31303330205839
:106F2000332E3030332059322E3636360A4E313039
:106F300033352058322E3935372059322E363835F0
:106F40000A4E313034302058322E39303720593201
:106F50002E3639390A4E313034352058322E3836F3
:106F6000302059322E3731310A4E313035302058E9
:106F7000322E3831392059322E3732370A4E3130DD
:106F800035352058322E3736382059322E373435A1
:106F90000A4E313036302058322E373136205932B1
:106FA0002E3735370A4E313036352058322E3637A7
:106FB000352059322E3735370A4E31303730205888
:106FC000322E3537392059322E3733310A4E31308F
:106FD00037352058322E3537302059322E3732335C
:106FE0000A4E313038302058322E3535392059325A
:106FF0002E3732300A4E313038352058322E353364
:10700000302059322E3730310A4E31303930205845
:10701000322E3530312059322E3639330A4E313046
:1070200039352058322E3437312059322E36383304
:107030000A4E313130302058322E34343320593218
:107040002E3636380A4E313130352058322E33390B
:10705000362059322E3633340A4E313131302058F1
:10706000322E3335342059322E3539310A4E3131F2
:1070700031352058322E3335322059322E353931C0
:107080000A4E313132302058322E333235205932C7
:107090002E3534330A4E313132352058322E3331C9
:1070A000352059322E3532310A4E313133302058A5
:1070B000322E3330372059322E3439380A4E31319E
:1070C00033352058322E3239362059322E34363468
:1070D0000A4E313134302058322E32393320593271
:1070E0002E3432370A4E313134352058322E32396F
:1070F000352059322E3336360A4E3131353020584C
:10710000322E3332312059322E3330330A4E313160
:1071100035352058322E3335382059322E32343717
:107120000A4E313136302058322E3431392059321E
:107130002E3230330A4E313136352058322E34312A
:10714000392059322E3137390A4E313137302058F3
:10715000322E3430352059322E3135380A4E313105
:1071600037352058322E3336322059322E313233D1
:107170000A4E313138302058322E333534205932CE
:107180002E3130340A4E313138352058322E3335D5
:10719000342059322E3039310A4E313139302058AD
:1071A000322E3338302059322E3036350A4E3131B6
:1071B00039352058322E3431302059322E30353185
:1071C0000A4E313230302058322E3431302059328C
:1071D0002E3034370A4E313230352058322E34308A
:1071E000352059322E3032380A4E31323130205863
:1071F000322E3430382059322E3031300A4E31326E
:1072000031352058322E3431362059312E39393526
:107210000A4E313232302058322E34333320593135
:107220002E3938320A4E313232352058322E34332C
:10723000382059312E3936330A4E31323330205806
:10724000322E3434372059312E3934380A4E313207
:1072500033352058322E3436312059312E393338D7
:107260000A4E313234302058322E343830205931E1
:107270002E3933310A4E313234352058322E3437DC
:10728000382059312E3839390A4E313235302058AC
:10729000322E3438372059312E3837350A4E3132B4
:1072A00035352058322E3530342059312E3835348A
:1072B0000A4E313236302058322E3532372059318D
:1072C0002E3834380A4E313236352058322E353485
:1072D000392059312E3834390A4E3132373020585E
:1072E000322E3537372059312E3836310A4E313269
:1072F00037352058322E3630342059312E38363634
:107300000A4E313238302058322E3633312059313E
:107310002E3835340A4E313238352058322E363434
:10732000302059312E3832370A4E31323930205818
:10733000322E3634302059312E3739320A4E31321E
:1073400039352058322E3632392059312E373539D9
:107350000A4E313330302058322E363132205931F6
:107360002E3732370A4E313330352058322E3537EA
:10737000362059312E3639340A4E313331302058C7
:10738000322E3533362059312E3636320A4E3133CD
:1073900031352058322E3437302059312E3631369F
:1073A0000A4E313332302058322E333435205931A1
:1073B0002E3535310A4E313332352058322E3330A6
:1073C000372059312E3532310A4E3133333020587F
:1073D000322E3236302059312E3438320A4E313383
:1073E00033352058322E3234332059312E3437374A
:1073F0000A4E313334302058322E3232382059314F
:107400002E3436390A4E313334352058322E32324A
:10741000322059312E3434380A4E31333530205829
:10742000322E3232382059312E3432350A4E313331
:1074300035352058322E3235342059312E343035FE
:107440000A4E313336302058322E323638205931F8
:107450002E3337330A4E313336352058322E3237F9
:10746000392059312E3334320A4E313337302058D7
:10747000322E3330382059312E3238370A4E3133DC
:1074800037352058322E3334302059312E323534AE
:107490000A4E313338302058322E343037205931AB
:1074A0002E3230310A4E313338352058322E3434B2
:1074B000312059312E3135360A4E3133393020588A
:1074C000322E3435342059312E3133310A4E313396
:1074D00039352058322E3436302059312E3130365D
:1074E0000A4E313430302058322E3436342059315F
:1074F0002E3130320A4E313430352058322E343766
:10750000312059312E3033360A4E31343130205843
:10751000322E3436362059302E3937310A4E313436
:1075200031352058322E3435312059302E38393704
:107530000A4E313432302058322E34313520593011
:107540002E3739310A4E313432352058322E34300C
:10755000332059302E3736370A4E313433302058E5
:10756000322E3338382059302E3736350A4E3134E2
:1075700033352058322E3330362059302E383431BE
:107580000A4E313434302058322E323232205930C3
:107590002E3931310A4E313434352058322E3131C2
:1075A000342059302E3939350A4E3134353020588F
:1075B000322E3030322059312E3037360A4E3134A7
:1075C00035352058312E3930352059312E31333967
:1075D0000A4E313436302058312E37353420593167
:1075E0002E3232330A4E313436352058312E36336E
:1075F000372059312E3237380A4E3134373020583F
:10760000312E3538322059312E3330310A4E313453
:1076100037352058312E3535382059312E33313514
:107620000A4E313438302058312E3436302059311A
:107630002E3335320A4E313438352058312E333915
:10764000392059312E3336300A4E313439302058F2
:10765000312E3333382059312E3335340A4E3134FC
:1076600039352058312E3238372059312E333239BE
:107670000A4E313530302058312E323438205931CD
:107680002E3239340A4E313530352058312E3231D0
:10769000372059312E3235340A4E313531302058A9
:1076A000312E3231342059312E3235320A4E3135B5
:1076B00031352058312E3137322059312E3139357C
:1076C0000A4E313532302058312E3132382059317E
:1076D0002E3133390A4E313532352058312E313181
:1076E000302059312E3131370A4E31353330205860
:1076F000302E3935382059302E3934310A4E313553
:1077000033352058302E3839312059302E38373320
:107710000A4E313534302058302E38323520593029
:107720002E3830380A4E313534352058302E373522
:10773000352059302E3734370A4E31353530205800
:10774000302E3631392059302E3633330A4E31350A
:1077500035352058302E3437372059302E353236D3
:107760000A4E313536302058302E343737205930D4
:107770002E3532340A4E313536352058302E3431DC
:10778000312059302E3437360A4E313537302058B3
:10779000302E3333312059302E3435340A4E3135C2
:1077A00037352058302E3237382059302E34323782
:1077B0000A4E313538302058302E3233312059308E
:1077C0002E3339370A4E313538352058302E31387E
:1077D000332059302E3337390A4E3135393020585D
:1077E000302E3133352059302E3336350A4E31356F
:1077F00039352058302E3037362059302E33343139
:107800000A4E3136303520473030204633302E3066
:107810000A4E31363130204D3035200A4E31363166
:107820003520473930205830205930205A300A4E00
:1078300031363135204D33300A28456E64206F666D
:1078400020434E432050726F6772616D2900284DAE
:1078500053472A2A2A2A204D6963726F7374657010
:107860002054657374205B76315D202A2A2A2A29E8
:107870000A473030204731372047323120473430F3
:107880002047343920473830204739300A6730786C
:107890003079307A300A7B22316D69223A317D0AA3
:1078A0007B22326D69223A317D0A7B22336D692257
:1078B0003A317D0A7B22346D69223A317D0A673084
:1078C000207831300A7B22316D69223A327D0A7884
:1078D000300A7B22316D69223A347D0A7831300AD0
:1078E0007B22316D69223A387D0A78300A67302070
:1078F0007931300A7B22326D69223A327D0A793041
:107900000A7B22326D69223A347D0A7931300A7B52
:1079100022326D69223A387D0A79300A6730207A3E
:1079200031300A7B22336D69223A327D0A7A300A7D
:107930007B22336D69223A347D0A7A31300A7B2208
:10794000336D69223A387D0A7A300A673020613116
:10795000300A7B22346D69223A327D0A61300A7B1B
:1079600022346D69223A347D0A6131300A7B223437
:107970006D69223A387D0A61300A6D3200284D5314
:10798000472A2A2A2A20436F6F7264696E617465E0
:10799000206F6666736574732074657374205B76FC
:1079A000315D202A2A2A2A290A6730306731376751
:1079B00032316734306734396738306739300A67B5
:1079C00035340A673932783079307A300A663630A1
:1079D000300A284D53472A2A2A2A207465737420B6
:1079E000473932206F6666736574732A2A2A2A29FA
:1079F0000A286D73675374657020313A204D6F7695
:107A0000652066726F6D20302C3020746F2033300B
:107A10002C30206D6D20696E20706F7369746976EB
:107A200065205820646972656374696F6E290A283D
:107A30006D73675374657020323A205265736574B4
:107A4000206F726967696E20746F20302E30207548
:107A500073696E6720473932290A286D736753743A
:107A6000657020333A204D6F766520746F20323078
:107A70002C302E2053686F756C64206D6F766520F6
:107A80003230206D6D20696E20706F736974697675
:107A900065205820646972656374696F6E20616E39
:107AA0006420737461747573207265706F727420D2
:107AB00073686F756C642073746172742066726F82
:107AC0006D20302C30290A286D736753746570203F
:107AD000343A204D6F766520746F20302E30202090
:107AE0002053686F756C64206D6F7665203230208E
:107AF0006D6D20696E206E656761746976652058CA
:107B000020646972656374696F6E20616E642073AE
:107B10007461747573207265706F72742073686F0E
:107B2000756C642073746172742066726F6D20329C
:107B3000302C30290A67317833300A67393278308F
:107B40000A67317832300A6731783079300A247325
:107B5000720A67393278300A673470302E350A2855
:107B60004D53472A2A2A2A207465737420473535D5
:107B7000206F6666736574732A2A2A2A290A286D7B
:107B800073675374657020313A2053657420436FD6
:107B90006F7264696E6174652073797374656D20AA
:107BA00032205B6735355D20746F206F66667365C4
:107BB00074206F662035302C3530290A286D7367A4
:107BC0005374657020323A2053656C6563742047A6
:107BD000353520636F6F7264696E617465207379E7
:107BE0007374656D290A286D73675374657020334B
:107BF0003A204D6F766520746F20302C302E20484F
:107C00006561642073686F756C64206D6F766520A4
:107C1000646961676F6E616C6C7920696E202B58A6
:107C200020616E64202B5920616E6420737461742E
:107C30007573207265706F72742073686F756C64F1
:107C40002073746172742066726F6D20302C30293D
:107C50000A6731304C3270327835307935300A6706
:107C600035350A6730783079300A673470302E3510
:107C70000A284D53472A2A2A2A20746573742047FC
:107C80003533206162736F6C757465206F76657231
:107C90007269646573202A2A2A2A290A286D736763
:107CA0005374657020313A2052756E2061207371D3
:107CB0007561726520696E2047353520737973745C
:107CC000656D290A286D73675374657020323A20F8
:107CD00052756E20612073717561726520772F4730
:107CE0003533206F76657272696465290A6730786A
:107CF0003079300A673078323079300A673078323C
:107D0000307932300A673078307932300A6730782B
:107D10003079300A673470302E350A673533673072
:107D2000783079300A673533673078323079300A05
:107D300067353367307832307932300A67353367E8
:107D40003078307932300A673533673078307930BF
:107D50000A6730783079300A673470302E350A2857
:107D60004D53472A2A2A2A20746573742052657459
:107D700075726E20746F20686F6D65202A2A2A2A1A
:107D8000290A286D73675374657020313A20526553
:107D90007475726E20746F20686F6D6520757369DD
:107DA0006E6720473238290A286D736753746570EF
:107DB00020323A20526573657420746F2047353441
:107DC00020636F6F72642073797374656D290A671D
:107DD00032380A6735340A6D333000284D53472A4C
:107DE0002A2A2A2054657374206163637572616363
:107DF00079206F6620736C6F77206D6F76657320C6
:107E00005B76315D202A2A2A2A290A6735350A67D6
:107E100030783079300A673470302E350A67347024
:107E2000302E350A67317831306632320A673534A0
:107E30000A6730783079300A6D333000284D534767
:107E40002A2A2A2A20546573742076657279207351
:107E5000686F7274206D6F766573205B76315D207C
:107E60002A2A2A2A290A6730783079300A6734703A
:107E7000302E350A673178302E3166313030300A95
:107E800078300A78302E310A78300A78302E310A6C
:107E900078300A78302E310A78300A78302E310A5C
:107EA00078300A78302E310A78300A78302E310A4C
:107EB00078300A78302E310A78300A78302E310A3C
:107EC00078300A78302E310A78300A78302E310A2C
:107ED00078300A78302E310A78300A78302E310A1C
:107EE00078300A78302E310A78300A78302E310A0C
:107EF000673470302E350A78300A78302E30310AE7
:107F000078300A78302E30310A78300A78302E30C6
:107F1000310A78300A78302E30310A78300A7830D9
:107F20002E30310A78300A78302E30310A78300A13
:107F300078302E30310A78300A78302E30310A7895
:107F4000300A78302E30310A78300A78302E3031CD
:107F50000A78300A78302E30310A78300A78302E9C
:107F600030310A78300A78302E30310A78300A7889
:107F7000302E30310A6730783079300A6D3200287F
:107F80004D53472A2A2A2A20526F74617279204160
:107F9000786973204D6F74696F6E20546573742017
:107FA0005B76315D202A2A2A2A290A673030673118
:107FB0003767323167343067343967383067393082
:107FC0000A6730783079307A306130623063300A55
:107FD0006735350A6730783079300A6633363030A5
:107FE000300A6730613336300A623336300A633321
:107FF00036300A61300A62300A63300A6731613113
:108000003434300A62313434300A63313434300A63
:1080100061300A62300A63300A67316131343430CA
:1080200062373230633336300A783079307A3061F3
:1080300030623063300A6731783630613134343041
:1080400062373230633336300A783079307A3061D3
:1080500030623063300A67317836307935306131DB
:1080600034343062373230633336300A7830793026
:108070007A306130623063300A6731783630793572
:1080800030783235613134343062373230633336F0
:10809000300A783079307A306130623063300A6784
:1080A00035340A6730783079300A6D333000284D26
:1080B00053472A2A2A2A20496E766572736520540E
:1080C000696D65204D6F74696F6E205465737420FF
:1080D0005B76315D202A2A2A2A290A6730306731E7
:1080E0003767323167343067343967383067393051
:1080F0000A6735350A6730783079300A6739330ACC
:1081000066302E30310A67317831300A7931300AE1
:108110007A31300A6131300A78300A79300A7A309F
:108120000A61300A67317831307931307A2D313057
:108130006131300A6730783079307A3061300A66E0
:10814000302E310A6732783130792D31307A2D3244
:10815000306931300A6730783079307A300A6733E5
:10816000783130792D31307A2D32306931300A67EB
:1081700030783079307A300A673278323079307A34
:108180002D32306931300A6730783079307A300AF0
:10819000673378323079306931300A673078307936
:1081A000307A300A6732783079307A2D333069315D
:1081B000300A6733783079307A306931300A673085
:1081C000783079307A300A673278307930693230F5
:1081D0002028435720333630206465677265657305
:1081E000290A673378307930693230202843435781
:1081F000203336302064656772656573290A6739F4
:10820000340A6735340A6730783079300A6D333094
:10821000007B226763223A2267303067313767324A
:1082200031673430673439673830673930227D0A36
:108230007B226763223A22673535227D0A7B2267DB
:1082400063223A22673078307930227D0A7B2267B8
:1082500063223A2266353030227D0A7B2267632210
:108260003A22284D53477371756172657329227DD7
:108270000A7B226763223A226730783230227D0AF5
:108280007B226763223A22793230227D0A7B226781
:1082900063223A227830227D0A7B226763223A22C7
:1082A0007930227D0A7B226763223A226731783156
:1082B00030227D0A7B226763223A22793130227D87
:1082C0000A7B226763223A227830227D0A7B22676A
:1082D00063223A227930227D0A7B226763223A2286
:1082E000284D5347636972636C657329227D0A7B4D
:1082F000226763223A226732783130792D31306932
:108300003130227D0A7B226763223A22673078303F
:108310007930227D0A7B226763223A2267337831E3
:1083200030792D3130693130227D0A7B226763221A
:108330003A22673078307930227D0A7B22676322C7
:108340003A2267327832307930693130227D0A7BC7
:10835000226763223A22673078307930227D0A7BA7
:10836000226763223A2267337832307930693130BC
:10837000227D0A7B226763223A2267307830793087
:10838000227D0A7B226763223A2267327830793075
:10839000693130227D0A7B226763223A2267337873
:1083A000307930693130227D0A7B226763223A229C
:1083B000673534227D0A7B226763223A2267307850
:1083C000307930227D0A7B226763223A226D333076
:1083D000227D00284D53472A2A2A2A204D636F64A4
:1083E00065732074657374205B76315D202A2A2AB8
:1083F0002A290A6735350A6730783079300A6D33B3
:108400000A673470310A6D350A673470310A6D3489
:108410000A673470310A6D350A673470310A6D3776
:108420000A673470310A6D390A673470310A6D3861
:108430000A673470310A6D390A663530300A6730A0
:108440007832300A7932300A6D330A78300A6D3466
:108450000A79300A6D350A67317831300A6D370A8A
:108460007931300A6D380A78300A6D390A79300A64
:108470006732783130792D31306931300A6D330A05
:108480006730783079300A6D340A67337831307963
:108490002D31306931300A6D350A673078307930E6
:1084A0000A6D370A673278323079306931300A6DB7
:1084B000380A6730783079300A6D390A6733783294
:1084C0003079306931300A6730783079300A673274
:1084D000783079306931300A6733783079306931F2
:1084E000300A6735340A6730783079300A6D3330B6
:1084F00000284D53472A2A2A2A2046656564686F5A
:108500006C642054657374205B76315D202A2A2ABE
:108510002A290A284D53472A2A2A2A204D616E7596
:10852000616C6C7920656E746572202120616E64C7
:10853000207E20647572696E67206D6F76656D654B
:108540006E7420746F2074657374202A2A2A2A2975
:108550000A6735350A6730783079300A6734703306
:108560000A67303067313767323167343067343902
:108570006738306739300A663630300A673078310C
:1085800030307637362E3736350A783079300A670C
:1085900035340A6730783079300A6D333000284D31
:1085A00053472A2A2A2A204477656C6C2054657325
:1085B00074205B76315D202A2A2A2A290A67303006
:1085C0006731376732316739300A6735350A6730C6
:1085D000783079300A663530300A67307831300AC1
:1085E000673470310A67307832300A673470310A84
:1085F00067307831300A673470310A67307830304C
:108600000A673470310A79350A6735340A67307879
:108610003079300A6D330A673470310A6730783147
:10862000307931300A6D350A673470310A67307835
:1086300032307932300A6D340A673470310A67306B
:108640007833307933300A6D380A673470310A670D
:10865000307834307934300A6D390A673470310A31
:1086600067307835307935300A6730783079300ABC
:108670006D3330004E31206730306731376732312B
:108680006734306734396738306739300A4E3130F3
:10869000206730783079300A4E32302066353030FD
:1086A0000A4E3330206732783130792D31306931DC
:1086B0003020284357203237302064656772656563
:1086C00073290A4E3430206730783079300A4E35BD
:1086D00030206733783130792D31306931302028BE
:1086E0004343572039302064656772656573290AF2
:1086F0004E3630206730783079300A4E3830206777
:10870000327832307930693130202843572031387F
:10871000302064656772656573290A4E37302067BB
:1087200030783079300A4E383020673378323079FB
:108730003069313020284343572031383020646578
:108740006772656573290A4E393020673078307951
:10875000300A4E39392046313230300A4E3130300D
:1087600020673278307930693230202843572033FF
:1087700036302064656772656573290A4E31313081
:1087800020673278307930693230202843572033DF
:10879000363020616761696E290A4E3132302066B9
:1087A00037303020284368616E67652066656564F0
:1087B0002072617465207768696C6520696E204756
:1087C00032206D6F74696F6E206D6F6465290A4E7B
:1087D00031333020673278307930693230202843A5
:1087E0005720333630203372642074696D65290A4E
:1087F0004E31343020673278307930693230202879
:10880000435720333630203474682074696D6529ED
:108810000A4E31353020663530300A4E3136302040
:108820006733783079307A343069323020284343E6
:108830005720333630206465677265657320776929
:108840007468206C696E6561722074726176656C03
:10885000290A4E313730206733783079307A3069E1
:108860003230202843435720333630206167616916
:108870006E290A4E313830206637303020286D732B
:10888000672A2A2A2A4368616E67652066656564DF
:108890002072617465207768696C6520696E204775
:1088A00033206D6F74696F6E206D6F64652A2A2A9C
:1088B0002A290A4E313930206733783079306932CD
:1088C00030202843435720333630203372642074DD
:1088D000696D65290A4E323030206733783079303F
:1088E00069323020284343572033363020347468AF
:1088F0002074696D65290A4E32313020286D736706
:108900002A2A2A2A473138204576616C20746573FB
:10891000742A2A2A2A290A4E323230204731205816
:1089200033302E373037205A35302E373237204605
:108930003530300A4E32333020473138204730321C
:10894000205836372E373338205A32332E363137C7
:108950002052323520463235300A4E3234302067CC
:1089600038300A4E323530206730783079307A30FE
:108970000A4E323630206D333000284D53472A2AB4
:108980002A2A2053717561726573204D6F74696F67
:108990006E2054657374205B76315D202A2A2A2A62
:1089A000290A6730306731376732316734306734CE
:1089B000396738306739300A6730783079300A677C
:1089C0003078323020287472617665727365206168
:1089D0002032306D6D2073717561726520696E2073
:1089E0005820616E642059290A7932300A78300A99
:1089F00079300A673178313066353030202864723A
:108A0000617720612031306D6D2073717561726501
:108A100020696E205820616E6420592061742046C0
:108A2000353030290A7931300A78300A79300A67CE
:108A3000307A3230202874726176657273652061F5
:108A40002032306D6D2073717561726520696E2002
:108A50005820616E64205A290A7832300A7A300A26
:108A600078300A67317832307932307A3230663590
:108A7000303020286665656420612032306D6D20BD
:108A8000646961676F6E616C20696E20582C205993
:108A900020616E64205A290A783079307A300A7859
:108AA00034307934307A34302028747261766572CB
:108AB000736520612034306D6D20637562652069B7
:108AC0006E20582C205920616E64205A290A78346F
:108AD0003079307A300A78307934307A34300A7824
:108AE00034307934307A300A783079307A34300A58
:108AF00078307934307A300A78343079307A3430DA
:108B00000A783079307A300A6738300A673078303E
:108B100079300A673078310A673078300A6D33303F
:108B200000284D53472A2A2A2A20486F6D696E670C
:108B30002054657374205B76315D202A2A2A2A2905
:108B40000A6732382E32783079307A300A6D333015
:108B500000284D53472A2A2A2A20536D6F6B65201F
:108B600054657374205B76315D202A2A2A2A290AEB
:108B700047303020473137204732312047343020CA
:108B800047343920473830204739300A6D3367344D
:108B900070310A6D35673470310A6D346734703165
:108BA0000A6D33673470310A6D35673470310A6D80
:108BB00037673470310A6D39673470310A6D386740
:108BC0003470310A6D390A6730783079307A300A7A
:108BD000673030207832300A78300A7932300A79BA
:108BE000300A7A32300A7A300A6132300A61300A49
:108BF0004730302078323020793230207A323020BD
:108C00006132300A473030207830207930207A3095
:108C10002061300A473031206633302078322079A5
:108C200032207A322061320A7830207930207A304E
:108C30002061300A673078310A673078300A6D3247
:108C4000002C000A00257300256C750025312E309C
:108C500066002573002C000A0025733A2573002551
:108C6000733A256C750025733A25312E3066002540
:108C7000733A2573005B74765D20207465787420E8
:108C8000766572626F7369747925313564205B3063
:108C90003D73696C656E742C313D766572626F73DD
:108CA000655D0A0025660A00256C750A0025640AC0
:108CB0000025730A0074696E7967205B25735D2057
:108CC0006572723A2025733A202573200074696E0C
:108CD0007967205B25735D206F6B3E2000456E64D5
:108CE000206F6620636F6D6D616E642066696C65D0
:108CF0000A0052C9FBC6BFC9E0C93FCA40C717CD69
:108D0000FBC6ABCD17CE45CC40C7000040064006A1
:108D10001040B800B817CDFBC6ABCD17CE45CC4040
:108D2000C70000400620060840B800B880CFFBC648
:108D3000A0CE1CCFCBD069CEA00840060506090105
:108D40000880CFFBC6A0CE1CCF51CA40C7B0084098
:108D5000060540B030800000000000F0E0D0C010F8
:108D60000100CF673322211F1B1301016E616E00CA
:108D7000696E66004E414E494E495459494E46CDA2
:108D8000CCCC3D0AD7233C17B7D13877CC2B3295C2
:108D900095E6241FB14F0A000020410000C84200A0
:108DA000401C4620BCBE4CCA1B0E5AAEC59D74006A
:108DB000407A10F35A00A0724E18090010A5D4E8AA
:108DC0000000E87648170000E40B54020000CA9A3D
:108DD0003B000000E1F5050000809698000000408F
:108DE000420F000000A086010000001027000000D4
:108DF00000E803000000006400000000000A00001A
:108E00000000000100000000002C76D888DC674FCD
:108E10000823DFC1DFAE59E1B1B796E5E3E453C6FD
:108E20003AE651997696E8E6C28426EB898C9B62F5
:108E3000ED407C6FFCEFBC9C9F40F2BAA56FA5F49F
:108E400090055A2AF75C936B6CF9676DC11BFCE0C7
:108E5000E40D47FEF520E6B500D0ED902E0300941A
:108E60003577050080841E080000204E0A000000AF
:108E7000C80C333333330F986E12831141EF8D21B9
:108E800014893BE65516CFFEE6DB18D1844B381B20
:108E9000F77C1D901DA4BBE424203284725E2281E5
:108EA00000C9F124ECA1E53D270011241FBECFEF3E
:108EB000CDBFDFE5DEBF00E00CBF13E2A0E0B0E213
:108EC000E4E9F8EC01E00BBF02C007900D92A63870
:108ED000B107D9F729E5A6E8B3E201C01D92A03E8B
:108EE000B207E1F70E942B800C9448E40C94000038
:108EF000FC0160817181828193810E9419D6609307
:108F0000AD320895FC0160817181828193810E945C
:108F100019D66093AC320895AF92BF92CF92DF9290
:108F2000EF92FF920F931F93CF93DF937B018C01FE
:108F300080E3C82E82E3D82EE601AA24A394BC2E97
:108F4000BC18F70161917191819191917F012CEA97
:108F500035EC47E257E30E94A8D718164CF4F80105
:108F600040815181628173818B2D0E949981A882F9
:108F70000C5F1F4F2196F2E3C633DF0701F7DF9145
:108F8000CF911F910F91FF90EF90DF90CF90BF9006
:108F9000AF900C94A481FC016081718182819381E6
:108FA0000E9419D66093AE32613019F481E00E94BC
:108FB000A07781E00C94C177CF93DF93CDB7DEB774
:108FC0006897CDBFDEBFFC01608171818281938192
:108FD0000E9419D66093AF3281E0613019F40E948B
:108FE000A0770CC00E94C177CE01019628E1FC0158
:108FF00011922A95E9F7BC010E94CB476896CDBF34
:10900000DEBFDF91CF9108950F931F93CF93DF932E
:10901000CDB7DEB72D97CDBFDEBF27E0E8EDF0E29C
:109020008E010F5F1F4FD80101900D922A95E1F735
:10903000BC01660F771F680F791F660F771F660FD9
:10904000771F660F771F68567A4E45E050E0CE01D5
:1090500008960E94B8E1688570E0C8010E94E6E1C8
:10906000009739F46B8570E0C8010E94E6E1009733
:1090700011F0801B01C08FEF2D96CDBFDEBFDF91B9
:10908000CF911F910F910895EF92FF920F931F932D
:10909000CF93DF938C01F62EE72EEC012D96FC0189
:1090A00061857285838594850E9419D61F926F937E
:1090B000DF93CF930F5E1F4F1F930F93DF93CF93D9
:1090C000EF92FF92ECEDF9E581818F9380818F9390
:1090D0000E947FE2EDB7FEB73C96EDBFFEBFDF9189
:1090E000CF911F910F91FF90EF9008950F931F93D1
:1090F000CF93DF93EC01162F072F8C819D810E9467
:10910000044883305CF58F3FA1F528C09E01235FA2
:109110003F4F9F938F938C858F938B858F938A85F9
:109120008F9389858F933F932F936196DF93CF938E
:109130003F932F930F931F938091DD598F938091CD
:10914000DC598F930E947FE28DB79EB740968DBF0A
:109150009EBFDF91CF911F910F910895E7E1F4E158
:10916000659174914FE450E084ED9CE30E94B8E176
:10917000CDCFE091A632F0E0EE0FFF1FED5EFB4E8B
:10918000659174914FE450E084ED9CE30E94B8E156
:10919000BDCF0F931F93CF93DF93EC01162F072FB3
:1091A0008C819D810E94044883307CF58F3FC1F5FE
:1091B0002CC0AE014F5E5F4F9E01235F3F4F9F93D8
:1091C0008F938C858F938B858F938A858F938985D9
:1091D0008F935F934F933F932F935F934F933F935F
:1091E0002F930F931F938091DD598F938091DC59BA
:1091F0008F930E947FE28DB79EB742968DBF9EBF30
:10920000DF91CF911F910F910895E7E1F4E165910E
:1092100074914FE450E084ED9CE30E94B8E1C9CF23
:10922000E091A632F0E0EE0FFF1FED5EFB4E659180
:1092300074914FE450E084ED9CE30E94B8E1B9CF13
:10924000DF92EF92FF920F931F93CF93DF93CDB7EF
:10925000DEB72897CDBFDEBF8B01E42ED52E37E0D9
:10926000EFEDF0E2DE01119601900D923A95E1F7F3
:1092700028870E940448F82E288582E08F1518F070
:10928000E22FF0E002C0E2E0F0E0EE0FFF1FED5E43
:10929000FB4E659174914FE450E084ED9CE30E9495
:1092A000B8E19F938F93F80183818F9382818F938D
:1092B00081818F9380818F93E1E0F0E0EC0FFD1FBF
:1092C000EF0DF11D80811F928F93DF92EF928091BD
:1092D000DD598F938091DC598F930E947FE2CDBF3F
:1092E000DEBF2896CDBFDEBFDF91CF911F910F91DA
:1092F000FF90EF90DF9008954F925F926F927F9270
:10930000AF92BF92CF92DF92EF92FF920F931F9393
:10931000CF93DF93C0E3D2E305EF10E35C018991C3
:10932000813009F042C0F801C480D580E680F78022
:109330004080518062807380A3019201C701B60111
:109340000E94FCD39F772CEA35EC47E257E30E945A
:10935000A5D587FD2AC020E034E244E759ECC701D7
:10936000B6010E94A8D718165CF4F501208131815E
:1093700042815381C701B6010E94A8D7181604F193
:1093800020E034E244E759ECC301B2010E94A8D7BF
:1093900018165CF4F5012081318142815381C301AB
:1093A000B2010E94A5D587FD0BC00B5C1F4FF4E0F6
:1093B000AF0EB11C82E3C633D80709F0B0CF02C0AC
:1093C0008CED01C080E0DF91CF911F910F91FF9054
:1093D000EF90DF90CF90BF90AF907F906F905F90B5
:1093E0004F90089580912C32811105C080912B32CD
:1093F00080932A3229C0823031F487E080932A3268
:1094000080912B3221C0833031F489E080932A325D
:1094100080912B3219C0843031F48AE080932A3253
:1094200080912B3211C080912D32813031F485E052
:1094300080932A3280912B3207C0823019F486E063
:1094400080932A3280912B32863019F080912A3213
:1094500008958BE080932A32089580912B320895ED
:1094600080932D32813059F018F0823041F0089508
:109470008BE592E38093593290935A32089583E2B8
:1094800096E58093593290935A320895FC01848175
:109490000895845B9F4FFC0180810895855B9F4FF9
:1094A000FC0180810895825B9F4FFC0180810895BB
:1094B000815B9F4FFC0180810895875B9F4FFC017A
:1094C000808108950C949A96CD96FC0160817181FB
:1094D000828193810895FC01648308958B5A9F4F84
:1094E000FC01608308958F5B9F4FFC014083518393
:1094F00062837383089560935B3270935C328093D0
:109500005D3290935E3280EE91E20C94E261BF9204
:10951000CF92DF92EF92FF920F931F93CF93DF933F
:10952000D090A8327C010DEC12E38091A73290E03C
:10953000EC01CC0FDD1FC80FD91FCC0FDD1FCC0FE6
:10954000DD1FCC0FDD1FCC5BDF4C81E0D816A9F00E
:10955000B881A981CA80BB8040912033413091F409
:10956000F80120813181428153816B2F7A2F8C2D1C
:109570009B2D0E94FDD39B0109C020E030E080E0DC
:1095800090E004C02B2F3A2F8C2D9B2DA901BC01FC
:10959000F701458F568F678F70A3F4E0EF0EF11C33
:1095A0000C5F1F4F249682E3053E180771F6DF918A
:1095B000CF911F910F91FF90EF90DF90CF90BF90D0
:1095C0000895835B9F4FFC0160838BE592E30C94CD
:1095D000874A4F925F926F927F928F929F92AF9243
:1095E000BF92CF92DF92EF92FF920F931F93CF9390
:1095F000DF93CDB7DEB76897CDBFDEBF8C0160913A
:10960000203370E080E090E00E9447D62B013C01BF
:10961000F80160817181828193810E9419D670E086
:109620005B01AA0CBB1CA60EB71EAA0CBB1CAA0C85
:10963000BB1CAA0CBB1CC5018C5B9F4C5C010DECD8
:1096400012E3FE0131964F01F501C190D190E190F6
:10965000F1905F01F80161917191819191918F0178
:10966000A30192010E944AD89B01AC01C701B60137
:109670000E94FDD3F40161937193819391934F0103
:10968000F2E3053E1F0701F7CE0101960E947D9689
:109690008BE592E30E94874A6896CDBFDEBFDF91DB
:1096A000CF911F910F91FF90EF90DF90CF90BF90DF
:1096B000AF909F908F907F906F905F904F900895A4
:1096C0008B55924369F4E62FF0E0EE0FFF1FEE0F8B
:1096D000FF1FEB54FD4C608171818281938108955D
:1096E000862F0C947296CF92DF92EF92FF920F9397
:1096F0001F93CF93DF93EC0182E3CB35D80709F0BA
:109700004AC070E0FB01EE0FFF1FEE0FFF1FEB548E
:10971000FD4CC080D180E280F3808091A8328130FE
:1097200059F18091A73290E0FC01EE0FFF1FE80F86
:10973000F91FEE0FFF1FE60FF71FEE0FFF1FEE0FD3
:10974000FF1FEC5BFF4C00811181B281A38120914E
:1097500020332130B1F4FB01EE0FFF1FEE0FFF1F8E
:10976000E353FD4C2081318142815381B8018B2F1D
:109770009A2F0E94FDD308C060E070E080E090E086
:1097800003C0B8018B2F9A2F9B01AC01C701B60112
:109790000E94FCD303C0862F0E948696C55BDF4FD4
:1097A0002881211106C023E333E34BEC51E40E94EE
:1097B000ACD5DF91CF911F910F91FF90EF90DF908B
:1097C000CF90089588E1E0E6F2E3A5EBB2E30190E3
:1097D0000D928A95E1F78091A43281110CC080919D
:1097E0005F32813041F41092983210929932109287
:1097F0009A3210929B3208954F925F926F927F92AD
:109800008F929F92AF92BF92CF92DF92EF92FF9290
:109810000F931F93CF93DF93CDB7DEB76997CDBF7B
:10982000DEBF80912C32811155C080915132813040
:1098300009F050C00E949AC681114CC0109251325A
:109840009CE5692E90E3792E26E3822E912C8E01E1
:109850000E5E1F4F36EEA32E30E2B32E33C0F7015B
:1098600081917F011F928F935F924F92BF92AF922F
:109870001F930F930E944AE3B80184E493E20E948D
:10988000475F8D839E83F60181919191A191B19162
:109890006F018A879B87AC87BD87CE0101960E94A6
:1098A000365CCDBFDEBF9EEDE91690E2F906B9F653
:1098B000E8E16E0E711CFFEF8F1A9F0A8CE3881689
:1098C000910441F0240189EDE82E80E2F82E630135
:1098D00088E7C8CF80E06996CDBFDEBFDF91CF912A
:1098E0001F910F91FF90EF90DF90CF90BF90AF90BE
:1098F0009F908F907F906F905F904F9008952F92E0
:109900003F924F925F926F927F928F929F92AF920F
:10991000BF92CF92DF92EF92FF920F931F93CF935C
:10992000DF93CDB7DEB72997CDBFDEBF4C015B011A
:109930004090AA325090A8322090A73260902033F5
:109940007090A6326B0180E692E3888799875CEE7F
:10995000E52E50E3F52E98E1299E10011124840193
:10996000D6016D917D918D919D916D012CEA35EC23
:1099700047E257E30E94A5D587FD80C0F7018081AB
:109980008150823008F07AC041104CC0F1E05F167F
:1099900009F1E885F985E20DF31DEC51F240808173
:1099A000898391819D83B281A381E1E06E1217C00A
:1099B000E885F985E359FF4F208131814281538148
:1099C000BC018B2F9A2F0E94FDD369837D838E83E8
:1099D0009F8307C019821D821E821F8202C0BE8320
:1099E000AF8371100CC023E333E34BEC51E4D80197
:1099F0006D917D918D919C910E944AD805C0F8018E
:109A0000608171818281938129813D814E815F8155
:109A10000E94FDD3A885B9856D937D938D939C930A
:109A200013972CC0A885B9858D919D910D90BC91FF
:109A3000A02D89839A83AB83BC8371100EC023E36E
:109A400033E34BEC51E4F8016081718182819381B1
:109A50000E944AD89B01AC0105C0D8012D913D91CF
:109A60004D915C9169817A818B819C810E94FDD3AB
:109A7000E885F985608371838283938388859985DE
:109A800004968887998795E3E90EF11C0C5F1F4FB8
:109A9000A885B985AC56B24309F062CF6090A63272
:109AA0007090AA32F091A832F983C090A732209129
:109AB00020332D838CE0A80EB11CABE8B1E3A8875E
:109AC000B9874CE6E42E42E3F42EB8E1CB9E600168
:109AD00011248401F50161917191819191915F014E
:109AE0002CEA35EC47E257E30E94A5D587FD8CC0F0
:109AF000A885B9858C91882309F486C0815082306D
:109B000030F4F80124843584468457843BC06110C6
:109B100016C023E333E34BEC51E4D8011C966D915E
:109B20007D918D919C911F970E944AD820E030E052
:109B300044EB53E40E944AD81B012C010DC020E0E5
:109B400030E044EB53E4F80164857585868597859C
:109B50000E944AD81B012C012BED3FE049EC50E458
:109B6000A885B98591966D917D918D919C919497E1
:109B70000E944AD89B01AC01C201B1010E94ACD540
:109B80001B012C01711031C0B981B130E1F0F70136
:109B9000EC0DFD1DEC51F240A081B18192808380DB
:109BA000ED81E130A1F4F701E359FF4F20813181CC
:109BB00042815381BD01892D982D0E94FDD3DB0187
:109BC000982E892E04C0A0E0B0E0912C812CA20137
:109BD0009101BD01892D982D0E94FDD3D7016D9370
:109BE0007D938D939C9313970FC0A2019101F70170
:109BF00060817181828193810E94FDD3D7016D9331
:109C00007D938D939C931397E885F985F596E88766
:109C1000F987F4E0EF0EF11C0C5F1F4F88859985E2
:109C20008A52924309F056CF2996CDBFDEBFDF910D
:109C3000CF911F910F91FF90EF90DF90CF90BF9049
:109C4000AF909F908F907F906F905F904F903F90DC
:109C50002F90089580912830909129308F3E924125
:109C600011F08FE508958091DF339091E0338F3EBE
:109C70009241B9F78091B1329091B2328F3E9241C8
:109C800081F780912733909128338F3E924149F795
:109C900080917B5690917C568F3E924111F7809136
:109CA0003857909139578F3E9241D9F680E0089508
:109CB000CF93C82F0E949DA782E080932B328C2FD8
:109CC000CF91089580912C32811104C083E080935C
:109CD0002B3203C085E080932B3280E00895CF9330
:109CE000C82F0E940EB380E00E94AFAE8C2F0E945E
:109CF0009DA786E080932B328C2FCF91089580937F
:109D0000A53280E008958093A63280E00895809384
:109D1000AA3280E008954F925F926F927F929F9255
:109D2000AF92BF92CF92DF92EF92FF920F931F9369
:109D3000CF93DF93C82FB62E8A01F22ED32F8FEF49
:109D40008C0F863008F082C06091B33370E080E001
:109D500090E00E9447D62CEA35EC47E257E30E9498
:109D6000A5D587FD75C082E0B81619F0E4E1BE12F2
:109D700071C09090A632CF2CDD2E8C2F90E0EC019C
:109D8000CC0FDD1FC80FD91FCC0FDD1FCC0FDD1F7F
:109D9000CC0FDD1FCC5BDF4C780105EB12E3AA246E
:109DA000A394F60161917191819191916F012CEAD7
:109DB00035EC47E257E30E94A8D71816DCF5F2E02D
:109DC000BF1214C091100CC023E333E34BEC51E4F9
:109DD000F70160817181828193810E944AD824C0F9
:109DE000F70160817181828193811EC0F8014080FA
:109DF00051806280738091100EC023E333E34BECFB
:109E000051E4F70160817181828193810E944AD877
:109E10009B01AC0105C0F701208131814281538152
:109E2000C301B2010E94FCD3688379838A839B8338
:109E3000A09251322496F4E0EF0EF11C0C5F1F4FFC
:109E400082E30D3C180709F0ACCF06C081EA05C0DB
:109E50008CEA03C08DEA01C080E0DF91CF911F91B1
:109E60000F91FF90EF90DF90CF90BF90AF909F90B9
:109E70007F906F905F904F900895CF93DF93CDB711
:109E8000DEB76897CDBFDEBF8093A732682F70E042
:109E900080E090E00E9445D669837A838B839C831F
:109EA0001D821E821F82188619861A861B861C86B2
:109EB0001D861E861F86188A198A1A8A1B8A1C8A82
:109EC0001D8A1E8A1F8A188EAE014F5F5F4FBA012E
:109ED00089EE9AE40E94DB8280E06896CDBFDEBF07
:109EE000DF91CF910895CF93DF93EBE5F2E386E521
:109EF000DF011D928A95E9F78BE5A9E2B3E3ED0155
:109F0000982F19929A95E9F7A4E8B3E3ED01199215
:109F10008A95E9F78FEE92E180932830909329306B
:109F20008093DF339093E0338093B1329093B232D9
:109F3000809327339093283380937B5690937C565D
:109F40008093385790933957E0935932F0935A32AF
:109F5000809141308093A63280913F300E943D4FE6
:109F6000809140308093A532809142308093A93215
:109F7000809143308093AA3281E08093A432809311
:109F8000213394E090935F32109252321092533208
:109F90001092543280932B3280932A320E944DAD1E
:109FA000DF91CF910C941D84CF92DF92EF92FF92BC
:109FB000CF93C82F6A017B01E82FF0E0DF01AA0FE1
:109FC000BB1FAA0FBB1FAB54BD4C4D935D936D934C
:109FD0007C931397EE0FFF1FEE0FFF1FE05AFD4C0F
:109FE00040835183628373838C2F0E948E81B701DB
:109FF000A6018C2F0E949981CF91FF90EF90DF9066
:10A00000CF900C94A4819F92AF92BF92CF92DF9297
:10A01000EF92FF920F931F93CF93DF93CDB7DEB7ED
:10A020006897CDBFDEBF962EA72EC62ED72E7C01F9
:10A0300000E010E0B12CF601619171918191919154
:10A040006F012CEA35EC47E257E30E94A8D71816B7
:10A05000A4F58091A63281110EC023E333E34BECCB
:10A0600051E4F70160817181828193810E944AD815
:10A07000AB01BC0105C0F701408151816281738150
:10A08000E1E0F0E0EC0FFD1FE00FF11F4083518392
:10A0900062837383C801885D9F4CFC01E357FD4FC9
:10A0A0004083518362837383E555F1094083518373
:10A0B000628373838B2D0E948E81B3940C5F1F4F3C
:10A0C000F4E0EF0EF11C0831110509F0B4CF492D71
:10A0D0005A2DBE016F5F7F4F8CE897E40E94DB82B0
:10A0E00080E06896CDBFDEBFDF91CF911F910F91C9
:10A0F000FF90EF90DF90CF90BF90AF909F9008952A
:10A100004F925F926F927F928F929F92AF92BF9287
:10A11000CF92DF92EF92FF920F931F93CF93DF9333
:10A12000CDB7DEB76897CDBFDEBF21E020932033E7
:10A130008090A7329090A6325B016C0105EB12E390
:10A14000882D90E07C01EE0CFF1CE80EF91EEE0C51
:10A15000FF1CEE0CFF1CEE0CFF1CC7018C5B9F4C20
:10A160007C01F50161917191819191915F012CEADE
:10A1700035EC47E257E30E94A8D7181664F5F701BB
:10A180002081318142815381F80160817181828116
:10A1900093810E94FCD32B013C0191100EC023E35C
:10A1A00033E34BEC51E4F60160817181828193814C
:10A1B0000E944AD89B01AC0105C0F6012081318183
:10A1C00042815381C301B2010E94FCD3F801608F28
:10A1D000718F828F938FF4E0CF0ED11C0C5F1F4FD5
:10A1E00084E0E80EF11C92E30D3C190709F0B9CFA9
:10A1F000682D70E080E090E00E9445D669837A8304
:10A200008B839C831D821E821F82188619861A8664
:10A210001B861C861D861E861F86188A198A1A8A26
:10A220001B8A1C8A1D8A1E8A1F8A188EAE014F5FE8
:10A230005F4FBA0189EE9AE40E94DB8280E0689663
:10A24000CDBFDEBFDF91CF911F910F91FF90EF90B7
:10A25000DF90CF90BF90AF909F908F907F906F9046
:10A260005F904F900895CF93DF93CDB7DEB7689797
:10A27000CDBFDEBF109220331092CD321092CE327D
:10A280001092CF321092D0321092D1321092D2323C
:10A290001092D3321092D4321092D5321092D6321C
:10A2A0001092D7321092D8321092D9321092DA32FC
:10A2B0001092DB321092DC321092DD321092DE32DC
:10A2C0001092DF321092E0321092E1321092E232BC
:10A2D0001092E3321092E4326091A73270E080E095
:10A2E00090E00E9445D669837A838B839C831D828C
:10A2F0001E821F82188619861A861B861C861D865A
:10A300001E861F86188A198A1A8A1B8A1C8A1D8A29
:10A310001E8A1F8A188EAE014F5F5F4FBA0189EE09
:10A320009AE40E94DB8280E06896CDBFDEBFDF91B9
:10A33000CF910895CF93DF93CDB7DEB76897CDBFA8
:10A34000DEBF109220336091A73270E080E090E091
:10A350000E9445D669837A838B839C831D821E82EB
:10A360001F82188619861A861B861C861D861E86E5
:10A370001F86188A198A1A8A1B8A1C8A1D8A1E8AB5
:10A380001F8A188EAE014F5F5F4FBA0189EE9AE4C3
:10A390000E94DB8280E06896CDBFDEBFDF91CF9167
:10A3A0000895CF93DF93CDB7DEB76897CDBFDEBFFB
:10A3B00081E0809320336091A73270E080E090E0EC
:10A3C0000E9445D669837A838B839C831D821E827B
:10A3D0001F82188619861A861B861C861D861E8675
:10A3E0001F86188A198A1A8A1B8A1C8A1D8A1E8A45
:10A3F0001F8A188EAE014F5F5F4FBA0189EE9AE453
:10A400000E94DB8280E06896CDBFDEBFDF91CF91F6
:10A410000895CF9310925F320E947F4C809132302A
:10A42000813069F480E692E30E947C49C82F88233A
:10A4300031F00E949DA782E080932B3217C08BE5FC
:10A4400092E30E94874A85E080932B3280912C32E0
:10A45000811105C081E080932C320E94B0AB8BE566
:10A4600092E30E94A7960E94E24BC0E08C2FCF910E
:10A47000089588E1E5EBF2E3A5EEB2E301900D92D9
:10A480008A95E1F780E008950F931F93CF93DF93B0
:10A49000CDB7DEB76A97CDBFDEBF8C0181E0809378
:10A4A000A8328BE592E3698F7A8F0E94874A698D83
:10A4B0007A8DC8010E9409520E9415828823E1F317
:10A4C00088E1E0E0F0E2DE01119601900D928A95BC
:10A4D000E1F7BE016F5F7F4F85EE92E30E94095264
:10A4E0006A96CDBFDEBFDF91CF911F910F91089586
:10A4F00088E1E5EBF2E3ADEFB2E301900D928A95CE
:10A50000E1F780E008950F931F93CF93DF93CDB7CA
:10A51000DEB76A97CDBFDEBF8C0181E08093A832A1
:10A520008BE592E3698F7A8F0E94874A698D7A8DD5
:10A53000C8010E9409520E9415828823E1F388E134
:10A54000E0E0F0E2DE01119601900D928A95E1F7CC
:10A55000BE016F5F7F4F8DEF92E30E9409526A96B2
:10A56000CDBFDEBFDF91CF911F910F910895FB0109
:10A57000DC018091A432811111C09B01AD0160E02A
:10A5800070E080E89FE30E94ACD5609398327093AE
:10A59000993280939A3290939B3218C08091A63260
:10A5A000811109C023E333E34BEC51E4CD010E9458
:10A5B0004AD8FB0101C0CD01AF01BC0140939832E4
:10A5C0005093993260939A3270939B3280E0089551
:10A5D0008093A43280E008958093A93280E00895AA
:10A5E0006093A0327093A1328093A2329093A332F1
:10A5F0000E94338380E008950F931F93CF93DF93DE
:10A60000EC018B018091A432882399F080919832DB
:10A6100090919932A0919A32B0919B32BC01CD01B8
:10A620009F772CEA35EC47E257E30E94A5D587FDDA
:10A6300030C081E080935F32B801CE010E947F4C30
:10A6400080913230813069F480E692E30E947C4947
:10A65000C82F882331F00E949DA782E080932B327F
:10A6600019C08BE592E30E94874A85E080932B32E4
:10A6700080912C32811105C081E080932C320E94A0
:10A68000B0AB8BE592E30E94A796C82F0E94E24BE5
:10A6900001C0CEE88C2FDF91CF911F910F910895CB
:10A6A000CF93DF93CDB7DEB76897CDBFDEBF682FFE
:10A6B00070E080E090E00E9445D669837A838B83C6
:10A6C0009C831D821E821F82188619861A861B860D
:10A6D0001C861D861E861F86188A198A1A8A1B8A5E
:10A6E0001C8A1D8A1E8A1F8A188EAE014F5F5F4F1B
:10A6F000BA0188E797E40E94DB8280E06896CDBFCC
:10A70000DEBFDF91CF910895CF93DF93CDB7DEB752
:10A710006897CDBFDEBF6091AD3270E080E090E021
:10A720000E9445D669837A838B839C831D821E8217
:10A730001F82188619861A861B861C861D861E8611
:10A740001F86188A198A1A8A1B8A1C8A1D8A1E8AE1
:10A750001F8A188EAE014F5F5F4FBA0182E897E4FF
:10A760000E94DB8280E06896CDBFDEBFDF91CF9193
:10A770000895CF93DF93CDB7DEB76897CDBFDEBF27
:10A78000682F70E080E090E00E9445D669837A836C
:10A790008B839C831D821E821F82188619861A86CF
:10A7A0001B861C861D861E861F86188A198A1A8A91
:10A7B0001B8A1C8A1D8A1E8A1F8A188EAE014F5F53
:10A7C0005F4FBA018BEC97E40E94DB8280E06896D1
:10A7D000CDBFDEBFDF91CF910895CF93DF93CDB78B
:10A7E000DEB76897CDBFDEBF682F70E080E090E0F5
:10A7F0000E9445D669837A838B839C831D821E8247
:10A800001F82188619861A861B861C861D861E8640
:10A810001F86188A198A1A8A1B8A1C8A1D8A1E8A10
:10A820001F8A188EAE014F5F5F4FBA018CED97E41F
:10A830000E94DB8280E06896CDBFDEBFDF91CF91C2
:10A840000895CF93FC0160817181828193810E9480
:10A8500019D660932B3210922D328BE592E38093C0
:10A86000593290935A3280912C32813011F41092E7
:10A870002C3210922E32109254320E946096C09167
:10A880002B32C430C9F40E94335180913F300E9472
:10A890003D4F809140308093A5328091433080932A
:10A8A000AA3280E00E94AFAE80E00E94ED5381E0CA
:10A8B0008093A432C0935F3281E0CF910C9474AA4C
:10A8C00080931D3380931E338093263380E0089558
:10A8D0002CEA35EC47E257E36091CB337091CC33EF
:10A8E0008091CD339091CE330E94A8D71816B4F43E
:10A8F0008091703390917133A0917233B091733322
:10A90000BC01CD019F772CEA35EC47E257E30E946A
:10A91000A5D587FF03C010921D3303C081E080934B
:10A920001D3380E0089580931D33809170339091A2
:10A930007133A0917233B091733380931533909338
:10A940001633A0931733B093183380E008952CEAA0
:10A9500035EC47E257E36091CB337091CC33809173
:10A96000CD339091CE330E94A8D71816B4F48091BD
:10A97000703390917133A0917233B0917333BC01F5
:10A98000CD019F772CEA35EC47E257E30E94A5D52D
:10A9900087FF03C010921E3303C081E080931E33F3
:10A9A00080E0089580931E338091703390917133CD
:10A9B000A0917233B09173338093193390931A330B
:10A9C000A0931B33B0931C3380E008952CEA35EC40
:10A9D00047E257E36091CB337091CC338091CD3314
:10A9E0009091CE330E94A8D71816B4F4809170339A
:10A9F00090917133A0917233B0917333BC01CD014A
:10AA00009F772CEA35EC47E257E30E94A5D587FFF4
:10AA100003C01092263303C081E08093263380E088
:10AA20000895809326338091703390917133A09173
:10AA30007233B09173338093223390932333A09376
:10AA40002433B093253380E00895BC018DEE90E26D
:10AA50000C94056281E080935232089581E08093E6
:10AA60005332089581E08093543208951F93CF9319
:10AA7000DF93CDB7DEB76897CDBFDEBF0E949A9651
:10AA80008130B9F10E9443D20E94988280E00E94F6
:10AA9000C5AB10E0812F0E947296AB01BC01812FE3
:10AAA0000E94D44F1F5F1630A9F780E090E0A0E429
:10AAB000B0E489839A83AB83BC831D821E821F828C
:10AAC000188619861A861B861C861D861E861F867A
:10AAD000188A198A1A8A1B8A1C8A1D8A1E8A1F8A4A
:10AAE000188EBE016F5F7F4FCB010E94215480E022
:10AAF00001C08AE66896CDBFDEBFDF91CF911F917E
:10AB00000895809152328130A9F420912D32213064
:10AB100079F480912E3281110BC082E080932D3226
:10AB200083E296E58093593290935A3220932E32E5
:10AB30001092523280915332813091F480912D32B3
:10AB4000882331F0823061F490912E32943051F4A8
:10AB50000E949A96811104C0109253320E94365579
:10AB600090912E32809154328130C1F42091533231
:10AB7000211114C09150933088F01092543295E016
:10AB800090932E3290932B3290912C32911104C0DD
:10AB900080932C320E94B0AB0E940C9F80E00895FD
:10ABA00085E080932B3280912C32811105C081E0A9
:10ABB00080932C320C94B0AB0895CF93DF93CDB734
:10ABC000DEB76897CDBFDEBF80912C32882311F1AC
:10ABD00080E090E0A0E4B0E489839A83AB83BC83F7
:10ABE0001D821E821F82188619861A861B861C8665
:10ABF0001D861E861F86188A198A1A8A1B8A1C8A35
:10AC00001D8A1E8A1F8A188EBE016F5F7F4FCB017F
:10AC10000E9421546896CDBFDEBFDF91CF91089589
:10AC2000CF93DF93CDB7DEB76897CDBFDEBF80E0AF
:10AC300090E0A0E4B0E489839A83AB83BC831D8257
:10AC40001E821F82188619861A861B861C861D8600
:10AC50001E861F86188A198A1A8A1B8A1C8A1D8AD0
:10AC60001E8A1F8A188EAE014F5F5F4FBA0181E2C4
:10AC700094E50E94DB826896CDBFDEBFDF91CF9165
:10AC80000895CF93DF93CDB7DEB76897CDBFDEBF12
:10AC900080E090E0A0E8B0E489839A83AB83BC8332
:10ACA0001D821E821F82188619861A861B861C86A4
:10ACB0001D861E861F86188A198A1A8A1B8A1C8A74
:10ACC0001D8A1E8A1F8A188EAE014F5F5F4FBA0120
:10ACD00081E294E50E94DB826896CDBFDEBFDF9102
:10ACE000CF910895CF93DF93CDB7DEB72797CDBF30
:10ACF000DEBF97E0EFEDF0E2DE01119601900D92DC
:10AD00009A95E1F7873050F4E1E0F0E0EC0FFD1F99
:10AD1000E80FF11D87FDFA95808101C080E227963A
:10AD2000CDBFDEBFDF91CF910895EF92FF920F93D9
:10AD30001F93CF93DF931F92CDB7DEB77C018B01BA
:10AD4000642F70E080E090E049830E9445D6F701CF
:10AD5000618772878387948782E087834981E42FA4
:10AD6000F0E0EE0FFF1FE00FF11F659174914FE4CB
:10AD700050E084ED9CE30E94B8E1BC01C7010F9054
:10AD8000DF91CF911F910F91FF90EF900C94A761ED
:10AD9000CF93DF93EC010E94F249482F61E573E104
:10ADA000CE01DF91CF910C94955640912B3262E108
:10ADB00073E10C94955640912C3269EE72E10C943B
:10ADC000955640912D3265ED72E10C949556409167
:10ADD0002E3267EA72E10C94955640912F326AE860
:10ADE00072E10C949556E0915932F0915A32E55B3C
:10ADF000FF4F408164EB73E10C949556E09159321A
:10AE0000F0915A32E45BFF4F408160EC71E10C94A9
:10AE10009556E0915932F0915A32448166E271E1DF
:10AE20000C949556E0915932F0915A32E65BFF4FFF
:10AE3000408163EF70E10C949556E0915932F091A6
:10AE40005A32E25BFF4F408169EA70E10C949556FB
:10AE5000E0915932F0915A32E15BFF4F408168E650
:10AE600070E10C949556E0915932F0915A32E75BBB
:10AE7000FF4F408169EF7FE00C949556CF93DF93AD
:10AE8000EC01E0915932F0915A32EF5AFF4F608154
:10AE900070E080E090E00E9445D669877A878B87D2
:10AEA0009C8782E08F8380E0DF91CF910895CF93DC
:10AEB000DF93EC0160915B3270915C3280915D3286
:10AEC00090915E320E9445D669877A878B879C87EE
:10AED00082E08F8380E0DF91CF910895CF93DF935D
:10AEE000EC01E0915932F0915A3260817181828196
:10AEF00093810E9445D669877A878B879C8782E0F9
:10AF00008F8380E0DF91CF910895CF93DF93EC01A1
:10AF100080912D32811105C019861A861B861C86E8
:10AF200014C00E94699669877A878B879C872091D5
:10AF30006E5621110AC025E832E441E25DE30E9429
:10AF40004AD869877A878B879C878C819D81FC0191
:10AF5000EE0FFF1FE80FF91FEE0FFF1FEE0FFF1F91
:10AF6000EE0FFF1FE156FA4E85919491888784E099
:10AF70008F8380E0DF91CF910895CF93DF93EC0131
:10AF80002091593230915A32F901FD9660817181D8
:10AF90008281938169877A878B879C873E962081FF
:10AFA00021110AC025E832E441E25DE30E944AD85B
:10AFB00069877A878B879C878C819D81FC01EE0F46
:10AFC000FF1FE80FF91FEE0FFF1FEE0FFF1FEE0F21
:10AFD000FF1FE156FA4E85919491888784E08F8314
:10AFE00080E0DF91CF910895CF93DF93EC018C81C6
:10AFF0009D810E940448682F8091593290915A3265
:10B000000E94734B69877A878B879C878C819D818F
:10B01000FC01EE0FFF1FE80FF91FEE0FFF1FEE0FF1
:10B02000FF1FEE0FFF1FE156FA4E8591949188871E
:10B0300084E08F8380E0DF91CF910895CF93DF93F9
:10B04000EC018C819D810E940448209159323091FD
:10B050005A322B55324369F4E82FF0E0EE0FFF1F10
:10B06000EE0FFF1FEB54FD4C608171818281938153
:10B0700002C00E94729669877A878B879C878C8131
:10B080009D81FC01EE0FFF1FE80FF91FEE0FFF1F60
:10B09000EE0FFF1FEE0FFF1FE156FA4E85919491C0
:10B0A000888784E08F8380E0DF91CF910895CF93EC
:10B0B000DF93EC018C819D810E940448E09159321C
:10B0C000F0915A3294E0899FE00DF11D1124458DD5
:10B0D000568D678D70A149875A876B877C878C81D5
:10B0E0009D81FC01EE0FFF1FE80FF91FEE0FFF1F00
:10B0F000EE0FFF1FEE0FFF1FE156FA4E8591949160
:10B10000888784E08F8380E0DF91CF910895CF938B
:10B11000DF93EC010E941A5D69857A858B859C8599
:10B120000E9419D6462F60EE73E1CE01DF91CF91D8
:10B130000C949556CF93DF93EC018C819D810E94F6
:10B140000448833054F48F3FA9F407C0CE010E9415
:10B15000C45D80E01CC08DE61AC020E030E040E411
:10B1600050E469857A858B859C850E94A8D718163E
:10B1700094F3ECCF20E030E040E050E469857A853C
:10B180008B859C850E94A8D718162CF3DFCFDF9102
:10B19000CF91089595E3899FF0011124E350FF4C6E
:10B1A00060817181828193810895CF92DF92EF92C5
:10B1B000FF92CF93DF936A017B0125E3829FC00159
:10B1C0001124885D9F4CFC01EB52FF4F408351835B
:10B1D00062837383EC01C352DF4F20E034E244E723
:10B1E00059E4C701B6010E944AD89B01AC0160E056
:10B1F00070E080E89FE30E94ACD5688379838A83FE
:10B200009B83DF91CF91FF90EF90DF90CF900895D7
:10B21000CF92DF92EF92FF92CF93DF93EC01C9843C
:10B22000DA84EB84FC8420E034E244E759E4C7018B
:10B23000B6010E94A8D7181664F420E034E244E76F
:10B2400059E4C701B6010E94ACD569877A878B871C
:10B250009C87CE010E94C162C984DA84EB84FC849D
:10B260008C819D810E94044825E3829FC0011124A6
:10B27000885D9F4CFC01EB52FF4FC082D182E2827D
:10B28000F382EC01C352DF4F20E034E244E759E49B
:10B29000C701B6010E944AD89B01AC0160E070E092
:10B2A00080E89FE30E94ACD5688379838A839B837F
:10B2B00080E0DF91CF91FF90EF90DF90CF900895E5
:10B2C000CF92DF92EF92FF92CF93DF93EC01C9848C
:10B2D000DA84EB84FC8420E034E244E759E4C701DB
:10B2E000B6010E94A8D7181664F420E034E244E7BF
:10B2F00059E4C701B6010E94ACD569877A878B876C
:10B300009C87CE010E94C16280E0DF91CF91FF90C7
:10B31000EF90DF90CF90089581E08093533280E0EA
:10B3200008952CEA35EC47E257E3FC01618572850C
:10B33000838594850E94A8D7181614F40E94CA6ABF
:10B3400080E0089560915532709156328091573265
:10B350009091583208950E94D05E80E00E944D6D19
:10B3600080E008950E94D05E81E00E944D6D80E0F3
:10B3700008950E94D05E82E00E944D6D80E00895A5
:10B380000E94D05E83E00E944D6D80E00895CF93CF
:10B39000DF93EC01E0915932F0915A32E55BFF4FB7
:10B3A000E081F0E0EE0FFF1FED5EFB4E65917491C2
:10B3B0004FE450E084ED9CE30E94B8E1AC0162EE02
:10B3C0007FE0CE01DF91CF910C94F7C1CF93DF9353
:10B3D000EC01E0915932F0915A32E55BFF4FE08188
:10B3E000F0E0EE0FFF1FED5EFB4E659174914FE4B0
:10B3F00050E084ED9CE30E94B8E1AC016AEC7FE090
:10B40000CE01DF91CF910C94F7C1CF93DF93EC0184
:10B4100081EF90E20E941DE3CE010E94C759CE0148
:10B420000E94E65966EB7FE0CE010E94BEC16DE945
:10B430007FE0CE010E9489C164E87FE0CE010E94D6
:10B4400089C16BE67FE0CE010E9489C162E57FE0A1
:10B45000CE010E9489C169E37FE0CE010E9489C1CB
:10B4600060E27FE0CE010E9489C167E07FE0CE010B
:10B470000E9489C16EEE7EE0CE010E9489C165ED19
:10B480007EE0CE010E9489C16CEB7EE0CE010E947D
:10B4900089C163EA7EE0CE010E9489C16AE87EE04C
:10B4A000CE010E9489C161E77EE0CE010E9489C180
:10B4B00068E57EE0CE010E94BEC180E0DF91CF91C1
:10B4C000089566EB7FE00C94BEC16DE97FE00C94BB
:10B4D00089C164E87FE00C9489C16BE67FE00C943D
:10B4E00089C162E57FE00C9489C169E37FE00C9437
:10B4F00089C160E27FE00C9489C167E07FE00C9431
:10B5000089C16EEE7EE00C9489C165ED7EE00C94FD
:10B5100089C16CEB7EE00C9489C163EA7EE00C94F7
:10B5200089C16AE87EE00C9489C161E77EE00C94F1
:10B5300089C168E57EE00C94BEC16CED7DE00C94A1
:10B54000BEC16BEA7DE00C94BEC166E77DE00C9461
:10B55000BEC16BE37DE00C94BEC167E07DE00C945E
:10B56000BEC1CF93DF93EC01E0915932F0915A3292
:10B57000E55BFF4FE081F0E0EE0FFF1FED5EFB4E5D
:10B58000659174914FE450E084ED9CE30E94B8E132
:10B59000AC0163EE7CE0CE01DF91CF910C94F7C15A
:10B5A000CF93DF93EC01E0915932F0915A32E55B91
:10B5B000FF4FE081F0E0EE0FFF1FED5EFB4E659167
:10B5C00074914FE450E084ED9CE30E94B8E1AC013B
:10B5D00062EC7CE0CE01DF91CF910C94F7C165EA7B
:10B5E0007CE00C949FC1CF93DF93EC01E091593242
:10B5F000F0915A32E55BFF4FE081F0E0EE0FFF1F64
:10B60000ED5EFB4E659174914FE450E084ED9CE358
:10B610000E94B8E1AC0166E87CE0CE01DF91CF91F9
:10B620000C94F7C10F931F93CF93DF938C01FC0110
:10B6300061857285838594850E9419D6E62FF0E096
:10B64000EE0FFF1FE052FC4E659174914FE450E005
:10B6500084ED9CE30E94B8E1E8012D969F938F93BF
:10B66000F80161857285838594850E9419D61F92A1
:10B670006F93DF93CF930F5E1F4F1F930F93DF9353
:10B68000CF938AE69CE09F938F93ECEDF9E581815F
:10B690008F9380818F930E947FE2EDB7FEB73E9635
:10B6A000EDBFFEBFDF91CF911F910F91089562E42E
:10B6B0007CE00C9476486AE17CE00C94764868EF74
:10B6C0007BE00C94764866ED7BE00C94764864EA67
:10B6D0007BE00C94764863E77BE00C9476486AE361
:10B6E0007BE00C9476486AE17BE00C94764868ED48
:10B6F0007AE00C94444866E97AE00C9444486FE69A
:10B700007AE00C94764869E47AE00C94764868E232
:10B710007AE00C94764868E07AE00C9476486BEE18
:10B7200079E00C94C9486CEC79E00C94C948BC01F0
:10B73000675F7F4F2091A63242E45EE0FC01848186
:10B7400095810C942049BC01675F7F4F21E048E25E
:10B750005EE0FC01848195810C942049BC01675F07
:10B760007F4F21E04FE05EE0FC01848195810C94E5
:10B7700020490F931F93CF93DF93EC010C811D8120
:10B780000E94746408171907C4F48C819D81FC0120
:10B79000EE0FFF1FE80FF91FEE0FFF1FEE0FFF1F49
:10B7A000EE0FFF1FEC55FA4E25913491CE01F901B1
:10B7B000DF91CF911F910F91199485E1DF91CF9186
:10B7C0001F910F9108950F931F93CF93DF93EC0177
:10B7D0000C811D810E94746408171907C4F48C81C0
:10B7E0009D81FC01EE0FFF1FE80FF91FEE0FFF1FF9
:10B7F000EE0FFF1FEE0FFF1FEE55FA4E259134910D
:10B80000CE01F901DF91CF911F910F91199485E13C
:10B81000DF91CF911F910F9108950F931F93CF93B5
:10B82000DF93EC010C811D810E94746408171907D5
:10B83000C4F48C819D81FC01EE0FFF1FE80FF91FFE
:10B84000EE0FFF1FEE0FFF1FEE0FFF1FE056FA4E29
:10B8500025913491CE01F901DF91CF911F910F9184
:10B860001994DF91CF911F910F910895CF93DF939A
:10B87000EC018C819D810E9487648823C9F08C81B2
:10B880009D81FC01EE0FFF1FE80FF91FEE0FFF1F58
:10B89000EE0FFF1FEE0FFF1FE256FA4EE491E1FF9D
:10B8A00005C0CE01DF91CF910C94B48080E001C03F
:10B8B00085E1DF91CF9108950F931F93CF93DF938D
:10B8C000EC0181E00E94834E1C821D8280E090E0AA
:10B8D0008E010F5E1F4F47C08C819D819C01220FFE
:10B8E000331FF901E80FF91FEE0FFF1FEE0FFF1FC7
:10B8F000EE0FFF1FE256FA4EE491E0FF2EC0280F34
:10B90000391F220F331F220F331F220F331F2855D9
:10B910003A4EF901459155916591749149875A873D
:10B920006B877C87BC01660F771F680F791F660FD6
:10B93000771F660F771F660F771F68567A4E45E0B0
:10B9400050E0C8010E94B8E1CE010E94B95BCE016F
:10B950000E94365C2C813D8101C09C012F5F3F4FCE
:10B960002C833D83C9010E9477648111B5CF81E0AA
:10B970000E9423A8DF91CF911F910F910C940BA8E7
:10B98000CF93DF93EC012CEA35EC47E257E369856E
:10B990007A858B859C850E94A5D587FF05C0CE0141
:10B9A000DF91CF910C94AE79CE010E945C5C82E075
:10B9B0008F8340E050E060E87FE349875A876B87D8
:10B9C0007C8780E0DF91CF910895809196399091A6
:10B9D00097398F3E924111F08AE508958091D839C8
:10B9E0009091D9398F3E9241B9F780916C34909102
:10B9F0006D348F3E924181F780918E3790918F37D1
:10BA00008F3E924149F780919037909191378F3EC8
:10BA1000924111F780919439909195398F3E9241DE
:10BA2000D9F68091233D8111D7CF0895FC0117826B
:10BA300089E60895CF93DF93EC018C819D81FC0111
:10BA4000EE0FFF1FE80FF91FEE0FFF1FEE0FFF1F96
:10BA5000EE0FFF1FEA55FA4EA591B4916C9170E07C
:10BA600080E090E00E9445D669877A878B879C8723
:10BA700082E08F8380E0DF91CF910895CF93DF93B1
:10BA8000EC018C819D81FC01EE0FFF1FE80FF91F77
:10BA9000EE0FFF1FEE0FFF1FEE0FFF1FEA55FA4ECE
:10BAA000A591B4916D917D918D919C910E9445D607
:10BAB00069877A878B879C8782E08F8380E0DF911C
:10BAC000CF910895CF93DF93DC0114968D919C91D3
:10BAD0001597FC01EE0FFF1FE80FF91FEE0FFF1F78
:10BAE000EE0FFF1FEE0FFF1FEA55FA4EC591D491DE
:10BAF000488159816A817B8119964D935D936D933D
:10BB00007C931C9783E017968C9380E0DF91CF9114
:10BB10000895CF93DF93DC0114968D919C91159736
:10BB2000FC01EE0FFF1FE80FF91FEE0FFF1FEE0FD6
:10BB3000FF1FEE0FFF1FEA55FA4EC591D4914881C1
:10BB400059816A817B8119964D935D936D937C93A6
:10BB50001C97FC01EE0FFF1FE80FF91FEE0FFF1FF0
:10BB6000EE0FFF1FEE0FFF1FE156FA4E85919491E5
:10BB700018968C93189784E017968C9380E0DF9149
:10BB8000CF91089588E608950F931F93CF93DF9385
:10BB9000EC018C819D81FC01EE0FFF1FE80FF91F66
:10BBA000EE0FFF1FEE0FFF1FEE0FFF1FEA55FA4EBD
:10BBB0000591149169857A858B859C850E9419D69B
:10BBC000F801608382E08F8380E0DF91CF911F9145
:10BBD0000F910895CF93DF93EC0169857A858B856A
:10BBE0009C850E9419D66230B0F48C819D81FC0145
:10BBF000EE0FFF1FE80FF91FEE0FFF1FEE0FFF1FE5
:10BC0000EE0FFF1FEA55FA4EA591B4916C9382E0B6
:10BC10008F8380E001C08EE6DF91CF910895CF93AE
:10BC2000DF93EC0169857A858B859C850E9419D606
:10BC30006330B0F48C819D81FC01EE0FFF1FE80F93
:10BC4000F91FEE0FFF1FEE0FFF1FEE0FFF1FEA554C
:10BC5000FA4EA591B4916C9382E08F8380E001C08D
:10BC60008EE6DF91CF910895CF93DF93EC01698544
:10BC70007A858B859C850E9419D66430B0F48C81BE
:10BC80009D81FC01EE0FFF1FE80FF91FEE0FFF1F54
:10BC9000EE0FFF1FEE0FFF1FEA55FA4EA591B4916C
:10BCA0006C9382E08F8380E001C08EE6DF91CF91BC
:10BCB00008950F931F93CF93DF93EC018C819D81A7
:10BCC000FC01EE0FFF1FE80FF91FEE0FFF1FEE0F35
:10BCD000FF1FEE0FFF1FEA55FA4E0591149169857B
:10BCE0007A858B859C850E9419D6F80160837183C3
:10BCF00082E08F8380E0DF91CF911F910F910895B3
:10BD00000F931F93CF93DF93EC018C819D81FC01F6
:10BD1000EE0FFF1FE80FF91FEE0FFF1FEE0FFF1FC3
:10BD2000EE0FFF1FEA55FA4E0591149169857A8549
:10BD30008B859C850E9419D6F8016083718382836C
:10BD4000938382E08F8380E0DF91CF911F910F91E9
:10BD50000895CF93DF93DC0114968D919C911597F4
:10BD6000FC01EE0FFF1FE80FF91FEE0FFF1FEE0F94
:10BD7000FF1FEE0FFF1FEA55FA4EC591D491199699
:10BD80004D915D916D917C911C97488359836A8395
:10BD90007B8383E017968C9380E0DF91CF910895A9
:10BDA000CF93DF93DC0114968D919C911597FC0144
:10BDB000EE0FFF1FE80FF91FEE0FFF1FEE0FFF1F23
:10BDC000EE0FFF1FEA55FA4EC591D49119964D9189
:10BDD0005D916D917C911C97488359836A837B8325
:10BDE000FC01EE0FFF1FE80FF91FEE0FFF1FEE0F14
:10BDF000FF1FEE0FFF1FE156FA4E859194911896A2
:10BE00008C93189784E017968C9380E0DF91CF9104
:10BE100008951F93CF93DF93EC018091F839882325
:10BE2000D1F01DE10A80DB81C02D209711F480E064
:10BE300013C08F818F3FD9F3811104C0CE010E94BE
:10BE4000E35B06C0CE010E94B95BCE010E94365C66
:10BE5000115041F7ECCF85E6DF91CF911F91089506
:10BE6000CF93DF93EC01BC018FEF90E20E94F1E1F0
:10BE7000892B41F0BE0182E091E20E94F1E121E0D4
:10BE8000892B09F420E0822FDF91CF9108950F9341
:10BE90001F93CF93DF93CDB7DEB72997CDBFDEBF1A
:10BEA0008B0144E050E0BC01CE0101960E9411E2FA
:10BEB00046E050E0B801CE0101960E9401E20E94E6
:10BEC0007464181619060CF03FC07981AA81BB81F1
:10BED0001C810D8128E935E140E050E0F9016491D1
:10BEE000671327C03196E491E11103C0A11121C06D
:10BEF00029C0EA131EC0F9013296E491E11103C092
:10BF0000B11117C01FC0EB1314C0F9013396E491AF
:10BF1000E11103C011110DC015C0E1130AC0F901F0
:10BF20003496E491E11103C0011103C00BC0E01786
:10BF300049F04F5F5F4F285E3F4F4817590709F0A0
:10BF4000CDCF02C0CA0102C08FEF9FEF2996CDBFAF
:10BF5000DEBFDF91CF911F910F910895CF93DF93B3
:10BF6000FC012189222371F1EC016196BE0186E07A
:10BF700091E20E94F1E1892B39F1BE018FEF90E24D
:10BF80000E94F1E1892B11F1BE0189E091E20E944A
:10BF9000F1E1892BD9F0BE018DEE90E20E94F1E132
:10BFA000892BB1F0BE018CE091E20E94F1E1892B76
:10BFB00079F0BE0180EE91E20E94F1E1892B51F40B
:10BFC00085E009C080E007C082E005C083E003C0CF
:10BFD00084E001C081E0DF91CF910895FC018FEFF3
:10BFE0008783148215821186128613861486108622
:10BFF000118A1586178A108EA081B181109711F4CD
:10C0000016820DC017968C911797873029F41696D3
:10C010008C918F5F868303C016968C918683CF01A7
:10C020000895EF92FF920F931F93CF93DF93EC014C
:10C030000C811D810E947464081719070CF06FC0F1
:10C040000C811D81CE010E94EE5F0C831D837E0159
:10C0500081E1E80EF11CB801660F771F600F711FB8
:10C06000660F771F660F771F660F771F68567A4E29
:10C07000C7010E9499E18E01035F1F4F2C813D8112
:10C08000B901660F771F620F731F660F771F660F68
:10C09000771F660F771F6C567A4EC8010E9499E190
:10C0A0008D85882311F18C819D81FC01EE0FFF1F8E
:10C0B000E80FF91FEE0FFF1FEE0FFF1FEE0FFF1F20
:10C0C000E256FA4EE491E2FF02C01D8610C0F8016C
:10C0D00001900020E9F7BF01601B710B605F7F4F8B
:10C0E0006C0F7D1FC7010E94FAE18C819D81FC01CC
:10C0F000EE0FFF1FE80FF91FEE0FFF1FEE0FFF1FE0
:10C10000EE0FFF1FEE55FA4E25913491CE01F90145
:10C11000DF91CF911F910F91FF90EF901994DF91D4
:10C12000CF911F910F91FF90EF9008958F929F9262
:10C13000AF92BF92CF92DF92EF92FF920F931F9335
:10C14000CF93DF9300D01F92CDB7DEB76C015C01B7
:10C1500081E1A80EB11C87E0F6018783A4E9EA2EED
:10C16000A5E1FA2E00E010E01DC0B701CE01019656
:10C170000E9499E1BE016F5F7F4FC5010E94F1E10E
:10C18000892B59F44601F9E18F0E911CF601058FB8
:10C19000168FC4010E94116064010F5F1F4FF8E108
:10C1A000EF0EF11CC8010E9477648111DECF249646
:10C1B000CDBFDEBFDF91CF911F910F91FF90EF9028
:10C1C000DF90CF90BF90AF909F908F900895CF93C6
:10C1D000DF931092923710929337A5E5B4E3EEE621
:10C1E000F4E391E08FEFA083B18379965B96ED93B2
:10C1F000FC935C975D961D921C925E97EF0163978E
:10C20000988322961882219788832A9618825996B5
:10C2100027E3EE38F20739F7109277371092783724
:10C2200010926E3410926F341092743487E08093C1
:10C23000753482E790E080937F349093803487E870
:10C2400094E3DF91CF9108950F931F93CF93DF93E2
:10C250000E94E760EC018FEE92E180939639909313
:10C2600097398093D8399093D93980936C349093CF
:10C270006D3480938E3790938F378093903790935F
:10C280009137809394399093953981E00E94834E41
:10C290001C821D82CE010E948B802091E03930915A
:10C2A000E1394091E2395091E33969857A858B858E
:10C2B0009C850E94A5D5882339F0CE01DF91CF91CE
:10C2C0001F910F910C945C5C0E9410A81C821D822F
:10C2D00080E090E08E010F5E1F4F2FC06C817D814A
:10C2E0009B01220F331FF901E60FF71FEE0FFF1F0F
:10C2F000EE0FFF1FEE0FFF1FE256FA4EE491E0FF34
:10C3000017C0620F731F660F771F660F771F660FC8
:10C31000771F68567A4E45E050E0C8010E94B8E1A8
:10C32000CE010E948B80CE010E94B95B6C817D8121
:10C330006F5F7F4F6C837D83CB010E947764811197
:10C34000CDCFDF91CF911F910F910C9423A8EF9245
:10C35000FF920F931F93CF93DF938C01209192371D
:10C3600030919337EB0109900020E9F72197C61B24
:10C37000D70BAE01420F531F41305240D8F4F901A0
:10C38000EC56F84C7F01AE014F5F5F4FCF010E942A
:10C39000D2E140919237509193374F5F5F4F4C0FEE
:10C3A0005D1F4093923750939337F801E78AF08EE0
:10C3B00080E001C08DE0DF91CF911F910F91FF9040
:10C3C000EF900895CF93DF932EE1C7E8D4E33F8148
:10C3D0003F3F59F00A80DB81C02D209719F480E09F
:10C3E00090E010C0215099F7FACFBC0184E493E2A9
:10C3F0000E94475F8C839D83019689F3CE010E9442
:10C400001160CE01DF91CF910895EF92FF920F93CB
:10C410001F93CF93DF938B012EE1C7E8D4E33F81D5
:10C420003F3F59F00A80DB81C02D209719F480E04E
:10C4300090E01DC0215099F7FACF7E0121E1E20E74
:10C44000F11C45E050E0BC01C7010E9411E2B801B7
:10C45000CE010E94A7618111EACFB70184E493E283
:10C460000E94475F8C839D8385E08F83CE01DF919F
:10C47000CF911F910F91FF90EF9008952091F8397F
:10C48000213021F42091D03C213029F4BC018DEEE3
:10C4900090E20C94056280E090E008959091F83964
:10C4A000913019F4642F0C94077F0C9409C1CF9339
:10C4B000DF93EC018091E52F811103C00E943BD2F4
:10C4C00002C00E9449C9682F70E080E090E00E949D
:10C4D00045D669877A878B879C8782E08F8380E047
:10C4E000DF91CF9108950F931F93CF93DF93CDB733
:10C4F000DEB7C058D109CDBFDEBFFC0161857285B2
:10C50000838594850E9419D68FEF860F863030F090
:10C5100080E491E20E943E628EE62AC06093E02FA2
:10C5200081E08093E12FE62FF0E0EE0FFF1FE15A4C
:10C53000FA4E659174914FE450E084ED9CE30E94C3
:10C54000B8E19F938F9386E294E19F938F938E013E
:10C550000F5F1F4F1F930F930E9473E3C8010E9448
:10C560003E620F900F900F900F900F900F9080E011
:10C57000C058DF4FCDBFDEBFDF91CF911F910F912C
:10C5800008950F931F93CF93DF93EC018BE592E314
:10C590000E944E4A882329F009851A858B859C853F
:10C5A00011C023E333E34BEC51E469857A858B8535
:10C5B0009C850E944AD88B01AB01BC0149875A87F0
:10C5C0006B877C872C813D81F901EE0FFF1FE20F05
:10C5D000F31FEE0FFF1FEE0FFF1FEE0FFF1FEA55B9
:10C5E000FA4EA591B491A801BC014D935D936D9352
:10C5F0007C931397F901EE0FFF1FE20FF31FEE0F6D
:10C60000FF1FEE0FFF1FEE0FFF1FE156FA4E859141
:10C610009491888784E08F8380E0DF91CF911F9190
:10C620000F91089560E375E10C949FC16CE075E192
:10C630000C949FC160ED74E10C949FC16CE974E1AE
:10C640000C949FC16FE474E10C949FC11F93CF932E
:10C65000DF93EC0110E08881882301F10E94E760FC
:10C6600045E050E0BE0188E994E30E9411E268E9E8
:10C6700074E384E493E20E94475F80938B34909349
:10C680008C3487E894E30E94116042E063E080E02C
:10C690000E944E621F5F26961D31E9F684E0DF910D
:10C6A000CF911F910895CF93DF93CDB7DEB7EC976D
:10C6B000CDBFDEBF8CE3E8E1F0E2DE011196019030
:10C6C0000D928A95E1F7CE0101960E942663EC96C1
:10C6D000CDBFDEBFDF91CF910895CF93DF93CDB76C
:10C6E000DEB7AA97CDBFDEBF8AE2E4E5F0E2DE0165
:10C6F000119601900D928A95E1F7CE0101960E9464
:10C700002663AA96CDBFDEBFDF91CF910895CF9368
:10C71000DF93CDB7DEB76E97CDBFDEBF8EE1EEE71C
:10C72000F0E2DE01119601900D928A95E1F7CE01BB
:10C7300001960E9426636E96CDBFDEBFDF91CF913A
:10C740000895CF93DF93EC0143E759E763E770E087
:10C75000498B5A8B6B8B7C8B0E94966042E063E026
:10C7600080E00E944E62CE010E948763CE010E944B
:10C770006D6320E731E340E0298B3A8B4B8BCE0190
:10C780000E94966042E063E080E00E944E62CE012B
:10C79000DF91CF910C945363CF92DF92EF92FF928F
:10C7A000FC01C184D284E384F48420E030E040E8DA
:10C7B0005FE3C701B6010E94A8D71816FCF0C701B5
:10C7C000B6010E9419D66093E22FC701B6019F7788
:10C7D0002CEA35EC47E257E30E94A8D718163CF440
:10C7E00060E470E080E00E9429C780E008C060E853
:10C7F00070E080E00E9429C780E001C08EE6FF90D3
:10C80000EF90DF90CF900895CF92DF92EF92FF925A
:10C81000FC01C184D284E384F48420E030E040E071
:10C8200050E4C701B6010E94A8D71816FCF0C70152
:10C83000B6010E9419D66093E42FC701B6019F7715
:10C840002CEA35EC47E257E30E94A8D718163CF4CF
:10C8500064E070E080E00E9429C780E008C068E0E2
:10C8600070E080E00E9429C780E001C08EE6FF9062
:10C87000EF90DF90CF900895CF92DF92EF92FF92EA
:10C88000FC01C184D284E384F48420E030E040E8F9
:10C890005FE3C701B6010E94A8D71816FCF0C701D4
:10C8A000B6010E9419D66093E32FC701B6019F77A6
:10C8B0002CEA35EC47E257E30E94A8D718163CF45F
:10C8C00060E170E080E00E9429C780E008C060E27B
:10C8D00070E080E00E9429C780E001C08EE6FF90F2
:10C8E000EF90DF90CF9008958CE891E0089521E0DB
:10C8F0008334914008F020E0822F08959C012F5549
:10C90000314081E02932310508F080E0089521E0CE
:10C910008036914008F020E0822F0895CF92DF9278
:10C92000EF92FF92CF93DF93EC01C984DA84EB841A
:10C93000FC84A7019601C701B6010E946BD9811141
:10C940003CC0E894F7F82FEF3FEF4FE75FE7C701F0
:10C95000B6010E946BD981110AC02FEF3FEF4FE75C
:10C960005FE7C701B6010E94A5D5181634F18C8186
:10C970009D81FC01EE0FFF1FE80FF91FEE0FFF1F57
:10C98000EE0FFF1FEE0FFF1FE256FA4EE491E3FF9A
:10C9900014C08BE592E30E944E4A81110EC025E837
:10C9A00032E441E25DE369857A858B859C850E944E
:10C9B0004AD869877A878B879C87DF91CF91FF90D0
:10C9C000EF90DF90CF9008958091E12F882349F078
:10C9D0001092E12F6091E02F80E00E9431C780E04B
:10C9E000089583E00895CF93DF93E091163AF09194
:10C9F000173A04C0E093163AF093173AEF01819189
:10CA0000982F9D7F9032B1F38930A1F34FE750E02A
:10CA1000BE018AE19CE30E9411E26881611105C0B8
:10CA20008091F83981116DC039C0613221F4DF91F4
:10CA3000CF910C942A55653221F4DF91CF910C945B
:10CA40002E556E3721F4DF91CF910C9432556F3310
:10CA500079F4FE0101900020E9F73197EC1BFD0B02
:10CA6000329780F02196C093163AD093173A49C076
:10CA70006B3741F481E08093F839CE01DF91CF919B
:10CA80000C94047A70E080E791E20E94E6E1892B41
:10CA900059F01092F839CE010E9461BD6AE17CE341
:10CAA000DF91CF910C94A1BE8091F839811109C01A
:10CAB000CE010E9417706AE17CE3DF91CF910C9464
:10CAC000A1BE0E94E760EC0127E633E640E0298B37
:10CAD0003A8B4B8B6091163A7091173A0E94A7617E
:10CAE00085E08F838091163A9091173A0E941770D3
:10CAF00042E060E00E944E6280E0DF91CF910C94B2
:10CB000074AADF91CF910895FF920F931F93CF9353
:10CB1000DF931F921F92CDB7DEB7F82EEAEDF9E34F
:10CB200022EC32E0DF01C9011D920197E9F72FEEF7
:10CB300032E12083318320939A3C30939B3C0FE871
:10CB400012E22CED33E40093E0391093E1392093A5
:10CB5000E2393093E3390CEE11E528E73FE3009327
:10CB6000E4391093E5392093E6393093E73900E052
:10CB700010E020EA30E40093E8391093E93920937B
:10CB8000EA393093EB3900E010E020E83FE300930E
:10CB9000EC391093ED392093EE393093EF3983E07F
:10CBA0008093F9398F2D4A8369830E9441C7698137
:10CBB000862F0E944CC74A81842F0E9457C7F0924B
:10CBC000DF2FF092DD2F0F900F90DF91CF911F910B
:10CBD0000F91FF900895CF93DF931F921F92CDB7CF
:10CBE000DEB780E6F82E01E010E00E946C7882301B
:10CBF000E1F30E9473788230C1F30E942D4A86309F
:10CC000009F0D9C00E942BC58090FF399090003A5E
:10CC1000A090013AB090023A86169706A806B90687
:10CC200020F70E942BC56C597F4F8F4F9F4F609309
:10CC3000FF397093003A8093013A9093023A0E9430
:10CC4000E277D3CF0E943CBC882329F08CEC0E9471
:10CC50006F4E823051F20E948155823031F20E9433
:10CC6000669D823011F20E94E55C8093243D811123
:10CC70002EC08091DA399091DB398F3E924109F0D4
:10CC8000AAC080919A3C90919B3C8F3E924109F0C2
:10CC9000A2C097C00E9460818093243D811117C07B
:10CCA0000E94C9B28093243D811111C00E94E26F9D
:10CCB0008093243D81110BC00E9450C68093243D77
:10CCC000811105C00E949DB3823031F48ECF0E9445
:10CCD0006F4E8230B9F789CF0E94A6AA823009F43C
:10CCE00084CF0E9412AC823009F47FCF0E94CEAC78
:10CCF000823009F47ACF09831A8368E17AE3CE019E
:10CD000001960E9466C78093163A9093173A8F3F18
:10CD10002FEF920739F48DE00E94584E823009F4CB
:10CD200064CF04C0892B11F00E94F3640E94C58B6C
:10CD3000823009F45ACF0E94196B823009F455CF22
:10CD40000E94D86D823009F450CF0E94BD6F8230AE
:10CD500009F449CF0E94FC4B823009F444CF0E9471
:10CD600015828430F0F53FCF8091F939843038F462
:10CD700084E08093F9390E942E550E9415A883E023
:10CD800090E089839A8368E17AE3CE0101960E945C
:10CD900066C78093163A9093173A8F3F2FEF92070A
:10CDA00021F48DE00E94584E1ECF892B09F41BCF31
:10CDB0000E94F36418CF0E942D4A823009F44BCFB1
:10CDC00041CF1092243D0E942A4E8093243D882317
:10CDD00009F460CF7CCFF092243D80E60E946F4E34
:10CDE00078CF8091222A9091232A0E94AFD0682F79
:10CDF00070E080E090E00E9447D620E030E048E418
:10CE000051E40E94A8D787FFEECE0E94E4648230EE
:10CE100009F0AACFE8CE8091DF2F8093DD2F08950F
:10CE20008093DD2F08958093DE2F0895CF93C82F30
:10CE300080918F23882379F040E050E0BA018C2F55
:10CE40000E94D44FEC2FFF27E7FDF095E05DFD4CED
:10CE500081E080830AC06C2F83E296E50E94734BC9
:10CE6000AB01BC018C2F0E94D44F4091B62350914E
:10CE7000B7236091B8237091B9238C2F0E94D558A5
:10CE80008FED98E6809390239093912382E0CF9149
:10CE90000895CF92DF92EF92FF920F931F93CF935B
:10CEA000DF93CDB7DEB7E097CDBFDEBF98E17E015F
:10CEB000A9E1EA0EF11CF701A92F1192AA95E9F751
:10CEC000FE0131966F0111929A95E9F7F60194E00F
:10CED0008902E00DF11D1124408F518F628F738FF5
:10CEE00080E090E0A0E8BFE380839183A283B383D6
:10CEF000009398321093993220939A3230939B3258
:10CF00000E9498820E943255B601C7010E94FC52CD
:10CF10008093243D811101C082E0E096CDBFDEBF49
:10CF2000DF91CF911F910F91FF90EF90DF90CF9005
:10CF300008950F931F93E0918923FF27E7FDF09554
:10CF4000EB5FFF4C9381913099F400919A231091FB
:10CF50009B2320919C2330919D234091A2235091AB
:10CF6000A3236091A4237091A5230E9449671DC04B
:10CF7000E0918A23FF27E7FDF095EB5FFF4C93815B
:10CF8000913099F400919A2310919B2320919C2336
:10CF900030919D234091A2235091A3236091A4231B
:10CFA0007091A52370580E9449678FED97E6809392
:10CFB00090239093912382E01F910F9108950F93F6
:10CFC0001F93CF93C82F85E3C802F0011124EF5FB0
:10CFD000FE4C40815181628173818C2F0E94D55813
:10CFE00000919A2310919B2320919C2330919D23A3
:10CFF00040919623509197236091982370919923A3
:10D000008C2F0E9449678EE698E680939023909338
:10D01000912382E0CF911F910F9108950F931F9359
:10D0200000919A2310919B2320919C2330919D2362
:10D030004091A6235091A7236091A8237091A92322
:10D040000E94496786E197E680939023909391230D
:10D0500082E01F910F9108950E9498828091AF23E2
:10D060000E943D4F8091AE230E94834E8091B02359
:10D070000E94874E8091B1230E94E8528091B22392
:10D080009091B323A091B423B091B52380939832AB
:10D0900090939932A0939A32B0939B3264E08BE5DF
:10D0A00092E30E946B4A0E94DD5510922C3280E080
:10D0B0000895CF93C82F4091B6235091B723609124
:10D0C000B8237091B9230E94D5588C2F0E942C68E8
:10D0D00080E00E9474AA80EFCF9108950F931F9370
:10D0E000E0918923FF27E7FDF095EB5FFF4C9381EB
:10D0F000913039F089E598E68093902390939123BD
:10D1000018C000919E2310919F232091A02330915D
:10D11000A1234091A2235091A3236091A423709155
:10D12000A5230E9449678EE098E680939023909310
:10D13000912382E01F910F910895FF920F931F9307
:10D14000CF93DF93CDB7DEB7C058D109CDBFDEBFD7
:10D15000F82E0E94E7608EEFF81205C085E791E295
:10D160000E943E6219C08F2D0E9472561F928F93AB
:10D1700024EB3AE33F932F938E010F5F1F4F1F93D2
:10D180000F930E9473E3C8010E943E620F900F90BC
:10D190000F900F900F900F9042E062E080EF0E949E
:10D1A0004E628F2D0E942C6880EFC058DF4FCDBF9C
:10D1B000DEBFDF91CF911F910F91FF9008954F92A5
:10D1C0005F926F927F929F92AF92BF92CF92DF92C7
:10D1D000EF92FF920F931F93CF93DF938F3F09F04E
:10D1E00045C02CEA35EC47E257E3609193337091E8
:10D1F000943380919533909196330E94A8D7181656
:10D200000CF469C12CEA35EC47E257E360918B33AB
:10D2100070918C3380918D3390918E330E94A8D77A
:10D2200018160CF45DC12CEA35EC47E257E3609127
:10D230008F337091903380919133909192330E940B
:10D24000A8D718160CF455C12CEA35EC47E257E381
:10D2500060919733709198338091993390919A337C
:10D260000E94A8D718160CF43FC171C18230A1F5F5
:10D270002CEA35EC47E257E360918B3370918C33A5
:10D2800080918D3390918E330E94A8D718160CF49C
:10D2900027C12CEA35EC47E257E360918F33709158
:10D2A000903380919133909192330E94A8D71816B1
:10D2B0000CF41FC12CEA35EC47E257E36091973339
:10D2C000709198338091993390919A330E94A8D7A6
:10D2D00018160CF409C131C18823D9F2813051F3F9
:10D2E0002CC17E018DEEE80EF11CF7018081918149
:10D2F000A281B381BC01CD019F772CEA35EC47E2D6
:10D3000057E30E94A5D587FD46C06E01F1EFCF0E11
:10D31000D11CF601408051806280738020E030E0B3
:10D32000A901C301B2010E94A5D587FD34C0FE0149
:10D33000EF52FF4F208131814281538134976081C8
:10D340007181828193810E94FCD39B01AC015F7744
:10D35000C301B2010E94FDD32B013C019F772CEA4F
:10D3600035EC47E257E30E94A5D587FD14C0AB2CEE
:10D37000AA0C8A2D0E9436BC80938723992493940B
:10D380009A0C892D0E9436BC809388232091872394
:10D39000822780FD02C08B2DDBC0B0928623F8016E
:10D3A00080819181A281B381BF7780939A239093EA
:10D3B0009B23A0939C23B0939D23F701408151812F
:10D3C000628173817F7740939E2350939F23609364
:10D3D000A0237093A12320FF2DC0A09289239092B7
:10D3E0008A2377FA709477F870944092962350923B
:10D3F00097236092982370929923F60180819181FE
:10D40000A281B3818093A2239093A323A093A4230A
:10D41000B093A523CB50DF4F88819981AA81BB812E
:10D420008093A6239093A723A093A823B093A92326
:10D430008A2D2AC090928923A0928A234092962313
:10D44000509297236092982370929923F6018081DD
:10D450009181A281B381B0588093A2239093A3239A
:10D46000A093A423B093A523CB50DF4F888199814B
:10D47000AA81BB81B0588093A6239093A723A09341
:10D48000A823B093A923892D0E9436BC8D7F8130BB
:10D4900039F08FED98E6809390239093912369C0A3
:10D4A00080918A230E9436BC811103C08FEF809344
:10D4B0008A238B2D0E94CA586093B6237093B7239A
:10D4C0008093B8239093B92389E997E680939023BA
:10D4D000909391234EC082E090E032E0B32E0DC0D5
:10D4E00080E090E0B12C09C083E090E023E0B22E10
:10D4F00004C081E090E0BB24B394FC01E05DFD4CEE
:10D50000108225E3289FE001299FD00D1124C85DDA
:10D51000DF4C8E0107511F4FF80180819181A2815C
:10D52000B381BC01CD019F772CEA35EC47E257E38C
:10D530000E94A5D587FFD5CE2ECF81E080932F32D4
:10D540008CE298E6809390239093912312C08EEF03
:10D55000DF91CF911F910F91FF90EF90DF90CF90CF
:10D56000BF90AF909F907F906F905F904F900C9482
:10D570009D6882E0DF91CF911F910F91FF90EF9016
:10D58000DF90CF90BF90AF909F907F906F905F9013
:10D590004F900895CF93DF93C9E5D2E388819981B5
:10D5A0000E944E4A8093AE23888199810E94494A05
:10D5B0008093AF23888199810E94584A8093B02339
:10D5C000888199810E945D4A8093B12388819981E5
:10D5D0000E94644A6093B2237093B3238093B42370
:10D5E0009093B52381E00E94834E81E00E94874E94
:10D5F00080E00E943D4F81E00E94E85281E08093EC
:10D600008F238FEF809386238FED98E6809390236E
:10D610009093912383E080932C3210922F3280E0FC
:10D62000DF91CF9108950E94CA6A10928F2380E003
:10D63000089580912C32833059F40E94624A8130DF
:10D6400049F0E0919023F0919123809186231994E1
:10D6500083E0089582E0089584E39BE68093CB23E2
:10D660009093CC2382E008952F923F924F925F9245
:10D670006F927F928F929F92AF92BF92CF92DF92E2
:10D68000EF92FF920F931F93CF93DF93CDB7DEB747
:10D69000CA54D109CDBFDEBF98E19E01275E3F4F3E
:10D6A00029AB3AABD901E92F1D92EA95E9F7285148
:10D6B00031091901D9011D929A95E9F724E08202F6
:10D6C000F00111242B96EEAFFFAF2B97E20DF31D67
:10D6D00080E090E0A0E8BFE380839183A283B383DE
:10D6E000C090C323D090C423E090C523F090C623FC
:10D6F0004090BF235090C0236090C1237090C223FC
:10D700008090BB239090BC23A090BD23B090BE23FB
:10D71000A5019401C301B2010E94A5D518165CF0C1
:10D7200080E090E0A0E8BFE329968CAF9DAFAEAF5C
:10D73000BFAF29970AC080E090E0A0E8BFEB299630
:10D740008CAF9DAFAEAFBFAF2997A3019201C501CA
:10D75000B4010E94FCD30E9414D69B0177FF04C041
:10D7600022273327261B370BB901882777FD8095A1
:10D77000982F0E9447D625966CAF7DAF8EAF9FAF96
:10D780002597C0929832D0929932E0929A32F092D4
:10D790009B320E9498820E94325520E030E040E0A7
:10D7A00050E425966CAD7DAD8EAD9FAD25970E9462
:10D7B000A8D718166CF08091C7239091C823A09128
:10D7C000C923B091CA238BAF9CAFADAFBEAFDBC056
:10D7D0002AE037ED43E25CE325966CAD7DAD8EAD7E
:10D7E0009FAD25970E94A8D718162CF709E110E0E5
:10D7F0008AE0882E87ED982E83E2A82E8CE3B82E3F
:10D80000412C512C32012B96AEADBFAD2B97A20D02
:10D81000B31D58962196AEAFBFAF21974BAA5CAA15
:10D820006DAA7EAA8FAA98AEA9AEBAAE29962CADE3
:10D830003DAD4EAD5FAD29976FA978AD89AD9AAD7D
:10D840000E944AD89B01AC016091BF237091C02314
:10D850008091C1239091C2230E94FDD32196EEAD09
:10D86000FFAD21976083718382839383C092983246
:10D87000D0929932E0929A32F0929B32B101CE016D
:10D8800049960E94FC528093243D8111AAC020E059
:10D8900030E040E85FE36BA97CA98DA99EA90E94B6
:10D8A000FDD36BAB7CAB8DAB9EAB20E030E048ECA6
:10D8B00051E40E94ACD59B01AC0160E070E080E2D5
:10D8C00091E40E94ADD82B013C018091C723909137
:10D8D000C823A091C923B091CA238BAF9CAFADAF31
:10D8E000BEAFC090C323D090C423E090C523F09076
:10D8F000C623A7019601BC01CD010E94FCD34B01B8
:10D900005C0120E030E040E251E4C301B2010E943A
:10D91000ACD59B01AC01C501B4010E944AD89B0162
:10D92000AC01C701B6010E94FDD36B017C012BA99C
:10D930003CA94DA95EA9CA01B9010E94FDD320E00E
:10D9400030E048EC51E40E94ACD59B01AC016FA9DA
:10D9500078AD89AD9AAD0E94FDD36FAB78AF89AF3A
:10D960009AAF9B01AC0125966CAD7DAD8EAD9FADA0
:10D9700025970E94A8D7181634F4015011090115F3
:10D98000110509F053CF8BAD9CADADADBEAD80930D
:10D99000983290939932A0939A32B0939B322B96FF
:10D9A000EEADFFAD2B97E20DF31D8091BB2390915F
:10D9B000BC23A091BD23B091BE23808F918FA28FF5
:10D9C000B38FB101CE0149960E94FC528093243D51
:10D9D000811107C088E09DE68093CB239093CC23F0
:10D9E00082E0C65BDF4FCDBFDEBFDF91CF911F91DD
:10D9F0000F91FF90EF90DF90CF90BF90AF909F90EE
:10DA00008F907F906F905F904F903F902F900895F0
:10DA1000CF93DF931F92CDB7DEB789830E949882A0
:10DA20004091D5235091D6236091D7237091D8236C
:10DA300089810E94D5588091D2230E943D4F8091C8
:10DA4000D1230E94834E8091D3230E94874E8091E0
:10DA5000D4230E94E8528091CD239091CE23A091AF
:10DA6000CF23B091D0238093983290939932A09392
:10DA70009A32B0939B3264E08BE592E30E946B4A4A
:10DA80000E94DD5510922C3281EA91E20E941DE342
:10DA900080E00F90DF91CF9108950F931F93CF9364
:10DAA000C82F09E512E3F801808191810E944E4A56
:10DAB0008093D123F801808191810E94494A80930B
:10DAC000D223F801808191810E94584A8093D32308
:10DAD000F801808191810E945D4A8093D423F801EE
:10DAE000808191810E94644A6093CD237093CE23FC
:10DAF0008093CF239093D0238C2F0E94CA58609399
:10DB0000D5237093D6238093D7239093D82381E095
:10DB10000E94834E80E00E94874E80E00E943D4F2D
:10DB200081E00E94E85240E050E060E271E44093FE
:10DB3000C3235093C4236093C5237093C62385E306
:10DB4000C89FF0011124EF50FF4C40815181628148
:10DB500073814093C7235093C8236093C923709364
:10DB6000CA236C2F83E296E50E94604B6093BF232B
:10DB70007093C0238093C1239093C2230E94A25923
:10DB80006093BB237093BC238093BD239093BE23EB
:10DB9000C093BA238CE29BE68093CB239093CC2353
:10DBA00084E080932C3280E0CF911F910F910895F3
:10DBB00080912C32843059F40E94624A813049F0BD
:10DBC000E091CB23F091CC238091BA23199483E088
:10DBD000089582E00895E091DB23F0E0EB5FFF4CD5
:10DBE0008381882341F086E09EE68093D923909339
:10DBF000DA2382E0089568E274E280E194E20E9410
:10DC0000FC528093243D882371F308951F93CF9392
:10DC1000DF93E091DB23F0E0EB5FFF4C81E0938149
:10DC2000913009F080E080933632C7E3D2E310E010
:10DC3000812F0E948696AB01BC01812F0E94D44F98
:10DC4000612F8091593290915A320E94604B6993B2
:10DC50007993899399931F5F163051F78BEA91E27C
:10DC60000E94047A82E79EE68093D9239093DA2378
:10DC700082E0DF91CF911F9108951F93CF93DF939F
:10DC80000E9498828091DC2380930530E091DB2311
:10DC9000F0E08091DD23EB5FFF4C83870E9453BC53
:10DCA000C0EED3E210E04991599169917991812FA9
:10DCB0000E94D5581F5F1630B1F78091DF230E9474
:10DCC0003D4F8091DE230E94874E64E08BE592E316
:10DCD0000E946B4A0E94DD5510922C32DF91CF9149
:10DCE0001F9108950E943D6E80E008950F931F9349
:10DCF000CF93DF93CDB7DEB7C058D109CDBFDEBF1C
:10DD0000182F0E94E7601E3F29F488EB91E20E94E1
:10DD10003E6219C0812F0E9472561F928F9382EE2D
:10DD20009AE39F938F938E010F5F1F4F1F930F9363
:10DD30000E9473E3C8010E943E620F900F900F9003
:10DD40000F900F900F9042E062E08AEF0E944E62C7
:10DD50000E943D6E8AEFC058DF4FCDBFDEBFDF911E
:10DD6000CF911F910F910895FF920F931F93CF931F
:10DD7000DF931092363282E080932C3200EE13E271
:10DD8000C1E0D1E3F12C8F2D0E94CA58F8016193B4
:10DD90007193819391938F01488159816A817B812D
:10DDA0008F2D0E94D5586F2D8091593290915A3203
:10DDB0000E94604BF801648B758B868B978BF39474
:10DDC000E596F6E0FF12DFCF60E174E288EF93E2C0
:10DDD0000E942EC22AE43CE042E85EE30E94A5D500
:10DDE00087FF03C08EEF0E94766EC4E0D4E213E09A
:10DDF00069917991899199912C893D894E895F89A1
:10DE00000E94FCD39F772CEA35EC47E257E30E944F
:10DE1000A8D718161CF4812F0E94766E1F5F16304B
:10DE200039F784E08093DB23809114308093DD23E5
:10DE300081E080931430809105308093DC23109230
:10DE400005300E9453BC8091593290915A320E9401
:10DE5000494A8093DF238091593290915A320E942F
:10DE6000584A8093DE2380E00E94874E80E00E9423
:10DE70003D4F80E00E94AFAE8BEE9DE68093D923AC
:10DE80009093DA2382E0DF91CF911F910F91FF9061
:10DE900008950F931F93CF93DF938C01EB01809133
:10DEA000A432882399F08091983290919932A09170
:10DEB0009A32B0919B32BC01CD019F772CEA35ECB0
:10DEC00047E257E30E94A5D587FD4FC0888199811D
:10DED000AA81BB81BC01CD019F772CEA35EC47E2DA
:10DEE00057E30E94A8D71816F4F48C819D81AE8167
:10DEF000BF81BC01CD019F772CEA35EC47E257E3A7
:10DF00000E94A8D718167CF488859985AA85BB85B8
:10DF1000BC01CD019F772CEA35EC47E257E30E9424
:10DF2000A8D7181624F188E1F801A0E1B4E2019025
:10DF30000D928A95E1F788E1FE01A8E2B4E2019032
:10DF40000D928A95E1F788E1E7E3F2E3DF011D92A4
:10DF50008A95E9F782E08093363284EB9EE68093DF
:10DF6000D9239093DA2380E003C08EE801C086E8CD
:10DF7000DF91CF911F910F91089580912C328230C3
:10DF800021F080913632823049F40E94624A813019
:10DF900039F0E091D923F091DA23199483E00895C0
:10DFA00082E00895ECE9FCE380E2DF011D928A95AE
:10DFB000E9F78FEE92E18093BA3C9093BB3C80836B
:10DFC000918308958091BA3C9091BB3C8F3E9241E1
:10DFD00011F08CE5089580919C3C90919D3C8F3E82
:10DFE0009241B9F780E00895CF93DF93C82FCB011A
:10DFF000BA010E94F9D827E0C29FE0011124C4565B
:10E00000D34C0E9414D66D837E838F839887DF91D3
:10E01000CF91089597E0899FF0011124E456F34CC5
:10E0200065817681878190850E9447D608952F92D9
:10E030003F924F925F926F927F928F929F92AF9298
:10E04000BF92CF92DF92EF92FF920F931F93CF93E5
:10E05000DF93CDB7DEB72797CDBFDEBF8C011B8224
:10E0600080912B32823009F40EC7D801BC90B110D8
:10E0700037C780E06E01B3E0CB0ED11C3DC0F60186
:10E080008081811108C0B72CD7011C926E01B3E0CA
:10E09000CB0ED11C22C7883239F4B72CF70110827D
:10E0A000FFEFCF1ADF0A19C78B33B9F3A82EB12CB3
:10E0B000C5010E946DE1892B39F4B50182EE91E230
:10E0C0000E94E6E1892B51F047018FEF881A980AE8
:10E0D000C5010E9491E1D7018C937401BFEFCB1A67
:10E0E000DB0AF70180818111CACFB72CD8018C914E
:10E0F0006E01B3E0CB0ED11CF8011CC08E32E1F0F2
:10E1000090E0C0970A9790F08181803391F48281EA
:10E1100090E0C0970A9760F4DF01119611968C91F8
:10E1200011978D938111FACF808104C0818101C044
:10E1300080E331968111E2CFF601A080A11007C0E3
:10E1400036C0D6011196AC90BFEFCB1ADB0A760130
:10E150008A2C912CC4010E9481E1892B91F7C40182
:10E160000E9489E18D369105A1F4F601818190E04C
:10E170000E9489E18337910561F4D60112968C9152
:10E1800090E00E9489E18736910519F4F6013396F3
:10E1900002C0FE013396AA2061F08A2DD701893290
:10E1A00009F41C9211968C918111F9CF02C0FE01E5
:10E1B0003396BFE2BB1609F468C68081882319F044
:10E1C000CF010E94255580E1ECEBFCE3DF011D92BD
:10E1D0008A95E9F78BE5E4E8F3E3DF01982F1D92D8
:10E1E0009A95E9F7E9E2F3E3DF011D928A95E9F7F1
:10E1F0008BE592E30E94464A80932A33812C912C2E
:10E2000080E8A82E8FE3B82E5524539492E0492E2F
:10E2100024E0322E23C4C701B6010E9419D6862FEE
:10E2200090E08F35910508F034C6FC01EC50FF4FAB
:10E230000C94F0DD10922A33509285338091BD3CCE
:10E240008F5F8093BD3C0AC450922A33509285332D
:10E250008091BD3C8F5F8093BD3C00C440922A33C7
:10E26000509285338091BD3C8F5F8093BD3CF6C357
:10E2700083E080932A33509285338091BD3C8F5F39
:10E280008093BD3CEBC38DE080932933509284335F
:10E29000E5C388E0B2C0109259335092B4338091F4
:10E2A000BE3C8F5F8093BE3CD9C35092593350928D
:10E2B000B4338091BE3C8F5F8093BE3CCFC340920D
:10E2C00059335092B4338091BE3C8F5F8093BE3CF3
:10E2D000C5C310925A335092B5338091C13C8F5FC1
:10E2E0008093C13CBBC350925A335092B533809156
:10E2F000C13C8F5F8093C13CB1C3C701B6010E948E
:10E3000064D96C837D838E839F8320E030E040E27C
:10E3100051E4C701B6010E944AD86B017C0120E09C
:10E3200030E040E251E46C817D818E819F810E94CA
:10E330004AD89B01AC01C701B6010E94FCD30E94E0
:10E3400019D6623001F128F4662341F0613089F07A
:10E35000A0C56330E9F0643001F19BC5B5E0B0932E
:10E360002933509284338091BC3C8F5F8093BC3CB6
:10E3700075C330922933609384338091BC3C8F5FA6
:10E380008093BC3C6BC3509229335092843366C354
:10E39000409229335092843361C383E080932933C0
:10E3A000509284335BC3C701B6010E9464D96C8369
:10E3B0007D838E839F8320E030E040E251E4C701FB
:10E3C000B6010E944AD86B017C0120E030E040E2B7
:10E3D00051E46C817D818E819F810E944AD89B018E
:10E3E000AC01C701B6010E94FCD30E9419D6662376
:10E3F00019F0613061F04DC587E080932933509268
:10E4000084338091BC3C8F5F8093BC3C27C3E6E0A3
:10E41000E0932933609384338091BC3C8F5F809379
:10E42000BC3C1CC3C701B6010E9464D96C837D83C8
:10E430008E839F8320E030E040E251E4C701B601C3
:10E440000E944AD86B017C0120E030E040E251E4B8
:10E450006C817D818E819F810E944AD89B01AC0195
:10E46000C701B6010E94FCD30E9419D6623009F0A0
:10E4700010C58EE08093293350928433EFC25092BE
:10E480005C335092B733EAC250925B335092B6334A
:10E490008091C53C8F5F8093C53CE0C240925B3366
:10E4A0005092B6338091C53C8F5F8093C53CD6C2F5
:10E4B00083E016C030925B335092B6338091C53CF6
:10E4C0008F5F8093C53CCAC2F5E0F0935B335092F6
:10E4D000B6338091C53C8F5F8093C53CBFC286E058
:10E4E00080935B335092B6338091C53C8F5F8093AD
:10E4F000C53CB4C2C701B6010E9464D96C837D8358
:10E500008E839F8320E030E040E251E4C701B601F2
:10E510000E944AD86B017C0120E030E040E251E4E7
:10E520006C817D818E819F810E944AD89B01AC01C4
:10E53000C701B6010E94FCD30E9419D6662319F0C8
:10E54000613059F0A6C410925E335092B933809175
:10E55000C63C8F5F8093C63C81C260935E336093FC
:10E56000B9338091C63C8F5F8093C63C77C240929E
:10E570005E335092B9338091C63C8F5F8093C63C26
:10E580006DC230922A33509285338091BD3C8F5FAB
:10E590008093BD3C63C2C701B6010E9464D96C83FD
:10E5A0007D838E839F8320E030E040E251E4C70109
:10E5B000B6010E944AD86B017C0120E030E040E2C5
:10E5C00051E46C817D818E819F810E944AD89B019C
:10E5D000AC01C701B6010E94FCD30E9419D6662384
:10E5E00019F0613059F055C410925F335092BA332C
:10E5F0008091BF3C8F5F8093BF3C30C210926033EC
:10E600006093BB338091BF3C8F5F8093BF3C26C239
:10E61000C701B6010E9464D96C837D838E839F837A
:10E6200020E030E040E251E4C701B6010E944AD840
:10E630006B017C0120E030E040E251E46C817D819F
:10E640008E819F810E944AD89B01AC01C701B6010F
:10E650000E94FCD30E9419D6662319F0613059F04C
:10E6600018C450925F335092BA338091BF3C8F5F91
:10E670008093BF3CF3C1609360336093BB33809160
:10E68000BF3C8F5F8093BF3CE9C1C701B6010E94C8
:10E6900064D96C837D838E839F8320E030E040E2E9
:10E6A00051E4C701B6010E944AD86B017C0120E009
:10E6B00030E040E251E46C817D818E819F810E9437
:10E6C0004AD89B01AC01C701B6010E94FCD30E944D
:10E6D00019D6613089F028F06230A1F06330C1F0C2
:10E6E000D8C399E090932933509284338091BC3CF5
:10E6F0008F5F8093BC3CB2C1AAE0A09329336093A2
:10E700008433ACC1BBE0B093293350928433A6C1AB
:10E71000ECE0E093293350928433A0C1109254333B
:10E720005092AF338091C03C8F5F8093C03C96C1C4
:10E73000509254335092AF338091C03C8F5F80939E
:10E74000C03C8CC1C701B6010E9419D6862F90E04B
:10E750008D33910508F09BC3FC01ED5AFE4F0C94DC
:10E76000F0DD10922B33509286338091C73C8F5F3F
:10E770008093C73C73C150922B3350928633809163
:10E78000C73C8F5F8093C73C69C1509266335092FB
:10E79000C1338091C93C8F5F8093C93C5FC1409277
:10E7A00066335092C1338091C93C8F5F8093C93CDE
:10E7B00055C1109266335092C1338091C93C8F5F2E
:10E7C0008093C93C4BC1509263335092BE3346C1D3
:10E7D000509264335092BF338091CA3C8F5F8093D4
:10E7E000CA3C3CC1509265335092C0338091CA3CC0
:10E7F0008F5F8093CA3C32C1109265335092C03310
:10E800008091CA3C8F5F8093CA3C28C15092573395
:10E810005092B2338091CB3C8F5F8093CB3C1EC132
:10E82000109257335092B2338091CB3C8F5F8093DC
:10E83000CB3C14C1509255335092B0338091CB3CB5
:10E840008F5F8093CB3C0AC150926F335092CA3392
:10E850008091CB3C8F5F8093CB3C00C1C701B60158
:10E860000E9464D90E9419D6609362335092BD33DE
:10E87000F5C0C0924833D0924933E0924A33F092C7
:10E880004B338092A3339092A433A092A533B092DD
:10E89000A633E4C0C0927033D0927133E0927233E9
:10E8A000F09273338092CB339092CC33A092CD33DD
:10E8B000B092CE33D3C0C0926733D0926833E09227
:10E8C0006933F0926A338092C2339092C333A0923C
:10E8D000C433B092C533C2C0C0923033D09231330A
:10E8E000E0923233F092333380928B3390928C33B8
:10E8F000A0928D33B0928E33B1C0C0923433D09297
:10E900003533E0923633F092373380928F339092E2
:10E910009033A0929133B0929233A0C0C09238331A
:10E92000D0923933E0923A33F0923B338092933372
:10E9300090929433A0929533B09296338FC0C09248
:10E940003C33D0923D33E0923E33F0923F3380929D
:10E95000973390929833A0929933B0929A337EC0B5
:10E96000C0924033D0924133E0924233F09243332D
:10E9700080929B3390929C33A0929D33B0929E33B1
:10E980006DC0C0924433D0924533E0924633F0924A
:10E99000473380929F339092A033A092A133B092DC
:10E9A000A2335CC0C0927833D0927933E0927A334C
:10E9B000F0927B338092D3339092D433A092D533AC
:10E9C000B092D6334BC0C0927C33D0927D33E0926C
:10E9D0007E33F0927F338092D7339092D833A092D7
:10E9E000D933B092DA333AC0C0928033D0928133B7
:10E9F000E0928233F09283338092DB339092DC3367
:10EA0000A092DD33B092DE3329C0C0927433D0922D
:10EA10007533E0927633F09277338092CF339092D1
:10EA2000D033A092D133B092D23318C0C701B6010F
:10EA30000E9419D660932C3370932D3380932E331C
:10EA400090932F3381E090E0A0E0B0E08093873393
:10EA500090938833A0938933B0938A33D8012C9054
:10EA6000222009F424C2822D90E00E9478E1892BB3
:10EA700009F42FC23801BFEF6B1A7B0AF8018181BC
:10EA8000803349F48281883531F40E5F1F4FC12CE9
:10EA9000D12C760100C2BE016F5F7F4FC3010E947F
:10EAA00010DE6B017C0109811A816016710609F084
:10EAB000F2C111C2809154330E94E852182F01C054
:10EAC00010E06091A3337091A4338091A5339091AD
:10EAD000A6330E9419D6662359F06091483370918D
:10EAE000493380914A3390914B330E94B752182F8B
:10EAF0006091A7337091A8338091A9339091AA3384
:10EB00000E9419D6662371F060914C3370914D3399
:10EB100080914E3390914F330E9419D6862F0E94D8
:10EB20009354182F6091AB337091AC338091AD3317
:10EB30009091AE330E9419D6662371F060915033E4
:10EB40007091513380915233909153330E9419D672
:10EB5000862F0E94D254182F6091C2337091C33314
:10EB60008091C4339091C5330E9419D6662359F021
:10EB700060916733709168338091693390916A3303
:10EB80000E94E3AE182F6091C6337091C733809115
:10EB9000C8339091C9330E9419D6662371F06091F1
:10EBA0006B3370916C3380916D3390916E330E9412
:10EBB00019D6862F0E941155182F8091BD338823B6
:10EBC00029F0809162330E945053182F8091BE33F8
:10EBD000882329F0809163330E948453182F8091F9
:10EBE000C133882329F0809166330E94AFAE182F7D
:10EBF0008091BF33882329F0809164330E94B953F8
:10EC0000182F8091C033882329F0809165330E94AA
:10EC1000ED53182F8091B033882329F0809155331C
:10EC20000E946854182F8091B133882329F0809175
:10EC300056330E94A754182F8091CA33882329F095
:10EC400080916F330E94E654182F8091B23388234D
:10EC500029F0809157330E946054182F80912933F6
:10EC60008D3029F08091B4338823A9F00FC06091D2
:10EC700070337091713380917233909173330E942D
:10EC8000F0528093243D882369F32FC1809159333A
:10EC90000E947F4E182F8091B533882329F08091F0
:10ECA0005A330E94834E182F8091B633882329F05F
:10ECB00080915B330E943D4F182F8091B933882398
:10ECC00029F080915E330E94EC52182F8091BA3364
:10ECD000882329F080915F330E94874E182F40913E
:10ECE000293350E04F30510508F0B6C0FA01E05723
:10ECF000FE4F0C94F0DD0E943952182FADC06BE826
:10ED000073E380E393E30E944452182FA5C00E944E
:10ED10007852182FA1C06BE873E380E393E30E945D
:10ED20008352182F99C00E94CA6A182F95C06BE8A9
:10ED300073E380E393E30E940350182F8DC00E9479
:10ED4000136B182F89C06BE873E380E393E30E9491
:10ED5000496F182F81C06091703370917133809129
:10ED60007233909173330E9419D6862F2BE833E3C8
:10ED700040E353E3609158330E948B4E182F6CC0D0
:10ED80006BE873E380E393E30E948050182F64C024
:10ED90000E943351182F60C00E949A51182F5CC0F6
:10EDA0000E94D151182F58C060915C338BE592E3DB
:10EDB0000E94E14A80912A33843038F48230D8F4BA
:10EDC000882349F0813079F047C0843009F044C08D
:10EDD00080935F3241C06BE873E380E393E30E946A
:10EDE0000952182F39C06BE873E380E393E30E9464
:10EDF000FC52182F31C0A0908033B0908133C09066
:10EE00008233D0908333E0907C33F0907D33009157
:10EE10007E3310917F332091783330917933409154
:10EE20007A3350917B338F93809177338F93809196
:10EE300076338F93809175338F93809174338F9352
:10EE40006BE873E380E393E30E942884182F0F900C
:10EE50000F900F900F900F9060E08BE592E30E946F
:10EE6000E14A80918633813061F480912B338111A6
:10EE700004C00E941056812F38C00E944156812F35
:10EE800034C0812F32C08BEC30C083E02EC084E8C8
:10EE90002CC083E82AC0822D90E0FC01E154F109E6
:10EEA000EA31F105B0F7E156FE4F0C94F0DD109217
:10EEB000243D60912C3370912D3380912E339091AD
:10EEC0002F330E947B4A8091AF33882309F4F8CD19
:10EED000F1CD85E60AC086E608C0D8018C910CC940
:10EEE00068018B2D78017B2CD6C82796CDBFDEBF5D
:10EEF000DF91CF911F910F91FF90EF90DF90CF9016
:10EF0000BF90AF909F908F907F906F905F904F9049
:10EF10003F902F900895CF93DF93EC016AE17CE35B
:10EF20000E94A7618093243D811102C095E09F83D8
:10EF3000DF91CF910895FC018789908D0C94177013
:10EF400083FF06C0E091FD2FF091FE2F90E29583A4
:10EF500082FF06C0E091FF2FF091003090E2958390
:10EF600081FF06C0E0910130F091023090E295837C
:10EF700080FF06C0E0910330F091043080E2858389
:10EF8000089583FF06C0E091FD2FF091FE2F90E2DF
:10EF9000968382FF06C0E091FF2FF091003090E24F
:10EFA000968381FF06C0E0910130F091023090E23B
:10EFB000968380FF06C0E0910330F091043080E238
:10EFC000868308958091FA39811107C084E00E94F8
:10EFD000A07781E08093FA39089584E00E94C17798
:10EFE0001092FA390895CF92DF92EF92FF920F9329
:10EFF0001F93CF93DF93C12C26E0D22EC092ED2F2A
:10F00000D092EE2F30EAE32E36E0F32EE092EF2F8F
:10F01000F092F02F00E816E00093F12F1093F22FFA
:10F02000C0E6D6E0C093F32FD093F42FC092F52F13
:10F03000D092F62FC093F72FD093F82F0093F92F8B
:10F040001093FA2FE092FB2FF092FC2F2DEC3CEC6A
:10F050004CED50E40E94A8D7C092FD2FD092FE2F15
:10F06000E092FF2FF092003018164CF4C09301305C
:10F07000D0930230009303301093043008C0009303
:10F08000013010930230C0930330D0930430DF91ED
:10F09000CF911F910F91FF90EF90DF90CF90089547
:10F0A0000E944FD360E070E080E091E40E94F3772B
:10F0B0000C946ED381E08093033A089520E093E0AE
:10F0C00088ED08B618BE84BF90938000209182001E
:10F0D00021FDFCCF08BEFFCF8091033A81110E9431
:10F0E0005E7883E008958091043A882341F0F89493
:10F0F00061E089E790E00E9451D382E0089583E0C7
:10F100000895CF93DF93CDB7DEB7AD97CDBFDEBF08
:10F1100021E2E5EEF1E2DE01119601900D922A95D1
:10F12000E1F722E02093CA01DE019296E8E0F0E0E8
:10F1300024912D933196EE30F105D1F72DE228A7D9
:10F14000E0E1F0E0E491EF7121E030E02C0F3D1FB1
:10F150002E0F311DF901208129A7E2E1F0E0E491B1
:10F16000EF719E012E0F311DF90121812AA7E4E1E3
:10F17000F0E0E491EF719E012E0F311DF901218124
:10F180002BA71CA61092CA0125E0FC012783BE0113
:10F190006E5D7F4F0E94A7618093243DAD96CDBFE9
:10F1A000DEBFDF91CF91089581E08093043A80E043
:10F1B0000895CF93DF93EC0120E030E040E051E48C
:10F1C00069857A858B859C850E94A8D718166CF076
:10F1D000CE010E94D05E69857A858B859C850E94D0
:10F1E000F3770E9453BC80E001C08DE6DF91CF91A0
:10F1F000089564E87BE30C94DEC166E67BE30C943F
:10F20000DEC167E47BE30C94DEC169E27BE30C942E
:10F21000DEC165E17BE30C9489C1CF93DF938AEC77
:10F2200096E49F938F93CCEDD9E589818F93888164
:10F230008F930E947FE284E994E49F938F93898166
:10F240008F9388818F930E947FE28CE094E49F9358
:10F250008F9389818F9388818F930E947FE282E4CC
:10F2600093E49F938F9389818F9388818F930E94DA
:10F270007FE20E9415A88DB79EB740968DBF9EBFB6
:10F2800080E0DF91CF910895CF93DF938DE193E4F8
:10F290009F938F93CCEDD9E589818F9388818F934C
:10F2A0000E947FE28FEA91E49F938F9389818F93ED
:10F2B00088818F930E947FE284E290E49F938F93F2
:10F2C00089818F9388818F930E947FE28CE094E400
:10F2D0009F938F9389818F9388818F930E947FE280
:10F2E00082E493E49F938F9389818F9388818F9396
:10F2F0000E947FE28DB79EB744968DBF9EBF80E08F
:10F30000DF91CF910895CF93DF9383E090E49F93B3
:10F310008F93CCEDD9E589818F9388818F930E945B
:10F320007FE285E89CE39F938F9389818F93888107
:10F330008F930E947FE282E493E49F938F9389816D
:10F340008F9388818F930E947FE28DB79EB70C9632
:10F350008DBF9EBF80E0DF91CF910895CF93DF9363
:10F360008DE59CE39F938F93CCEDD9E589818F93B5
:10F3700088818F930E947FE28CEE9BE39F938F9313
:10F3800089818F9388818F930E947FE282E493E446
:10F390009F938F9389818F9388818F930E947FE2BF
:10F3A0008DB79EB70C968DBF9EBF80E0DF91CF9149
:10F3B0000895CF93DF9389EC9BE39F938F93CCEDDC
:10F3C000D9E589818F9388818F930E947FE280EABB
:10F3D0009BE39F938F9389818F9388818F930E9462
:10F3E0007FE282E493E49F938F9389818F93888156
:10F3F0008F930E947FE28DB79EB70C968DBF9EBF04
:10F4000080E0DF91CF9108952F923F924F925F92CB
:10F410006F927F928F929F92AF92BF92CF92DF9224
:10F42000EF92FF920F931F93CF93DF93CDB7DEB789
:10F430006A97CDBFDEBF5C010E94E7602C011F868A
:10F44000188A198A1A8AF50101900020E9F7319784
:10F45000EA19FB09E130F24008F002C2D5018C91B3
:10F46000882359F17501BFEFEB1AFB0A850120E0F3
:10F47000211115C0883229F08132C8F08F37B9F0D8
:10F4800001C021E06801EFEFCE1ADE0A90E02A8F7A
:10F490000E9489E1D8018C9386012A8D08C021E061
:10F4A000893209F420E0F80180830F5F1F4FD701F4
:10F4B0008D917D018111DCCF01C08501F8011082A1
:10F4C0001092243DFDE19F2EAAE36A2EA2E27A2E3D
:10F4D000812CB6E02B2E03C09A9409F49CC18BE7D3
:10F4E0009CE2A2E2B0E08B879C87AD87BE876B8AE7
:10F4F0007C8A8D8A8DE79CE2A2E2B0E08F839887B8
:10F50000A987BA87E6E0F2E2DE011196822D01902A
:10F510000D928A95E1F7C2010E94EE5F8501075FB7
:10F520001F4F75019FEFA91AB90AD7016C9170E0BE
:10F53000CE010B960E94E6E1892B21F487010E5D36
:10F540001F4F04C0A016B10661F793C16501BFEF5C
:10F55000AB1ABB0AF601608170E0CE0143960E94AF
:10F56000E6E1892B91F0D6011D928D0192012F5E6B
:10F570003F4F288F398F46E050E0B701C9010E9404
:10F5800011E23AE0C30ED11C04C0A016B106F1F698
:10F5900070C15801D8013D908D01E32CF12CC701B9
:10F5A0000E946DE1892B59F4B701CE0101960E94AA
:10F5B000E6E1892B21F40C151D0559F75AC1850187
:10F5C000BEE63B1641F0E2E23E120CC0D5011196B8
:10F5D0008C918232A9F5F201178211861286138668
:10F5E0001486A3C0B0E3EB1AF108EAE0EE16F104CA
:10F5F00018F0FDE23F1217C0BE016A5E7F4FC501E1
:10F600000E9410DED20119966D937D938D939C9389
:10F610001C978E899F898A159B0509F42DC1E4E00A
:10F620001796EC9382C0FBE73F124FC0E7E0D20190
:10F630001796EC93FFEFAF1ABF0AE2E0FE2E95C0DB
:10F640002FEFA21AB20AE5E0D2011796EC9362E21C
:10F6500070E0C5010E94E6E18E8B9F8B009709F454
:10F6600008C1DC011C92F50101900020E9F73197F7
:10F67000EA19FB093397C8F0F80181818033A9F4B6
:10F680008281883791F440E050E060E070E0C5018D
:10F690000E9481DFD20119966D937D938D939C9387
:10F6A0001C9783E017968C9308C0B501C2010E9495
:10F6B000A7618093243D811153C0AE88BF88BFEFFE
:10F6C000AB1ABB0AAE8ABF8A30C0E4E73E120EC056
:10F6D000E1E0D2011796EC9380E090E0A0E8BFE370
:10F6E000F20181879287A387B4871FC0F6E63F1295
:10F6F0000CC0E1E0D2011796EC93179719961D9272
:10F700001D921D921C921C9710C0BBE53B12B1C00C
:10F71000F2012782B501C2010E94A7618093243DB6
:10F7200081111EC077E6F72E7DC0BE01695F7F4F55
:10F73000C5010E942BE25C01009709F49AC0DC012C
:10F740008C918D3729F411968C91F50131965F01DA
:10F750008C3209F48BC0FFEFAF1ABF0AF12C05C041
:10F76000F82E22E0281708F45DC08F858201035F20
:10F770001F4F882341F043E050E0BE01615F7F4F9F
:10F78000C8010E9411E2688D798DC8010E94475F0F
:10F79000D20114968D939C9315978F3FBFEF9B07D3
:10F7A000B9F10E947E64882371F0888D998D0E9442
:10F7B000305F882341F043E050E0688D798DCE01C1
:10F7C0000F960E9411E2F2014280538041145104CD
:10F7D00011F1F11081CE80918E34811108C087E83B
:10F7E00094E30E94E35B8093243DF82E1BC080913C
:10F7F0002B32823099F087E894E30E94B95B8093C2
:10F80000243D81110EC087E894E30E94365C0AC053
:10F8100064E6F62E07C050E7F52E04C04BECF42E3C
:10F8200001C0F82E42E060E08F2D0E944E6281E020
:10F830000E9474AA6A96CDBFDEBFDF91CF911F915F
:10F840000F91FF90EF90DF90CF90BF90AF909F907F
:10F850008F907F906F905F904F903F902F90089582
:10F860008BE68093243D3BE6F32EDCCF22E0F22EA4
:10F870007CCF9FE6F92ED6CF86E6F82ED3CF2F92F7
:10F880003F924F925F926F927F928F929F92AF9230
:10F89000BF92CF92DF92EF92FF920F931F93CF937D
:10F8A000DF9300D000D0CDB7DEB78C0169837A83B7
:10F8B0004B835C835A0128E0A21AB108A60EB71E3A
:10F8C000DC0116967C907B01BFEFEB1AFB0A8BE7FD
:10F8D000FB01808380E0912C95E0692E20E1422E8F
:10F8E00022E2522E3CE0232E32E2332E4DE7842ECC
:10F8F000ED82FE82D80117969C919F3F09F429C1A1
:10F90000882339F02CE2ED81FE8120833196ED834E
:10F91000FE838091CE3C811119C0C80141969F930E
:10F920008F933F922F923E813F938D818F930E94C0
:10F930004AE3AD81BE81A80FB91FAD83BE830F908E
:10F940000F900F900F900F900F9018C0C801419624
:10F950009F938F935F924F92BE81BF93ED81EF9300
:10F960000E944AE32D813E81280F391F2D833E835B
:10F970000F900F900F900F900F900F90D801179647
:10F980008C911797843059F51996CD90DD90ED90B4
:10F99000FC901C97A7019601C701B6010E946BD984
:10F9A000811117C0E894F7F82FEF3FEF4FE75FE7BB
:10F9B000C701B6010E946BD9811121C12FEF3FEF22
:10F9C0004FE75FE7C701B6010E94A5D518160CF0F6
:10F9D00016C1F801118612861386148610C1811192
:10F9E00013C0E6E1F2E2AD81BE81862D01900D9259
:10F9F0008A95E1F72D813E812C5F3F4F2D833E8319
:10FA0000D80117968C9199C0823061F4F8018485F1
:10FA10008F9383858F9382858F9381858F93ABE1BD
:10FA2000B2E214C0833029F5D8011C968C911C9742
:10FA30008F931B968C911B978F931A968C911A9784
:10FA40008F9319968C918F93A1E2B2E2BF93AF93FB
:10FA5000FE81FF932D812F930E944AE3AD81BE81E9
:10FA6000A80FB11DAD83BE83F8018781CDBFDEBF76
:10FA700064C0853059F4D80158968C9158978F936B
:10FA800057968C918F93A9E2B2E20CC0863009F5AB
:10FA9000D80158968C9158978F9357968C918F9345
:10FAA000AEE2B2E2BF93AF93FE81FF932D812F931D
:10FAB0000E944AE3AD81BE81A80FB11DAD83BE8314
:10FAC000F80187810F900F900F900F900F900F907B
:10FAD00034C0813091F52CEA35EC47E257E3D80188
:10FAE00019966D917D918D919C911C970E94A5D541
:10FAF00087FF12C0E3E3F2E2AD81BE8186E00190B0
:10FB00000D928A95E1F7ED81FE813596ED83FE83B6
:10FB1000D80117968C9111C0E9E3F2E2AD81BE8164
:10FB2000862D01900D928A95E1F7ED81FE81349644
:10FB3000ED83FE83D80117968C91873049F42BE72B
:10FB4000ED81FE8120833196ED83FE8380E001C04C
:10FB500081E0AD81BE81AA15BB0518F08FEF9FEF44
:10FB600065C0F801028113810115110549F0D80122
:10FB700016969C912FEF290D99153CF0992EBACE2F
:10FB8000ED80FE807914B4F020C0ED81FE81D801B3
:10FB9000CF010196808216969C9016973FEF320F08
:10FBA00092161CF4232FFC01F3CF8D839E838D01CD
:10FBB00081E0A0CEF7012DE7CF01019620839A9432
:10FBC000791414F4FC01F8CF7C018DE79AE0A0E0F1
:10FBD000F70180839183A283F2E0EF0EF11C89810B
:10FBE0009A812B813C81820F931F8E159F0508F40B
:10FBF000B5CFC701A981BA818A1B9B0B17C0C80169
:10FC00000E948E64F8014185528563857485208544
:10FC10008D819E810E9422C42D813E81280F311D3D
:10FC20002D833E83D80117968C9187CF2696CDBF22
:10FC3000DEBFDF91CF911F910F91FF90EF90DF908A
:10FC4000CF90BF90AF909F908F907F906F905F907C
:10FC50004F903F902F90089540E052E06AE17AE3A0
:10FC60000E943F7C6091DC597091DD598AE19AE3F2
:10FC70000C94CEE2EF92FF920F931F93CF93DF93FA
:10FC8000CDB7DEB76297CDBFDEBFF82E9091CC3CEA
:10FC9000992309F4B2C08FE6F81212C00E94E760FF
:10FCA0006AE17CE38091163A9091173A0E9402C46F
:10FCB000BC018CE091E20E94056207E814E34AC0AF
:10FCC00080912B3207E814E3882309F443C0EE2423
:10FCD000EA94C8010E94AE5F8823E1F1823029F4E2
:10FCE0008091D33C811120C01DC0843029F48091C3
:10FCF000D03C811119C016C08530B1F48091D23C3E
:10FD0000882381F0F80181859285A385B485BC01A3
:10FD1000CD019F772CEA35EC47E257E30E94A5D549
:10FD200087FF02C0F801E782F80102811381011503
:10FD3000110579F60FC0F801028113810115110533
:10FD400049F440E052E06AE17AE38EE694E30E94EF
:10FD50003F7C53C0F80197819F3F69F78091E52F61
:10FD600081111AC08091193A8F938091183A8F931C
:10FD70001F92FF928EE392E29F938F93CE010196A2
:10FD80007C01FF928F930E944AE31092183A1092DE
:10FD9000193ACDBFDEBF13C00E9449C91F928F938D
:10FDA0001F92FF9286E492E29F938F93CE01019679
:10FDB0007C01FF928F930E944AE3CDBFDEBFB70163
:10FDC000C8010E94A761F801168286E0878386E653
:10FDD00090E0818B928B1282138240E052E06AE1C4
:10FDE0007AE38EE694E30E943F7C6091DC59709147
:10FDF000DD598AE19AE30E94CEE26296CDBFDEBF72
:10FE0000DF91CF911F910F91FF90EF900895613096
:10FE100019F0623029F0089587E894E30C942C7E61
:10FE20000C943A7ECF92DF92EF92FF92FC01C18454
:10FE3000D284E384F48420E030E040EA50E4C70157
:10FE4000B6010E94A8D718160CF453C0C701B6011A
:10FE50000E9419D66093CC3C1092CF3C1092D03CBB
:10FE60001092D13C1092D23C1092D33C20E030E072
:10FE700040E85FE3C701B6010E94A8D787FD03C031
:10FE800081E08093CF3C20E030E040E050E4C701C7
:10FE9000B6010E94A8D787FD03C081E08093D03CC3
:10FEA00020E030E040E450E4C701B6010E94A8D74A
:10FEB00087FD03C081E08093D13C20E030E040E842
:10FEC00050E4C701B6010E94A8D787FD03C081E0B6
:10FED0008093D23C20E030E040EA50E4C701B60114
:10FEE0000E94A8D787FD07C081E08093D33C80E0C3
:10FEF00003C08EE601C080E0FF90EF90DF90CF90CE
:10FF000008956CE677E40C949FC165E177E40C9466
:10FF10009FC161EE76E40C949FC1BF92CF92DF92B5
:10FF2000EF92FF920F931F93CF93DF93CDB7DEB77E
:10FF30006897CDBFDEBF6B0128E1FC01DE011196A1
:10FF400001900D922A95E1F78CEEE82E80E3F82ED1
:10FF50008E010F5F1F4FB12CF7018081823029F491
:10FF6000F801108211821282138280915E588B11E7
:10FF700014C020917158309172584091735850912B
:10FF80007458F80160817181828193810E944AD8FE
:10FF9000F601608371838283938380917D588B11F6
:10FFA00014C020919058309191584091925850919E
:10FFB0009358F80160817181828193810E944AD8AF
:10FFC000F601648375838683978380919C588B1197
:10FFD00014C02091AF583091B0584091B158509111
:10FFE000B258F80160817181828193810E944AD860
:10FFF000F60160877187828793878091BB588B1148
:020000021000EC
:1000000014C02091CE583091CF584091D058509183
:10001000D158F80160817181828193810E944AD810
:10002000F6016487758786879787B394F5E3EF0EAB
:10003000F11C0C5F1F4F86E0B8128ECF6896CDBFC3
:10004000DEBFDF91CF911F910F91FF90EF90DF9076
:10005000CF90BF900895F8940E9450780E948280BB
:100060000E946ED30E94D0C50E940EB30E94D26F30
:100070000E9453BC0E946AA540E060E080E00E94BC
:1000800084650E9424610E9470800E9474820E9494
:10009000734F0E9466D38091A20084608093A20077
:1000A0008091A20082608093A2008091A200816072
:1000B0008093A20078940E9415A80E9460BD0E94BF
:1000C000EB65FDCFE82FF0E0EE0FFF1FE856F84B91
:1000D000659174914FE450E084ED9CE30C94B8E199
:1000E0008091F739823041F440E060E081E00E9485
:1000F000846580E00E9413670C9442CA682F81E0F7
:100100000C94EBC61092253D1092263D1092273D8F
:100110001092283D0895CF93DF93EC018C819D814F
:10012000880F991F880F991F2091273D3091283DF6
:10013000820F931F8093293D90932A3D44E050E025
:100140006FE27DE30E9466D240912F3D5091303D99
:100150006091313D7091323D49875A876B877C872A
:1001600080E0DF91CF9108958F929F92AF92BF92DE
:10017000CF92DF92EF92FF92CF93DF93EC018091C9
:100180002C32882369F089E0DF91CF91FF90EF90C6
:10019000DF90CF90BF90AF909F908F900C949DA7D1
:1001A00089859A85AB85BC8580932B3D90932C3DAA
:1001B000A0932D3DB0932E3DCE010E948B80809365
:1001C000243D81116EC0C984DA84EB84FC84A701CC
:1001D0009601C701B6010E946BD981112FC046015B
:1001E0005701E894B7F82FEF3FEF4FE75FE7C501FE
:1001F000B4010E946BD981110AC02FEF3FEF4FE786
:100200005FE7C501B4010E94A5D51816BCF0809027
:100210002B3D90902C3DA0902D3DB0902E3DA50102
:100220009401C701B6010E94FCD39F772CEA35ECFC
:1002300047E257E30E94A8D7181674F580912B3D2A
:1002400090912C3DA0912D3DB0912E3D80932F3D5E
:100250009093303DA093313DB093323D8C819D8190
:10026000880F991F880F991F2091273D3091283DB5
:10027000820F931F8093293D90932A3D44E050E0E4
:100280006FE27DE30E94F7D280902B3D90902C3D51
:10029000A0902D3DB0902E3D89869A86AB86BC8677
:1002A00080E0DF91CF91FF90EF90DF90CF90BF90F3
:1002B000AF909F908F9008950E9469B880E0089554
:1002C0008091333D9091343D8F3E924111F08EE507
:1002D00008958091593D90915A3D8F3E9241B9F7D2
:1002E00080915B3D90915C3D8F3E924181F7809182
:1002F000E4549091E5548F3E924149F78091E65441
:100300009091E7548F3E924111F7809179569091E8
:100310007A568F3E9241D9F680E0089594E0899F05
:10032000F0011124ED5CF24C4283538364837583A6
:10033000089594E0899FF0011124EA51FB4A45ABEE
:1003400056AB67AB70AF08955F926F927F928F92BA
:100350009F92AF92BF92CF92DF92EF92FF920F9354
:100360001F93CF93DF93CDB7DEB76097CDBFDEBFCE
:10037000BE016F5F7F4F8BE195E50E948D7FCE01BF
:1003800001964C0183E9A82E85E5B82E93EAC92E83
:1003900095E5D92E23EBE22E25E5F22E03ED15E5AA
:1003A00035EF632E38E5732E512CF40141915191B4
:1003B000619171914F01F501419351936193719353
:1003C0005F01F60141935193619371936F01F701BE
:1003D00041935193619371937F01852D0E94F46F36
:1003E000F80111921192119211928F01F301108272
:1003F0001182128213825394F8E16F0E711C84E013
:100400005812D3CF6096CDBFDEBFDF91CF911F9141
:100410000F91FF90EF90DF90CF90BF90AF909F90A3
:100420008F907F906F905F90089580915D3D0895CB
:100430001F93CF93DF938BE897E1EBE5FDE3DF01BB
:100440009C011D9221503040E1F78FEE92E18093A4
:100450005B3D90935C3D8093E4549093E554C4E6F7
:10046000DDE3C0935E3DD0935F3DC093603DD0938C
:10047000613DC093623DD093633D81E090E068E2CE
:1004800074E520E030E01CEB129FA001139F500D9B
:100490001124FA01E55AF24CD90111961A9F9001E4
:1004A0001B9F300D11242C59324C238734876187D0
:1004B0007287BA016C59724C9C0101968032910589
:1004C00019F78CEB829FF001839FF00D1124E55A00
:1004D000F24CC387D4876187728780E280935D3D49
:1004E000DF91CF911F910895CF93DF93E6EEF4E56E
:1004F00085E991E0DF01EC011D922197E9F7A3E383
:10050000BDE388E2ED0119928A95E9F78FEE92E159
:100510008D939C938093593D90935A3D8083918312
:100520008093795690937A56DF91CF910C941882EC
:100530000E94918C0E94188280E00C94304AE091D5
:100540005E3DF0915F3D848581111BC02281338126
:10055000808191814CEBDF011D924A95E9F722835E
:1005600033838083918381E0848780915D3D8150D6
:1005700080935D3D8281938180935E3D90935F3D4A
:1005800005C08CE10E949DA7E0E0F0E0CF01089556
:10059000A0E6BDE3ED91FC911197858781E0878707
:1005A00082E08487828193818D939C9381E00E9475
:1005B000C5AB0C94AFB5EF92FF920F931F93CF93FF
:1005C000DF9300D01F92CDB7DEB78C014B835C83E5
:1005D00069837A830E949F82FC014B815C816981DF
:1005E0007A81009761F48EE02496CDBFDEBFDF9163
:1005F000CF911F910F91FF90EF900C946F4E83E07D
:1006000085878CE591E884839583068317838B0126
:100610007A0126E0D8014D915D916D917D918D011A
:10062000CF0185599F4FDC014D935D936D937C9372
:100630001397D7014D915D916D917D917D01418B16
:10064000528B638B748B215034962111E3CF83E05E
:100650002496CDBFDEBFDF91CF911F910F91FF9008
:10066000EF900C94C882CF92DF92EF92FF926B01D1
:100670007C010E949F82009739F48EE0FF90EF90FA
:10068000DF90CF900C946F4E26EB33E8FC0124836F
:100690003583E556FF4FC082D182E282F38221E0AA
:1006A000FC01278782E00E94C88280E0FF90EF90E3
:1006B000DF90CF9008958091623D9091633DFC0161
:1006C00024853EEF320F323018F424E02487089559
:1006D000243011F080E090E00895E091623DF091C7
:1006E000633D22813381808191814CEBDF011D923A
:1006F0004A95E9F72283338380839183E091623DB9
:10070000F091633D0280F381E02DE093623DF09330
:10071000633D8485823011F483E0848780915D3D60
:100720008F5F80935D3D8FEF0E94C5AB81E040916C
:100730005E3D50915F3D2091623D3091633D421797
:10074000530709F080E00895BC016F5E7F4FDC0124
:100750001696ED91FC91179785599F4F19950E9418
:100760006D8381110E94DD5580E0089585569F4F6D
:1007700020E034E244E759E4FC0160817181828128
:1007800093810E944AD80E9419D60E9445D60E94A1
:1007900073B80E946D8381110E94DD5580E0089539
:1007A0008091623D9091633DFC0124853EEF320FC4
:1007B000323018F424E024870895243011F080E0CA
:1007C00090E00895CF93DF93C091623DD091633D57
:1007D0008C859EEF980F923018F484E08C8705C0CA
:1007E000843019F080E090E010C02097D9F3DE014A
:1007F0001296ED91FC9113978785882329F0EC17C9
:10080000FD0711F0DF01F4CFCD01DF91CF91089505
:10081000CF93DF93EC012A813B81888199814CEB56
:10082000FB01DE0101900D924A95E1F72A833B839B
:1008300088839983DF91CF9108958FEE92E1809321
:100840007B5690937C5680933857909339570895F0
:100850002F923F924F925F926F927F928F929F92D0
:10086000AF92BF92CF92DF92EF92FF920F931F93BE
:10087000CF93DF93CDB7DEB76A97CDBFDEBF4C0114
:100880001B0129013A01E986FA860B871C871A2D7C
:100890000B2DE8A8B9A8AAA82BA929838091A43276
:1008A000882399F08091983290919932A0919A3250
:1008B000B0919B32BC01CD019F772CEA35EC47E229
:1008C00057E30E94A5D587FD11C78091CF33909142
:1008D000D033A091D133B091D233BC01CD019F77F9
:1008E00031E03D832CEA35EC47E257E30E94A8D77C
:1008F000181614F01D8210C02DEC3CEC4CEC5DE39E
:100900006091743370917533809176339091773321
:100910000E94A5D587FDECC6F10180819181A2815D
:10092000B381BC01CD019F77F1E0FD872CEA35EC66
:1009300047E257E30E94A8D718160CF01D86F10174
:1009400084819581A681B781BC01CD019F77F1E0BB
:10095000F98B2CEA35EC47E257E30E94A8D718162A
:100960000CF0198AF10180859185A285B3852091CB
:10097000D3333091D4334091D5335091D6332E8B2D
:100980003F8B488F598F2091D7333091D833409186
:10099000D9335091DA332A8B3B8B4C8B5D8B409152
:1009A000DB335091DC336091DD337091DE33F090B6
:1009B000A532F11021C01092C35681E08093C45635
:1009C00082E08093C5563D81332341F04D8541112E
:1009D00095C65989511192C68CE9C1C6CB01BA019D
:1009E0009F772CEA35EC47E257E30E94A8D7181608
:1009F0000CF089C68BE9B3C6BC01CD019F77A1E09D
:100A0000AA8F2CEA35EC47E257E30E94A8D71816C4
:100A10000CF01A8EB1E0FB1216C01092C35682E0A1
:100A20008093C456F092C556ED81EE2339F0FD85D2
:100A3000F11164C62A8D222379F260C66A897B8906
:100A40008C899D89CDCF32E0F31217C081E080936D
:100A5000C356F092C4561092C5564D81442341F0BE
:100A6000598951114BC68A8D882309F4B5CF46C6E2
:100A70006E897F89888D998DB3CFB101C4010E94A1
:100A80007F4C9D81992309F451C0209160323091AF
:100A9000613240916232509163326091B53270910F
:100AA000B6328091B7329091B8320E94FCD39F77D2
:100AB0002CEA35EC47E257E30E94A5D587FF36C004
:100AC00020916432309165324091663250916732A4
:100AD0006091B9327091BA328091BB329091BC3240
:100AE0000E94FCD39F772CEA35EC47E257E30E9443
:100AF000A5D587FF1BC020916832309169324091A3
:100B00006A3250916B326091BD327091BE328091E9
:100B1000BF329091C0320E94FCD39F772CEA35EC13
:100B200047E257E30E94A5D587FDE4C58CA98093D1
:100B30005F328BE592E30E94874A86E5EBE5F2E3BC
:100B4000A2EEB6E501900D928A95E1F788E1E5EB1A
:100B5000F2E3AEE7B6E501900D928A95E1F7809158
:100B6000A6328111D5C523E333E34BEC51E46E2D5E
:100B70007B2D8A2D99810E944AD84B015C0160939C
:100B8000AE567093AF568093B0569093B15623E310
:100B900033E34BEC51E4C301B2010E944AD86093A5
:100BA000965670939756809398569093995623E350
:100BB00033E34BEC51E469857A858B859C850E94F3
:100BC0004AD860939A5670939B5680939C56909304
:100BD0009D5623E333E34BEC51E4612F702FC601A4
:100BE0000E944AD8162F072F412F502FBC01409347
:100BF0009E5650939F566093A0567093A156809135
:100C0000703390917133A0917233B0917333BC0102
:100C1000CD019F770E9482D60E9419D66093BF565D
:100C20007093C0568093C1569093C256A091C356FC
:100C3000A98BB091C456BA8BEB2FF0E0ED83FE8305
:100C40007F01EE0CFF1CEE0CFF1CF101EE0DFF1DF1
:100C500080819181A281B381BC01CD019F772CEA73
:100C600035EC47E257E30E94A5D5D82EDD1CDD24E4
:100C7000DD1C3989232F30E029833A838901000F55
:100C8000111F000F111FF101E00FF11F80819181F1
:100C9000A281B381BC01CD019F772CEA35EC47E2FC
:100CA00057E30E94A5D5881F8827881F8D21809330
:100CB000BE562CEA35EC47E257E3C501B4019F77F5
:100CC0000E94A8D718160CF0F9C0F801E05AFD4CA4
:100CD000D801AB54BD4C2D913D914D915C916081FB
:100CE0007181828193810E94FCD36B017C01ED8133
:100CF000FE81EE0FFF1FEE0FFF1FE05AFD4CAD818E
:100D0000BE81AA0FBB1FAA0FBB1FAB54BD4C2D91B8
:100D10003D914D915C9160817181828193810E94AE
:100D2000FCD369877A878B879C87A5019401C501CD
:100D3000B4010E944AD820E030E040E850E40E942C
:100D40004AD86D877E878F87988BA7019601C70148
:100D5000B6010E944AD82B013C0129853A854B8572
:100D60005C85CA01B9010E944AD89B01AC01C3014C
:100D7000B2010E94FDD39B01AC016D857E858F85FC
:100D800098890E94FCD32B013C0120E030E0A901AE
:100D90000E94A8D71816C4F4C301B2010E9423D937
:100DA0002B013C0129853A854B855C85C701B6013D
:100DB0000E94B5D79B01AC01C301B20190580E94BB
:100DC000ACD52B013C0103C0412C512C3201809148
:100DD0005F32833021F477FA709477F8709420E0D2
:100DE00030E0A901C501B4010E94A5D587FF04C068
:100DF00077FA709477F8709409811A81000F111FA7
:100E0000000F111FA8014558594A5A01A301920128
:100E100069857A858B859C850E944AD89B01AC01A7
:100E2000C701B6010E94FCD320E030E040E05FE360
:100E30000E944AD8D5015B966D937D938D939C93C8
:100E40005E97AD80BE80AA0CBB1CAA0CBB1CF50132
:100E5000E558F94A4F01A3019201C701B6010E946A
:100E60004AD89B01AC0169857A858B859C850E9457
:100E7000FDD320E030E040E05FE30E944AD8D40197
:100E80005B966D937D938D939C935E97E091C55691
:100E9000F0E0EE0FFF1FEE0FFF1FE558F94A138E2B
:100EA000148E158E168EB091AE56B987E091AF565E
:100EB000ED872090B0563090B15625C05701F7010C
:100EC000E558F94A838D948DA58DB68D9C01AD01B1
:100ED0005058F801E558F94A838D948DA58DB68D4B
:100EE000BC01CD0190580E94B5D79B01AB01BC015C
:100EF0004093AE565093AF566093B0567093B15630
:100F000029873D871C01D801A558B94A5B96CD9029
:100F1000DD90ED90FC905E97E981FA81EE0FFF1F66
:100F2000EE0FFF1FE951F94A13962D913D914D9116
:100F30005C91169760817181828193810E94FCD3BC
:100F4000A70196010E94FCD369837A838B839C83DB
:100F5000D501A558B94A5B964D905D906D907C90F7
:100F60005E97ED81FE81EE0FFF1FEE0FFF1FE9512F
:100F7000F94A13962D913D914D915C9116976081A0
:100F80007181828193810E94FCD3A30192010E940E
:100F9000FCD36D837E838F8398879B01AC0169812D
:100FA0007A818B819C810E94B5D729853D85A101DD
:100FB0000E94FCD34B015C01E894B7F820E030E0DC
:100FC00040E85FE3C501B4010E94A8D718160CF4ED
:100FD000C3C32AE037ED43EA5BE3C501B4010E94D5
:100FE000A8D7181694F42FE632E143E85AE369854E
:100FF0007D85C1010E944AD89B01AC01C501B401A5
:101000000E94A8D718160CF4A7C3A3019201505848
:10101000C701B60190580E9470D44B015C016093E7
:10102000A6567093A7568093A8569093A956809180
:10103000A532813039F4412C512C30E8632E3FEB3E
:10104000732E06C0412C512C20E8622E2FE3722E05
:101050008091BE568823D1F16091BF567091C056E1
:101060008091C1569091C2560E9445D66B017C0179
:101070002CEA35EC47E257E30E94A5D587FD10C066
:1010800010915F322BED3FE049EC50E4C701B6010F
:101090000E944AD89B01AC01C12CD12C7601B9C069
:1010A00081E090E0A0E0B0E08093BF569093C056FE
:1010B000A093C156B093C25610915F322BED3FE022
:1010C00049EC50E4C12CD12C7601A3C02D813E8186
:1010D0004F81588569817A818B819C810E9470D46F
:1010E00069837A838B839C836093AA567093AB56F3
:1010F0008093AC569093AD56A50194010E94FCD309
:101100006B017C019F772CEA35EC47E257E30E94A4
:10111000A5D587FF18C010915F326091BF567091BE
:10112000C0568091C1569091C2560E9445D62BED73
:101130003FE049EC50E40E944AD89B01AC01C12C2D
:10114000D12C760166C029813A814B815C81C50131
:10115000B4010E94A8D71816F4F42BED3FE049EC37
:1011600050E4C301B2010E944AD89B01AC016981DD
:101170007A818B819C810E94FDD36093AA567093E3
:10118000AB568093AC569093AD56A50194010E9446
:10119000FCD36B017C0110915F32133099F06091A8
:1011A000BF567091C0568091C1569091C2560E9410
:1011B00045D62BED3FE049EC50E40E944AD89B0114
:1011C000AC0127C02BED3FE049EC50E4C301B20174
:1011D0000E944AD89B01AC01C701B6010E94FCD312
:1011E0007B018C016091BF567091C0568091C156B1
:1011F0009091C2560E9445D62BED3FE049EC50E459
:101200000E944AD89B01AC01C701D8016C017D0145
:101210000BC0123049F4C301B2010E944AD8A701A1
:1012200096010E94FDD30AC0C301B2010E944AD8B0
:101230009B01AC01C701B6010E94FCD37B01AB014D
:10124000BC014093B2565093B3566093B45670931A
:10125000B5568C015090C556A52DB0E0FD01EE0F9E
:10126000FF1FEE0FFF1FE951F94AAA0FBB1FAA0F7C
:10127000BB1FA558B94A13962D913D914D915C9194
:10128000169760817181828193810E94FCD34B010A
:101290005C016093B6567093B7568093B85690939E
:1012A000B9569701A80169857D85C1010E944AD878
:1012B0006B017C016093BA567093BB568093BC5609
:1012C0009093BD56A50194010E94B5D769837A8396
:1012D0008B839C836093A2567093A3568093A456ED
:1012E0009093A5568091A432811117C0F091983245
:1012F000FD834090993220919A322E8B30919B320F
:101300003A8F109298321092993210929A3210922B
:101310009B3281E08093A43212C0209198323091A8
:10132000993240919A3250919B3269817A818B81B6
:101330009C810E94ACD56D83472E8E8B9A8F5989E4
:1013400045E3549FF0011124E351FF4C208131818A
:1013500042815381C701B6010E94ACD5662E072F8A
:10136000182F792E2D81342D4E895A8D0E94A5D5A6
:1013700087FF04C06D80042D1E897A8C9A8985E3CD
:10138000989FF0011124E351FF4C2081318142816B
:101390005381C701B6010E94ACD56B017C019B0152
:1013A000AC01662D702F812F972D0E94A8D718169B
:1013B00024F06C2C0D2D1E2D7F2C862D902FA12F0F
:1013C000B72D8093C6569093C756A093C856B09336
:1013D000C95620E030E0A901C501B4019F770E9401
:1013E000A8D7181684F5A5E35A9EF0011124E351FD
:1013F000FF4C2081318142815381C501B4010E949B
:10140000ACD54B015C01E894B7F8A5019401662DB9
:10141000702F812F972D0E94A8D7181614F4A72C8F
:1014200004C0682C092D1A2DAB2C862D902FA12FCE
:10143000BA2D8093C6569093C756A093C856B093C2
:10144000C956B62C02C0B62CA72CC0902E30D09016
:101450002F30E0903030F090313020E030E040E844
:1014600050E4C701B6010E944AD82B013C012985EE
:101470003D85A10169857D85C1010E94FDD3A7013C
:1014800096010E94FCD39B01AC01C301B2010E94F2
:101490004AD80E9423D92B013C0120EC31EE44E6CE
:1014A0005CE46B2D702F812F9A2D0E944AD820E08A
:1014B00030E44CE156E40E94ACD56B017C012091F4
:1014C0003730309138304091393050913A3069811D
:1014D0007A818B819C810E94ACD54B015C01A30178
:1014E000920169817A818B819C810E94ACD58701B0
:1014F0007601A50194010E940AC30E9482D67B0155
:101500008C0120E030E040E85FE30E94A8D7181685
:101510003CF4B701C8010E9414D64B015C0108C01D
:10152000812C912C54018394E12CF12C00E81FE3D1
:10153000C701D8018093CA569093CB56A093CC563E
:10154000B093CD569701A8016091C6567091C756C9
:101550008091C8569091C9560E94ACD56093175798
:10156000709318578093195790931A578092CE56BC
:101570009092CF56A092D056B092D1569701A80122
:101580006091B2567091B3568091B4569091B55611
:101590000E94ACD56093D2567093D3568093D456A4
:1015A0009093D5569701A8016091B6567091B756A1
:1015B0008091B8569091B9560E94ACD56093D6569A
:1015C0007093D7568093D8569093D9568090A6564C
:1015D0009090A756A090A856B090A956C501B40106
:1015E0000E9419D9C090AE56D090AF56E090B05638
:1015F000F090B1560091C35610E0000F111F000F7C
:10160000111F0558194AA70196010E944AD89B014B
:10161000AC01F80163817481858196810E94FCD3BD
:101620006093DA567093DB568093DC569093DD56C8
:10163000C501B4010E94A9D59B01AC010091C4561B
:1016400010E0000F111F000F111F0558194AC701A4
:10165000B6010E944AD89B01AC01D80113966D9146
:101660007D918D919C9116970E94FCD36093DE56DC
:101670007093DF568093E0569093E156A091C55643
:10168000B0E0FD01EE0FFF1FEE0FFF1FE951F94A19
:10169000AA0FBB1FAA0FBB1FA558B94A13968D915D
:1016A0009D910D90BC91A02D80839183A283B383E3
:1016B0001092243D8091A2569091A356A091A456D9
:1016C000B091A556BC01CD019F772CEA35EC47E2DD
:1016D00057E30E94A5D587FD0FC00E94D05582E038
:1016E00080937D560E94E24B80E039C08EE837C07F
:1016F0008EE935C08FE933C089EC31C0B101C40136
:101700000E947F4CC2C9B101C4010E947F4C0ECA25
:101710008E2D9B2DAA2DB9818093AE569093AF56F6
:10172000A093B056B093B1564092965650929756A9
:10173000609298567092995629853A854B855C85BA
:1017400020939A5630939B5640939C5650939D56A7
:101750004C015D01C60148CA8BE98093243D6A961D
:10176000CDBFDEBFDF91CF911F910F91FF90EF9022
:10177000DF90CF90BF90AF909F908F907F906F90B1
:101780005F904F903F902F9008958F929F92AF92CD
:10179000BF92CF92DF92EF92FF92CF93DF9380912F
:1017A0007D56882309F4B1C00E941582843010F45C
:1017B00082E0ACC02091D2563091D3564091D4569D
:1017C0005091D5566091A6567091A7568091A85613
:1017D0009091A9560E94FDD36B017C016093A6569F
:1017E0007093A7568093A8569093A9560E9419D932
:1017F0008090AE569090AF56A090B056B090B15633
:10180000C091C356D0E0CC0FDD1FCC0FDD1FC951F6
:10181000D94AA50194010E944AD89B01AC0160916C
:10182000DA567091DB568091DC569091DD560E941D
:10183000FDD3688379838A839B83C701B6010E94A5
:10184000A9D59B01AC01C091C456D0E0CC0FDD1FDF
:10185000CC0FDD1FC951D94AC501B4010E944AD835
:101860009B01AC016091DE567091DF568091E0568D
:101870009091E1560E94FDD3688379838A839B838C
:10188000C091C556D0E0CC0FDD1FCC0FDD1FC95174
:10189000D94A2091D6563091D7564091D85650917A
:1018A000D956688179818A819B810E94FDD36883A2
:1018B00079838A839B8382EE96E50E94A79688E1CE
:1018C000E7EEF6E5AEE7B6E501900D928A95E1F711
:1018D0008091CE569091CF56A091D056B091D156CE
:1018E0000197A109B1098093CE569093CF56A0934A
:1018F000D056B093D156181619061A061B060CF4CA
:1019000057CF10927D5680E001C083E0DF91CF91E8
:10191000FF90EF90DF90CF90BF90AF909F908F900F
:10192000089510927D5608954F925F926F927F9224
:101930008F929F92AF92BF92CF92DF92EF92FF92DF
:10194000CF93DF93CDB7DEB76497CDBFDEBF69839A
:101950007A838B839C8369017A0120E030E040E741
:1019600051E40E944AD84B015C0120E030E040E79E
:1019700051E4C701B6010E944AD89B01AC01C501E0
:10198000B4010E94FCD36D877E878F87988B20E0FF
:1019900030E040E251EC69817A818B819C810E9428
:1019A0004AD84B015C0120E030E040E251E4C7013D
:1019B000B6010E944AD89B01AC01C501B4010E9446
:1019C000FDD3698B7A8B8B8B9C8B2091FB5530914F
:1019D000FC554091FD555091FE5560E070E080E867
:1019E0009FE30E94ACD54B015C0120E030E040EC6D
:1019F00050EC69817A818B819C810E944AD82B01AD
:101A00003C0120E030E040EC50E4C701B6010E9408
:101A10004AD89B01AC01C301B2010E94FDD3A501CC
:101A200094010E944AD8A50194010E944AD8A501B8
:101A300094010E944AD8A50194010E944AD8A501A8
:101A400094010E944AD86B017C01A50194016D8527
:101A50007E858F8598890E944AD8A50194010E94AD
:101A60004AD8A50194010E944AD8A50194010E9478
:101A70004AD86D837E838F839887A50194016989F5
:101A80007A898B899C890E944AD8A50194010E9479
:101A90004AD8A50194010E944AD869877A878B8722
:101AA0009C8720E030E042EF50E4C701B6010E947D
:101AB0004AD82B013C0120E030E040EA50E46D813F
:101AC0007E818F8198850E944AD89B01AC01C30119
:101AD000B2010E94FDD32B013C0120E030E040E543
:101AE00050E469857A858B859C850E944AD89B0144
:101AF000AC01C301B2010E94FDD360931F567093E5
:101B00002056809321569093225620E030E045EAFB
:101B100052E4C701B6010E944AD82B013C0120E0E3
:101B200030E048EE51E46D817E818F8198850E947E
:101B30004AD89B01AC01C301B2010E94FDD32B0125
:101B40003C0120E030E040E151E469857A858B85F5
:101B50009C850E944AD89B01AC01C301B2010E943E
:101B6000FDD360931B5670931C5680931D56909323
:101B70001E5620E030E04FE753E4C701B6010E9453
:101B80004AD82B013C0120E030E040E452E46D8172
:101B90007E818F8198850E944AD89B01AC01C30148
:101BA000B2010E94FDD32B013C0120E030E040EC6B
:101BB00050E469857A858B859C850E944AD89B0173
:101BC000AC01C301B2010E94FDD36093175670931C
:101BD00018568093195690931A5620E030E046E943
:101BE00053E4C701B6010E944AD82B013C0120E012
:101BF00030E040EC51E46D817E818F8198850E94B8
:101C00004AD89B01AC01C301B2010E94FDD360938D
